:04000003F000B2CD8A
:020000040000FA
:1000000000040020810A000015070000610A0000BA
:100010001F07000029070000330700000000000050
:10002000000000000000000000000000A50A000021
:100030003D070000000000004707000051070000D6
:100040005B070000650700006F07000079070000EC
:10005000830700008D07000097070000A10700003C
:10006000AB070000B5070000BF070000C90700008C
:10007000D3070000DD070000E7070000F1070000DC
:10008000FB070000050800000F0800001908000029
:10009000230800002D080000370800004108000078
:1000A0004B080000550800005F08000069080000C8
:1000B000730800007D080000870800009108000018
:1000C0009B080000A5080000AF080000B908000068
:1000D000C3080000CD080000D7080000E1080000B8
:1000E000EB080000F5080000FF0800000909000007
:1000F000130900001D090000270900003109000054
:100100003B0900001FB500F003F88DE80F001FBD8C
:1001100000F0ACBC40F6FC7108684FF01022401CA7
:1001200008D00868401C09D00868401C04D0086842
:1001300000F037BA9069F5E79069F9E7704770B554
:100140000B46010B184400F6FF70040B4FF0805073
:100150000022090303692403406943431D1B104621
:1001600000F048FA29462046BDE8704000F042BA47
:10017000F0B54FF6FF734FF4B4751A466E1E11E0DA
:10018000A94201D3344600E00C46091B30F8027B3B
:10019000641E3B441A44F9D19CB204EB134394B25D
:1001A00004EB12420029EBD198B200EB134002EBB2
:1001B000124140EA0140F0BDF34992B00446D1E952
:1001C0000001CDE91001FF224021684600F0F4FB58
:1001D00094E80F008DE80F00684610A902E004C8FB
:1001E00041F8042D8842FAD110216846FFF7C0FF7C
:1001F0001090AA208DF8440000F099F9FFF78AFFCB
:1002000040F6FC7420684FF01025401C0FD0206889
:1002100010226946803000F078F92068401C08D030
:100220002068082210A900F070F900F061F9A869AF
:10023000EEE7A869F5E74FF080500369406940F6A2
:10024000FC71434308684FF01022401C06D0086838
:1002500000F58050834203D2092070479069F7E788
:100260000868401C04D00868401C03D00020704778
:100270009069F9E70420704770B504460068C34DE3
:10028000072876D2DFE800F033041929631E250021
:10029000D4E9026564682946304600F062F92A46CE
:1002A0002146304600F031F9AA002146304600F0E0
:1002B00057FB002800D0032070BD00F009FC4FF46C
:1002C000805007E0201D00F040F90028F4D100F034
:1002D000FFFB60682860002070BD241D94E80700C3
:1002E000920000F03DFB0028F6D00E2070BDFFF715
:1002F000A2FF0028FAD1D4E901034FF0805100EBAE
:10030000830208694D69684382420ED840F6F8704E
:1003100005684FF010226D1C09D0056805EB8305B8
:100320000B6949694B439D4203D9092070BD55694A
:10033000F4E70168491C03D00068401C02D003E0C8
:100340005069FAE70F2070BD2046FFF735FFFFF731
:1003500072FF0028F7D1201D00F0F7F80028F2D135
:1003600060680028F0D100F0E2F8FFF7D3FE00F05B
:10037000BFF8072070BD10B50C46182802D0012028
:10038000086010BD2068FFF777FF206010BD41684E
:10039000054609B1012700E0002740F6F8742068FF
:1003A0004FF01026401C2BD02068AA68920000F065
:1003B000D7FA38B3A86881002068401C27D020688D
:1003C000FFF7BDFED7B12068401C22D026684FF051
:1003D0008050AC686D68016942695143A9420DD9EA
:1003E000016940694143A14208D92146304600F0E5
:1003F000B8F822462946304600F087F800F078F831
:100400007069D2E700F093F8FFF784FEF6E77069B1
:10041000D6E77669DBE740F6FC7420684FF01026DB
:10042000401C23D02068401C0CD02068401C1FD0EA
:100430002568206805F18005401C1BD027683879A5
:10044000AA2819D040F6F8700168491C42D001680A
:10045000491C45D00168491C3ED001680968491C07
:100460003ED00168491C39D000683EE0B069DAE747
:10047000B569DEE7B769E2E710212846FFF778FEA5
:100480003968814222D12068401C05D0D4F8001080
:1004900001F18002C03107E0B169F9E730B108CA63
:1004A00051F8040D984201D1012000E000208A4259
:1004B000F4D158B1286810B1042803D0FEE72846CB
:1004C000FFF765FF3149686808600EE0FFF722FE1C
:1004D00000F00EF87169BBE77169BFE7706904E06D
:1004E0004FF480500168491C01D000F0CBFAFEE7C0
:1004F000BFF34F8F26480168264A01F4E06111439B
:100500000160BFF34F8F00BFFDE72DE9F0411746B3
:100510000D460646002406E03046296800F054F8EF
:10052000641C2D1D361DBC42F6D3BDE8F08140F69B
:10053000FC700168491C04D0D0F800004FF48051D1
:10054000FDE54FF010208069F8E74FF080510A690F
:10055000496900684A43824201D810207047002050
:10056000704770B50C4605464FF4806608E0284693
:1005700000F017F8B44205D3A4F5806405F5805562
:10058000002CF4D170BD0000F40A0000000000202F
:100590000CED00E00400FA05144801680029FCD0C5
:1005A0007047134A0221116010490B68002BFCD0E0
:1005B0000F4B1B1D186008680028FCD0002010603D
:1005C00008680028FCD07047094B10B501221A605A
:1005D000064A1468002CFCD0016010680028FCD08A
:1005E0000020186010680028FCD010BD00E4014015
:1005F00004E5014070B50C46054600F073F810B9EB
:1006000000F07EF828B121462846BDE8704000F091
:1006100007B821462846BDE8704000F037B8000012
:100620007FB5002200920192029203920A0B000B06
:100630006946012302440AE0440900F01F0651F80C
:10064000245003FA06F6354341F82450401C8242F8
:10065000F2D80D490868009A10430860081D016827
:10066000019A1143016000F03DF800280AD00649C4
:1006700010310868029A10430860091D0868039A3F
:10068000104308607FBD00000006004030B50F4CED
:10069000002200BF04EB0213D3F800582DB9D3F8A1
:1006A000045815B9D3F808581DB1521C082AF1D3C3
:1006B00030BD082AFCD204EB0212C2F80008C3F8CD
:1006C00004180220C3F8080830BD000000E0014013
:1006D0004FF08050D0F83001082801D0002070473A
:1006E000012070474FF08050D0F83011062905D016
:1006F000D0F83001401C01D0002070470120704725
:100700004FF08050D0F830010A2801D00020704707
:100710000120704708208F490968095808471020B0
:100720008C4909680958084714208A4909680958FA
:100730000847182087490968095808473020854923
:100740000968095808473820824909680958084744
:100750003C20804909680958084740207D490968BC
:100760000958084744207B49096809580847482028
:1007700078490968095808474C207649096809589A
:10078000084750207349096809580847542071499F
:1007900009680958084758206E49096809580847E8
:1007A0005C206C4909680958084760206949096854
:1007B00009580847642067490968095808476820AC
:1007C00064490968095808476C2062490968095852
:1007D000084770205F4909680958084774205D4937
:1007E00009680958084778205A490968095808478C
:1007F0007C205849096809580847802055490968EC
:10080000095808478420534909680958084788202F
:1008100050490968095808478C204E490968095809
:10082000084790204B4909680958084794204949CE
:10083000096809580847982046490968095808472F
:100840009C204449096809580847A0204149096883
:1008500009580847A4203F49096809580847A820B3
:100860003C49096809580847AC203A4909680958C1
:100870000847B0203749096809580847B420354966
:10088000096809580847B8203249096809580847D3
:10089000BC203049096809580847C0202D4909681B
:1008A00009580847C4202B49096809580847C82037
:1008B0002849096809580847CC2026490968095879
:1008C0000847D0202349096809580847D4202149FE
:1008D000096809580847D8201E4909680958084777
:1008E000DC201C49096809580847E02019490968B3
:1008F00009580847E4201749096809580847E820BB
:100900001449096809580847EC2012490968095830
:100910000847F0200F49096809580847F4200D4995
:10092000096809580847F8200A490968095808471A
:10093000FC2008490968095808475FF48070054998
:10094000096809580847000003480449024A034B54
:100950007047000000000020000B0000000B0000AA
:1009600040EA010310B59B070FD1042A0DD310C82C
:1009700008C9121F9C42F8D020BA19BA884201D97E
:10098000012010BD4FF0FF3010BD1AB1D30703D0C6
:10099000521C07E0002010BD10F8013B11F8014B7C
:1009A0001B1B07D110F8013B11F8014B1B1B01D198
:1009B000921EF1D1184610BD02F0FF0343EA032254
:1009C00042EA024200F005B87047704770474FF0A6
:1009D00000020429C0F0128010F0030C00F01B800C
:1009E000CCF1040CBCF1020F18BF00F8012BA8BF1A
:1009F00020F8022BA1EB0C0100F00DB85FEAC17CDE
:100A000024BF00F8012B00F8012B48BF00F8012B90
:100A100070474FF0000200B51346944696462039C1
:100A200022BFA0E80C50A0E80C50B1F12001BFF4A7
:100A3000F7AF090728BFA0E80C5048BF0CC05DF80D
:100A400004EB890028BF40F8042B08BF704748BF5B
:100A500020F8022B11F0804F18BF00F8012B7047CF
:100A6000014B1B68DB6818470000002009480A4951
:100A70007047FFF7FBFFFFF745FB00BD20BFFDE719
:100A8000064B1847064A1060016881F308884068E1
:100A900000470000000B0000000B000017040000DE
:100AA000000000201EF0040F0CBFEFF30881EFF3ED
:100AB0000981886902380078182803D100E0000015
:100AC000074A1047074A12682C3212681047000084
:100AD00000B5054B1B68054A9B58984700BD0000B0
:100AE0007703000000000020F00A0000040000006E
:100AF000001000000000000000FFFFFF0090D00386
:10100000C8130020395E020085C100009F5D020008
:1010100085C1000085C1000085C1000000000000FE
:10102000000000000000000000000000C55E02009B
:1010300085C100000000000085C1000085C10000DE
:101040002D5F0200335F020085C1000085C10000F2
:1010500085C1000085C1000085C1000085C1000078
:10106000395F020085C1000085C100003F5F0200BA
:1010700085C10000455F02004B5F0200515F020026
:1010800085C1000085C1000085C1000085C1000048
:1010900085C1000085C1000085C1000085C1000038
:1010A00085C10000575F020085C1000085C10000B6
:1010B00085C1000085C1000085C1000085C1000018
:1010C0005D5F020085C1000085C1000085C1000090
:1010D00085C1000085C1000085C1000085C10000F8
:1010E00085C1000085C1000085C1000085C10000E8
:1010F00085C1000085C1000085C1000085C10000D8
:1011000085C1000085C1000000F002F824F083FED4
:101110000AA090E8000C82448344AAF10107DA4552
:1011200001D124F078FEAFF2090EBAE80F0013F0F7
:10113000010F18BFFB1A43F00103184718530200B0
:10114000385302000A444FF0000C10F8013B13F032
:10115000070408BF10F8014B1D1108BF10F8015B10
:10116000641E05D010F8016B641E01F8016BF9D103
:1011700013F0080F1EBF10F8014BAD1C0C1B09D15A
:101180006D1E58BF01F801CBFAD505E014F8016BCC
:1011900001F8016B6D1EF9D59142D6D3704700005E
:1011A0000023002400250026103A28BF78C1FBD870
:1011B000520728BF30C148BF0B6070471FB500F011
:1011C00003F88DE80F001FBD24F022BE70B51A4C45
:1011D00005460A202070A01C00F0D5F85920A080F8
:1011E00029462046BDE8704008F082B908F08BB966
:1011F00070B50C461149097829B1A0F160015E294A
:1012000008D3012013E0602804D0692802D043F2FB
:1012100001000CE020CC0A4E94E80E0006EB8000A2
:10122000A0F58050241FD0F8806E2846B04720607B
:1012300070BD012070470000080000201C00002045
:10124000A05F02003249884201D20120704700208D
:10125000704770B50446A0F500002E4EB0F1786FCF
:1012600002D23444A4F500042948844201D2012565
:1012700000E0002500F043F848B125B9B44204D39A
:101280002548006808E0012070BD002070BD002DD9
:10129000F9D1B442F9D321488442F6D2F3E710B52C
:1012A0000446A0F50000B0F1786F03D21948044459
:1012B000A4F5000400F023F84FF0804130B1164847
:1012C000006804E08C4204D2012003E01348844209
:1012D000F8D2002080F0010010BD10B520B1FFF75A
:1012E000DEFF08B1012010BD002010BD10B520B1F7
:1012F000FFF7AFFF08B1012010BD002010BD084866
:1013000008490068884201D10120704700207047D9
:1013100000700200000000202000002008000020D3
:101320005C000020BEBAFECA10B5044600210120B0
:1013300000F042F800210B2000F03EF800210820C8
:1013400000F03AF80421192000F036F804210D20AD
:1013500000F032F804210E2000F02EF804210F20B6
:1013600000F02AF80421C84300F026F806211620D0
:1013700000F022F80621152000F01EF82046FFF7A5
:1013800025FF002010BD40F2231101807047FFF7B8
:101390002DBF1148704710487047104A10B51468A7
:1013A0000E4B0F4A08331A60FFF722FF0B48001D4F
:1013B000046010BD704770474907090E002804DB20
:1013C00000F1E02080F80014704700F00F0000F1F9
:1013D000E02080F8141D704703F900421005024018
:1013E00001000001FD48002101604160018170475A
:1013F0002DE9FF4F93B09B46209F160004460DD069
:101400001046FFF726FF18B1102017B0BDE8F08F87
:101410003146012001F0D3FE0028F6D101258DF8D8
:1014200042504FF4C050ADF84000002210A92846A9
:1014300006F0C5FC0028E8D18DF84250A8464FF4CC
:1014400028500025ADF840001C2229466846079523
:101450000DF01DF89DF81C000DF11C0A20F00F0086
:10146000401C20F0F00010308DF81C0020788DF822
:101470001D0061789DF81E000DF1400961F34200E6
:1014800040F001008DF81E009DF8000008AA40F011
:1014900002008DF800002089ADF83000ADF8325020
:1014A0006089ADF83400CDF82CA060680E900AA9D0
:1014B000CDF82890684606F090FA0028A5D160681B
:1014C000FFF70BFF40B16068FFF710FF20B96078AD
:1014D00000F00300022801D0012000E00020BF4CF2
:1014E00008AA0AA92072BDF8200020808DF8428049
:1014F00042F60120ADF840009DF81E0020F00600E5
:10150000801C20F001008DF81E000220ADF8300094
:10151000ADF8340014A80E90684606F05EFA002874
:1015200089D1BDF82000608036B1211D304600F021
:101530005FF90028C2D109E0BBF1000F05D00CF023
:1015400021FDE8BB0CF01EFDD0BBA58017B1012F1B
:1015500043D04AE08DF8428042F6A620ADF8400024
:1015600046461C220021684607950CF090FF9DF826
:101570001C00ADF8346020F00F00401C20F0F0009B
:1015800010308DF81C009DF81D0020F0FF008DF834
:101590001D009DF81E0020F0060040F00100801C98
:1015A0008DF81E009DF800008DF8446040F00200A8
:1015B0008DF80000CDE90A9AADF8306011A800E07E
:1015C00011E00E9008AA0AA9684606F006FA00285B
:1015D000A6D1BDF82000E08008E00CF0D3FC10B9E3
:1015E0000CF0D0FC08B103200FE7E58000200CE7E9
:1015F0003EB50446794D0820ADF80000A88828B112
:101600002046FFF726FE18B110203EBD06203EBD45
:101610002146012001F0D3FD0028F8D12088ADF843
:1016200004006088ADF80600A088ADF80800E088E6
:10163000ADF80A00A88801AB6A46002106F0AAFDB1
:10164000BDF800100829E2D003203EBD7FB5634DF0
:101650000446A88868B1002002900820ADF8080070
:10166000CDF80CD02046FFF7F4FD20B1102004B0D7
:1016700070BD0620FBE7A98802AA4FF6FF7006F0AE
:10168000CCFF0028F3D1BDF80810082901D00320B1
:10169000EDE7BDF800102180BDF802106180BDF8B3
:1016A0000410A180BDF80610E180E0E701B582B02A
:1016B0000220ADF80000494802AB6A46408800218C
:1016C00006F068FDBDF80010022900D003200EBD11
:1016D0001CB5002100910221ADF800100190FFF728
:1016E000DEFD08B110201CBD3C486A4641884FF61B
:1016F000FF7006F092FFBDF800100229F3D003201E
:101700001CBDFEB5354C06461546207A0F46C0076F
:1017100005D00846FFF79DFD18B11020FEBD0F2033
:10172000FEBDF82D01D90C20FEBD3046FFF791FD1E
:1017300018BB208801A905F03AFE0028F4D13078C2
:101740008DF80500208801A906F003FD0028EBD1E3
:1017500000909DF800009DF8051040F002008DF803
:101760000000090703D040F008008DF80000208831
:10177000694606F08BFC0028D6D1ADF808502088C9
:101780003B4602AA002106F005FDBDF80810A9425B
:10179000CAD00320FEBD7CB5054600200090019014
:1017A0000888ADF800000C4628460195FFF795FD26
:1017B00018B92046FFF773FD08B110207CBD15B1A4
:1017C000BDF8000060B105486A4601884FF6FF7019
:1017D00006F023FFBDF8001021807CBD240200200C
:1017E0000C20FAE72F48C088002800D0012070475D
:1017F00030B5044693B000200D46014600901422F7
:1018000001A80CF044FE1C22002108A80CF03FFEA9
:101810009DF80000CDF808D020F00F00401C20F00B
:10182000F00010308DF800009DF8010006AA20F0AD
:10183000FF008DF801009DF8200001A940F0020092
:101840008DF8200001208DF8460042F60420ADF806
:10185000440011A801902088ADF83C006088ADF8E4
:101860003E00A088ADF84000E088ADF842009DF849
:10187000020020F00600801C20F001008DF802001C
:101880000820ADF80C00ADF810000FA8059008A8CE
:1018900006F0A3F8002803D1BDF818002880002026
:1018A00013B030BD24020020F0B5007B059F1E461A
:1018B00014460D46012800D0FFDF0C2030803A206E
:1018C0003880002C08D0287A032806D0287B0128ED
:1018D00000D0FFDF17206081F0BDA889FBE72DE96C
:1018E000F0470D4686B095F80C900E991446B9F164
:1018F000010F0BD01022007B2E8A9046052807D0BE
:10190000062839D0FFDF06B0BDE8F0870222F2E7F3
:10191000E8890C2200EB400002EB400018803320E5
:101920000880002CEFD0E8896081002720E0009635
:10193000688808F1020301AA696900F097FF06EBC5
:101940000800801C07EB470186B204EB4102BDF89A
:1019500004009081F848007808B1012300E00023DA
:101960000DF1060140460E3214F029F87F1CBFB27B
:101970006089B842DBD8C6E734200880E889B9F12D
:10198000010F11D0122148430E301880002CBAD01C
:10199000E88960814846B9F1010F00D00220207328
:1019A00000270DF1040A1FE00621ECE70096688885
:1019B00008F1020301AA696900F058FF06EB08006C
:1019C000801C86B2B9F1010F12D007EBC70004EBFF
:1019D0004000BDF80410C18110220AF1020110304C
:1019E0000CF02BFD7F1CBFB26089B842DED88AE7BD
:1019F00007EB470104EB4102BDF80400D0810AF176
:101A000002014046103213F0FCFFEBE72DE9F047EE
:101A10000E4688B090F80CC096F80C80378AF5898D
:101A20000C20DFF81493109902F10C04BCF1030FA1
:101A300008D0BCF1040F3DD0BCF1070F75D0FFDF1B
:101A400008B061E705EB850C00EB4C0018803120F5
:101A50000880002AF4D0A8F1060000F0FF0A5581A2
:101A600024E01622002101A80CF011FD00977088D7
:101A7000434601AA716900F0F9FEBDF80400208018
:101A8000BDF80600E080BDF80800208199F800004C
:101A900008B1012300E00023A21C0DF10A01504609
:101AA00013F08DFF07EB080087B20A346D1EADB24C
:101AB000D7D2C5E705EB850C00EB4C00188032202F
:101AC0000880002ABCD0A8F1050000F0FF0A55816B
:101AD00037E000977088434601AA716900F0C6FE9E
:101AE0009DF80600BDF80410E1802179420860F3FA
:101AF000000162F34101820862F38201C20862F3CD
:101B0000C301020962F30411420962F3451182091B
:101B100062F386112171C0096071BDF80700208150
:101B200099F8000010B1012301E00EE000232246E5
:101B30000DF10901504613F042FF07EB080087B290
:101B40000A346D1EADB2C4D27AE7A8F1020084B2A5
:101B500005FB08FC0CF10E00188035200880002AD7
:101B6000A7D05581948100971FFA8CF370880E32AC
:101B7000716900F07BFE63E72DE9F84F1E460A9D70
:101B80000C4681462AB1607A00F58070D080E089E9
:101B9000108199F80C000C274FF000084FF00E0A46
:101BA0000D2872D2DFE800F09D070E1B272F374566
:101BB000546972727200214648460095FFF774FE20
:101BC000BDE8F88F207B9146082802D0032800D07A
:101BD000FFDF3780302009E0A9F80A80F0E7207B9A
:101BE0009146042800D0FFDF378031202880B9F1EA
:101BF000000FF1D1E4E7207B9146042800D0FFDFFD
:101C000037803220F2E7207B9146022800D0FFDFA8
:101C100037803320EAE7207B1746022800D0FFDF19
:101C20003420A6F800A02880002FC9D0A7F80A8089
:101C3000C6E7207B1746042800D0FFDF3520A6F832
:101C400000A02880002FBBD04046A7F80A8012E0F1
:101C5000207B1746052802D0062800D0FFDF102081
:101C6000308036202880002FAAD0E0897881A7F81C
:101C70000E80B9F80E00B881A2E7207B91460728B4
:101C800000D0FFDF37803720B0E72AE04FF01200A6
:101C900018804FF038001700288091D0E0897881B3
:101CA000A7F80E80A7F8108099F80C000A2805D034
:101CB0000B2809D00C280DD0FFDF81E7207B0A28F4
:101CC00000D0FFDF01200AE0207B0B2800D0FFDFDF
:101CD000042004E0207B0C2800D0FFDF05203873AF
:101CE0006EE7FFDF6CE770B50C46054601F0AAFB16
:101CF00020B10078222804D2082070BD43F20200EF
:101D000070BD0521284612F0D1F8206008B10020EE
:101D100070BD032070BD30B44880087820F00F00FB
:101D2000C01C20F0F000903001F8080B1DCA81E8BB
:101D30001D0030BC07F05DBC100000202DE9FF47FE
:101D400084B0002782460297079890468946123051
:101D50000AF069FA401D20F00306079828B907A980
:101D60005046FFF7C0FF002854D1B9F1000F05D04D
:101D70000798017B19BB052504681BE098F8000053
:101D8000092803D00D2812D0FFDF46E0079903256C
:101D90004868B0B3497B42887143914239D98AB2CD
:101DA000B3B2011D11F0F5FE0446078002E0079C66
:101DB000042508340CB1208810B1032D29D02CE063
:101DC0000798012112300AF060FAADF80C000246C3
:101DD00002AB2946504608F0B8FA070001D1A01C12
:101DE000029007983A461230C8F80400A8F802A0FA
:101DF00003A94046029B0AF055FAD8B10A2817D227
:101E000000E006E0DFE800F007091414100B0D14E1
:101E10001412132014E6002012E6112010E6082008
:101E20000EE643F203000BE6072009E60D2007E665
:101E3000032005E6BDF80C002346CDE900702A46D4
:101E40005046079900F022FD57B9032D08D1079895
:101E5000B3B2417B406871438AB2011D11F0ADFEFF
:101E6000B9F1000FD7D0079981F80C90D3E72DE98D
:101E7000FE4F91461A881C468A468046FAB102AB4C
:101E8000494608F062FA050019D04046A61C27888A
:101E900012F04FF93246072629463B46009611F0CC
:101EA0005EFD20882346CDE900504A465146404613
:101EB00000F0ECFC002020800120BDE8FE8F002017
:101EC000FBE710B586B01C46AAB104238DF800309C
:101ED0001388ADF808305288ADF80A208A788DF85A
:101EE0000E200988ADF80C1000236A462146FFF742
:101EF00025FF06B010BD1020FBE770B50D4605218B
:101F000011F0D4FF040000D1FFDF294604F11200D4
:101F1000BDE870400AF0A2B92DE9F8430D468046AD
:101F2000002607F063FB04462878102878D2DFE803
:101F300000F0773B345331311231313108313131D6
:101F400031312879001FC0B2022801D0102810D1E9
:101F500014BBFFDF35E004B9FFDF0521404611F077
:101F6000A5FF007B032806D004280BD0072828D023
:101F7000FFDF072655E02879801FC0B2022820D055
:101F800050B1F6E72879401FC0B2022819D01028B6
:101F900017D0EEE704B9FFDF13E004B9FFDF2879BB
:101FA00001280ED1172137E00521404611F07EFFB0
:101FB000070000D1FFDF07F1120140460AF02BF9BC
:101FC0002CB12A4621464046FFF7A5FE29E0132101
:101FD000404602F01FFD24E004B9FFDF0521404622
:101FE00011F064FF060000D1FFDF694606F1120020
:101FF0000AF01BF9060000D0FFDFA988172901D2DB
:10200000172200E00A46BDF80000824202D90146CC
:1020100002E005E01729C5D3404600F047FCD0E7B1
:10202000FFDF3046BDE8F883401D20F0030219B100
:1020300002FB01F0001D00E000201044704713B5C2
:10204000009858B10024684611F04DFD002C04D1D1
:10205000F749009A4A6000220A701CBD0124002042
:10206000F2E72DE9F0470C461546242200212046D0
:102070000CF00DFA05B9FFDFA87860732888DFF847
:10208000B0A3401D20F00301AF788946DAF80400C0
:1020900011F047FD060000D1FFDF4FF00008266079
:1020A000A6F8008077B109FB07F1091D0AD0DAF81C
:1020B000040011F036FD060000D1FFDF6660C6F8AF
:1020C000008001E0C4F80480298804F11200BDE812
:1020D000F0470AF091B82DE9F047804601F112006F
:1020E0000D4681460AF09FF8401DD14F20F00302B3
:1020F0006E7B14462968786811F03EFD3EB104FB02
:1021000006F2121D03D06968786811F035FD0520CC
:1021100011F074FE0446052011F078FE201A012803
:1021200002D1786811F0F2FC49464046BDE8F0471C
:102130000AF078B870B50546052111F0B7FE040025
:1021400000D1FFDF04F112012846BDE870400AF01B
:1021500062B82DE9F04F91B04FF0000BADF828B008
:10216000ADF804B047880C4605469246052138462E
:1021700011F09CFE060000D1FFDF24B1A780A4F877
:1021800006B0A4F808B0297809220B20B2EB111F81
:1021900073D12A7A04F1100138274FF00C084FF060
:1021A00012090291102A69D2DFE802F068F2F1F018
:1021B0008008D3898EA03DDCF3EEB7B7307B0228D0
:1021C00000D0FFDFA88908EBC001ADF80410302172
:1021D000ADF82810002C25D06081B5F80E800027BE
:1021E0001DE004EBC709317C89F80E10F189A9F8CC
:1021F0000C10CDF800806888042305AA296900F036
:1022000035FBBDF81410A9F8101008F10400BDF852
:1022100016107F1C1FFA80F8A9F81210BFB260894F
:10222000B842DED80CE1307B022800D0FFDFE9891C
:1022300008EBC100ADF804003020ADF8280095F897
:102240000C90002CA9F10400C0B20F90EAD061817B
:10225000B5F81080002725E0CDF8008068884B464F
:1022600003AA696900F002FB08EB09001FFA80F875
:102270006F48007818B1012302E0DDE0DAE00023C6
:1022800004EBC702009204A90C320F9813F097FBDD
:10229000009ABDF80C007F1C1082009ABDF80E0059
:1022A000BFB250826089B842D6D8C9E00AA800906F
:1022B00001AB224629463046FFF711FBC0E0307BD8
:1022C000082805D0FFDF03E0307B082800D0FFDFBF
:1022D000E8891030ADF804003620ADF82800002C55
:1022E0003FD0A9896181F189A18127E0307B09284C
:1022F00000D0FFDFA88901460C30ADF8040037207C
:10230000ADF82800002C2CD06181E8890090AB89C1
:10231000688804F10C02296955E0E88939211030F8
:1023200080B2ADF80400ADF82810002C72D0A98955
:102330006181287A0E280AD002212173E989E1817E
:10234000288A0090EB8968886969029A3BE001213C
:10235000F3E70AA8009001AB224629463046FFF772
:1023600055FB6DE0307B0A2800D0FFDFADF804900C
:10237000ADF828704CB3A9896181A4F810B0A4F815
:102380000EB0012020735BE020E002E030E038E096
:1023900041E0307B0B2800D0FFDF288AADF82870A1
:1023A0001230ADF8040084B104212173A989618140
:1023B000E989E181298A2182688A00902B8A6888CC
:1023C00004F11202696900F051FA39E0307B0C28FF
:1023D00000D0FFDFADF80490ADF828703CB30521C4
:1023E0002173A4F80AB0A4F80EB0A4F810B027E046
:1023F0000AA8009001AB224629463046FFF754FA5E
:102400001EE00AA8009001AB224629463046FFF79D
:10241000B3FB15E034E03B21ADF80400ADF8281023
:1024200074B30120E080A4F808B084F80AB007E093
:1024300010000020FFDF03E0297A012917D0FFDF19
:10244000BDF80400AAF800006CB1BDF82800208097
:10245000BDF804006080BDF82800392803D03C286E
:1024600001D086F80CB011B00020BDE8F08F3C21FF
:10247000ADF80400ADF8281014B1697AA172DFE755
:10248000AAF80000EFE72DE9F84356880F4680468A
:1024900015460521304611F009FD040000D1FFDF8B
:1024A000123400943B46414630466A680AF02EF8E2
:1024B000B8E570B50D46052111F0F8FC040000D117
:1024C000FFDF294604F11200BDE8704009F0B8BEF4
:1024D00070B50D46052111F0E9FC040000D1FFDFC5
:1024E000294604F11200BDE8704009F0D6BE70B56F
:1024F0000546052111F0DAFC040000D1FFDF04F1EC
:10250000080321462846BDE870400422AFE470B5B8
:102510000546052111F0CAFC040000D1FFDF214669
:1025200028462368BDE870400522A0E470B5064641
:10253000052111F0BBFC040000D1FFDF04F1120003
:1025400009F071FE401D20F0030511E0011D008817
:102550000322431821463046FFF789FC00280BD0A0
:10256000607BABB2684382B26068011D11F05BFB17
:10257000606841880029E9D170BD70B50E460546F6
:1025800007F034F8040000D1FFDF012020726672EA
:102590006580207820F00F00C01C20F0F000303063
:1025A0002070BDE8704007F024B8602801D00720F3
:1025B00070470878C54900F0010008700020704796
:1025C0002DE9F0438BB00D461446814606A9FFF76E
:1025D0008AFB002814D14FF6FF7601274FF42058CC
:1025E0008CB103208DF800001020ADF8100007A872
:1025F000059007AA204604A913F005FA78B1072030
:102600000BB0BDE8F0830820ADF808508DF80E70CF
:102610008DF80000ADF80A60ADF80C800CE006986B
:10262000A17801742188C1818DF80E70ADF8085031
:10263000ADF80C80ADF80A606A4602214846069B58
:10264000FFF77CFBDCE708B501228DF8022042F69B
:102650000202ADF800200A4603236946FFF731FC69
:1026600008BD08B501228DF8022042F60302ADF83C
:1026700000200A4604236946FFF723FC08BD00B585
:1026800087B079B102228DF800200A88ADF80820C1
:102690004988ADF80A1000236A460521FFF74EFB72
:1026A00007B000BD1020FBE709B1072309E40720AC
:1026B000704770B588B00D461446064606A9FFF768
:1026C00012FB00280ED17CB10620ADF808508DF821
:1026D0000000ADF80A40069B6A460821DC813046BE
:1026E000FFF72CFB08B070BD05208DF80000ADF899
:1026F0000850F0E700B587B059B107238DF80030D6
:10270000ADF80820039100236A460921FFF716FB64
:10271000C6E71020C4E770B588B00C460646002511
:1027200006A9FFF7E0FA0028DCD106980121123053
:1027300009F0ABFD9CB12178062921D2DFE801F038
:10274000200505160318801E80B2C01EE28880B2E4
:102750000AB1A3681BB1824203D90C20C2E7102042
:10276000C0E7042904D0A08850B901E00620B9E7E9
:10277000012913D0022905D004291CD005292AD00B
:102780000720AFE709208DF800006088ADF8080049
:10279000E088ADF80A00A068039023E00A208DF8D5
:1027A00000006088ADF80800E088ADF80A00A06875
:1027B0000A25039016E00B208DF800006088ADF824
:1027C0000800A088ADF80A00E088ADF80C00A06809
:1027D0000B25049006E00C208DF8000060788DF841
:1027E00008000C256A4629463046069BFFF7A6FAE4
:1027F00078E700B587B00D228DF80020ADF80810FD
:1028000000236A461946FFF799FA49E700B587B0F1
:1028100071B102228DF800200A88ADF8082049889D
:10282000ADF80A1000236A460621FFF787FA37E75A
:10283000102035E770B586B0064601200D46ADF88C
:1028400008108DF80000014600236A463046FFF765
:1028500075FA040008D12946304605F0B5FC002180
:10286000304605F0CFFC204606B070BDF8B51C46DA
:1028700015460E46069F11F04AFC2346FF1DBCB2CA
:1028800031462A46009411F036F8F8BD30B41146AE
:10289000DDE902423CB1032903D0002330BC08F03B
:1028A00032BE0123FAE71A8030BC704770B50C467F
:1028B0000546FFF722FB2146284605F094FC2846F2
:1028C000BDE87040012105F09DBC00001000002013
:1028D0004FF0E0224FF400400021C2F88001BFF326
:1028E0004F8FBFF36F8F1748016001601649900248
:1028F00008607047134900B500220A600A60124B55
:102900004FF060721A60002808BF00BD0F4A104BDC
:10291000DFF840C001280CD002281CBFFFDF00BD3B
:10292000032008601A604FF4000000BFCCF80000DC
:1029300000BD022008601A604FF04070F6E700B555
:10294000FFDF00BD00F5004008F50140A4020020B3
:1029500014F5004004F5014070B50B2000F0BDF9FE
:10296000082000F0BAF900210B2000F0D4F9002172
:10297000082000F0D0F9F44C01256560A560002026
:10298000C4F84001C4F84401C4F848010B2000F029
:10299000B5F9082000F0B2F90B2000F091F925609C
:1029A00070BD10B50B2000F098F9082000F095F9E3
:1029B000E548012141608160E4490A68002AFCD1B0
:1029C0000021C0F84011C0F84411C0F848110B2094
:1029D00000F094F9BDE81040082000F08FB910B560
:1029E0000B2000F08BF9BDE81040082000F086B9FC
:1029F00000B530B1012806D0022806D0FFDF002044
:102A000000BDD34800BDD34800BDD248001D00BD65
:102A100070B5D1494FF000400860D04DC00BC5F8EB
:102A20000803CF4800240460C5F840410820C4359D
:102A300000F053F9C5F83C41CA48047070BD08B5B0
:102A4000C14A002128B1012811D002281CD0FFDF83
:102A500008BD4FF48030C2F80803C2F84803BB48F1
:102A60003C300160C2F84011BDE80840D0E74FF4A7
:102A70000030C2F80803C2F84803B448403001608F
:102A8000C2F84411B3480CE04FF48020C2F80803A8
:102A9000C2F84803AD4844300160C2F84811AD485F
:102AA000001D0068009008BD70B516460D4604462E
:102AB000022800D9FFDF0022A348012304F11001FE
:102AC0008B4000EB8401C1F8405526B1C1F840218C
:102AD000C0F8043303E0C0F80833C1F84021C0F85F
:102AE000443370BD2DE9F0411D46144630B1012834
:102AF00033D0022838D0FFDFBDE8F081891E0022E4
:102B000021F07F411046FFF7CFFF012D23D0002099
:102B1000944D924F012668703E61914900203C39E6
:102B200008600220091D08608D49042030390860C2
:102B30008B483D34046008206C6000F0DFF83004FE
:102B4000C7F80403082000F0BBF88349F007091F09
:102B500008602E70D0E70120DAE7012B02D00022B6
:102B6000012005E00122FBE7012B04D00022022016
:102B7000BDE8F04198E70122F9E774480068704722
:102B800070B500F0D8F8704C0546D4F84001002626
:102B9000012809D1D4F80803C00305D54FF48030CB
:102BA000C4F80803C4F84061D4F8440101280CD1EA
:102BB000D4F80803800308D54FF40030C4F80803A4
:102BC000C4F84461012013F0EEFED4F84801012856
:102BD0000CD1D4F80803400308D54FF48020C4F882
:102BE0000803C4F84861022013F0DDFE5E4805606A
:102BF00070BD70B500F09FF85A4D0446287850B16A
:102C0000FFF706FF687818B10020687013F0CBFE5C
:102C10005548046070BD0320F8E74FF0E0214FF401
:102C20000010C1F800027047152000F067B84B494A
:102C300001200861082000F061B848494FF47C1079
:102C4000C1F808030020024601EB8003C3F84025C9
:102C5000C3F84021401CC0B20628F5D37047410A92
:102C600043F609525143C0F3080010FB02F000F58F
:102C7000807001EB5020704710B5430B48F2376469
:102C800063431B0C5C020C60384C03FB0400384BA4
:102C90004CF2F72443435B0D13FB04F404EB402098
:102CA00000F580704012107008681844086010BD6C
:102CB0002C484068704729490120C1F8000270473C
:102CC000002809DB00F01F0201219140400980002B
:102CD00000F1E020C0F80011704700280DDB00F083
:102CE0001F02012191404009800000F1E020C0F85E
:102CF0008011BFF34F8FBFF36F8F7047002809DB40
:102D000000F01F02012191404009800000F1E02005
:102D1000C0F8801270474907090E002804DB00F153
:102D2000E02080F80014704700F00F0000F1E02070
:102D300080F8141D70470C48001F00680A4A0D49AE
:102D4000121D11607047000000B0004004B5004043
:102D50004081004044B1004008F50140008000403F
:102D6000408500403C00002014050240F7C2FFFFF0
:102D70006F0C0100010000010A4810B50468094900
:102D800009480831086013F0A2FE0648001D0460DF
:102D900010BD0649002008604FF0E0210220C1F874
:102DA000800270471005024001000001FC1F004036
:102DB000374901200860704770B50D2000F049F8D0
:102DC000344C0020C4F800010125C4F804530D2040
:102DD00000F050F825604FF0E0216014C1F80001C8
:102DE00070BD10B50D2000F034F82A480121416073
:102DF0000021C0F80011BDE810400D2000F03AB8E5
:102E0000254810B504682449244808310860214940
:102E1000D1F80001012804D0FFDF1F48001D046025
:102E200010BD1B48001D00680022C0B2C1F800217F
:102E300014F07FFBF1E710B5164800BFD0F8001181
:102E40000029FBD0FFF7DCFFBDE810400D2000F0AB
:102E500011B800280DDB00F01F020121914040094C
:102E6000800000F1E020C0F88011BFF34F8FBFF366
:102E70006F8F7047002809DB00F01F02012191408D
:102E80004009800000F1E020C0F880127047000087
:102E900004D5004000D000401005024001000001B0
:102EA0004FF0E0214FF00070C1F8800101F5C071D2
:102EB000BFF34F8FBFF36F8FC1F80001394B8022F2
:102EC00083F8002441F8800C704700B502460420C6
:102ED000354903E001EBC0031B792BB1401EC0B2A2
:102EE000F8D2FFDFFF2000BD41F8302001EBC00128
:102EF00000224A718A7101220A7100BD2A4A00210A
:102F000002EBC0000171704710B50446042800D3DD
:102F1000FFDF254800EBC4042079012800D0FFDF43
:102F20006079A179401CC0B2814200D060714FF03D
:102F3000E0214FF00070C1F8000210BD70B504250B
:102F4000194E1A4C16E0217806EBC1000279012ACD
:102F500008D1427983799A4204D04279827156F835
:102F6000310080472078401CC0B22070042801D373
:102F7000002020706D1EEDB2E5D270BD0C4810B57A
:102F800004680B490B4808310860064890F80004B3
:102F90004009042800D0FFDFFFF7D0FF0448001DE0
:102FA000046010BD19E000E0E0050020580000209A
:102FB00010050240010000010548064A01689142DF
:102FC00001D1002101600449012008607047000020
:102FD0005C000020BEBAFECA40E5014070B50C4658
:102FE000054609F02FFC21462846BDE870400AF04E
:102FF00010BD7047704770470021016081807047A5
:103000002CFFFFFFDBE5B151007002002301FFFF41
:103010008C00000078DB6A007A2E9AC67DB66CFAC6
:10302000F35721CCC310D5E51471FB3C30B5FC4DF2
:103030000446062CA9780ED2DFE804F0030E0E0E2B
:103040000509FFDF08E0022906D0FFDF04E00329BD
:1030500002D0FFDF00E0FFDFAC7030BD30B50446CA
:103060001038EF4D07280CD2DFE800F0040C060CF6
:103070000C0C0C00FFDF05E0287E112802D0FFDFDA
:1030800000E0FFDF2C7630BD2DE9F04112F026FE86
:10309000044614F063F8201AC5B2062010F0AEFE04
:1030A0000446062010F0B2FE211ADD4C207E1228C4
:1030B00018D000200F18072010F0A0FE06460720A9
:1030C00010F0A4FE301A3918207E13280CD00020EE
:1030D0000144A078042809D000200844281AC0B26E
:1030E000BDE8F0810120E5E70120F1E70120F4E7E8
:1030F000CB4810B590F825004108C94800F12600DA
:1031000005D00EF0F5FEBDE8104006F08CB80EF0CC
:10311000D0FEF8E730B50446A1F120000D460A289C
:103120004AD2DFE800F005070C1C2328353A3F445B
:10313000FFDF42E0207820283FD1FFDF3DE0B848A4
:103140008178052939D0007E122836D020782428AD
:1031500033D0252831D023282FD0FFDF2DE0207851
:1031600022282AD0232828D8FFDF26E0207822280A
:1031700023D0FFDF21E0207822281ED024281CD075
:1031800026281AD0272818D0292816D0FFDF14E0C7
:103190002078252811D0FFDF0FE0207825280CD0DB
:1031A000FFDF0AE02078252807D0FFDF05E0207840
:1031B000282802D0FFDF00E0FFDF257030BD1FB5FB
:1031C00004466A46002001F0A5FEB4B1BDF8022015
:1031D0004FF6FF700621824201D1ADF80210BDF812
:1031E0000420824201D1ADF80410BDF808108142DC
:1031F00003D14FF44860ADF8080068460FF0E2FADA
:1032000006F011F804B010BD70B516460C46054620
:10321000FEF71FF848B90CB1B44208D90C2070BDB4
:1032200055F82400FEF715F808B1102070BD2046AF
:10323000641EE4B2F4D270BD2DE9F04105461F468C
:1032400090460E4600240068FEF750F830B9A98871
:1032500028680844401EFEF749F808B110203FE7EF
:1032600028680028A88802D0B84202D850E0002878
:10327000F5D0092034E72968085DB8B1671CCA5D3C
:10328000152A2ED03CDC152A3AD2DFE802F039129A
:10329000222228282A2A313139393939393939391C
:1032A00039392200085D30BB641CA4B2A242F9D8AF
:1032B00033E00228DDD1A01C085C88F80000072854
:1032C00001D2400701D40A200AE7307840F001001B
:1032D00015E0C143C90707E0012807D010E0062028
:1032E000FEE60107A1F180510029F5D01846F7E666
:1032F0003078810701D50B20F2E640F002003070F3
:103300002868005D384484B2A888A04202D2B0E7A1
:103310004FF4485382B2A242ADD80020E0E610B587
:10332000027843F2022354080122022C12D003DC5B
:103330003CB1012C16D106E0032C10D07F2C11D10A
:1033400012E0002011E080790324B4EB901F09D132
:103350000A700BE08079B2EB901F03D1F8E7807917
:103360008009F5D0184610BDFF200870002010BD60
:1033700008B500208DF80000294890F82E1051B1B2
:1033800090F82F0002280FD003280FD0FFDF00BFD6
:103390009DF8000008BD22486946253001F009FE6D
:1033A0000028F5D0FFDFF3E7032000E001208DF8CF
:1033B0000000EDE738B50C460546694601F0F9FD19
:1033C00000280DD19DF80010207861F3470020708F
:1033D00055F8010FC4F80100A888A4F805000020E2
:1033E00038BD38B5137888B102280FD0FF281BD01C
:1033F0000CA46D46246800944C7905EB9414247851
:1034000064F347031370032805D010E023F0FE0394
:1034100013700228F7D1D8B240F001000AE0000092
:10342000F00100200302FF0143F0FE00107010784D
:1034300020F0010010700868C2F801008888A2F826
:10344000050038BD022110F031BD38B50C460978B1
:10345000222901D2082038BDADF800008DF80220E5
:1034600068460EF087FD05F0DEFE050003D1212140
:103470002046FFF74FFE284638BD1CB500208DF8CA
:103480000000CDF80100ADF80500FB4890F82E00D3
:10349000022801D0012000E000208DF807006846D6
:1034A0000EF0F0FD002800D0FFDF1CBD00220A80D6
:1034B000437892B263F3451222F040020A8000780A
:1034C0000C282BD2DFE800F02A06090E1116191C71
:1034D0001F220C2742F0110009E042F01D00088075
:1034E0000020704742F0110012E042F0100040F05E
:1034F0000200F4E742F01000F1E742F00100EEE7CD
:1035000042F0010004E042F00200E8E742F002006D
:1035100040F00400E3E742F00400E0E707207047D2
:103520002DE9FF478AB00025BDF82C6082461C4675
:1035300091468DF81C50700703D56068FDF789FE31
:1035400068B9CD4F4FF0010897F82E0058B197F8A1
:103550002F00022807D16068FDF7C8FE18B11020BF
:103560000EB0BDE8F087300702D5A08980283DD88D
:10357000700705D4B9F1000F02D097F8240098B372
:10358000E07DC0F300108DF81B00627D0720032151
:103590005AB3012A2CD0022AE2D0042AE0D18DF8B5
:1035A0001710F00627D4A27D072022B3012A22D0CB
:1035B000022A23D0042AD3D18DF819108DF8159042
:1035C000606810B307A9FFF7AAFE0028C8D19DF8CC
:1035D0001C00FF2816D0606850F8011FCDF80F10AE
:1035E0008088ADF8130014E000E001E00720B7E7A1
:1035F0008DF81780D5E78DF81980DFE702208DF868
:103600001900DBE743F20220AAE7CDF80F50ADF82E
:103610001350E07B40B9207C30B9607C20B9A07C9D
:1036200010B9E07CC00601D0062099E78DF800A013
:10363000BDF82C00ADF80200A0680190A0680290CF
:1036400004F10F0001F0A9FC8DF80C00FFF790FECB
:103650008DF80D009DF81C008DF80E008DF81650A9
:103660008DF81850E07D08A900F00F008DF81A00C1
:1036700068460FF0E3F905F0D6FD71E7F0B58FB0BD
:1036800000258DF830508DF814508DF834500646D2
:103690008DF82850019502950395049519B10FC92D
:1036A00001AC84E80F00744CA078052801D00428F0
:1036B0000CD101986168884200D120B90398E16873
:1036C000884203D110B108200FB0F0BD207DC006A4
:1036D00001D51F2700E0FF273B460DAA05A903A837
:1036E000FFF7AAFD0028EFD1A08AC10702D0C006CB
:1036F00000D4EE273B460AAA0CA901A8FFF79CFDBF
:103700000028E1D19DF81400C00701D00A20DBE7B2
:10371000A08A410708D4A17D31B19DF828108907FE
:1037200002D043F20120CFE79DF82810C90709D045
:10373000400707D4208818B144F25061884201D96B
:103740000720C1E78DF818508DF81960BDF8080002
:10375000ADF81A000198079006A80FF07BF905F064
:1037600062FD0028B0D18DF820508DF82160BDF8A1
:103770001000ADF822000398099008A80FF08CF90A
:1037800005F051FD00289FD101AD241D95E80F00E3
:1037900084E80F00002097E770B586B00D4604005E
:1037A00005D0FDF7A3FD20B1102006B070BD0820A4
:1037B000FBE72078C107A98802D0FF2902D303E0E4
:1037C0001F2901D20920F0E7800763D4FFF75CFCD2
:1037D00038B12178C1F3C100012804D0032802D0F8
:1037E00005E01320E1E7244890F82400C8B1C80799
:1037F0004FF001064FF0000502D08DF80F6001E098
:103800008DF80F50FFF7B4FD8DF800002078694661
:10381000C0F3C1008DF8010060788DF80250C20835
:1038200001D00720C1E730B3C20701D08DF8026094
:10383000820705D59DF8022042F002028DF8022091
:10384000400705D59DF8020040F004008DF8020005
:10385000002022780B18C2F38002DA7001EB4002DC
:103860006388D380401CA388C0B253810228F0D360
:10387000207A78B905E001E0F00100208DF80260BF
:10388000E6E7607A30B9A07A20B9E07A10B9207BF7
:10389000C00601D0062088E704F1080001F07DFB96
:1038A0008DF80E0068460EF0F6FC05F0BCFC002812
:1038B00089D18DF810608DF81150E088ADF81200B4
:1038C000ADF8145004A80EF039FD05F0ACFC00284A
:1038D00088D12078C00701D0152000E01320FFF721
:1038E000BDFB002061E72DE9FF470220FD4E8DF86A
:1038F00004000027708EADF80600B84643F20209B6
:103900004CE001A810F039FA050006D0708EA8B37B
:10391000A6F83280ADF806803EE0039CA07F010748
:103920002DD504F124000090A28EBDF80800214698
:1039300004F1360301F0BCFC050005D04D452AD04A
:10394000112D3CD0FFDF3AE0A07F20F00801E07F9E
:10395000420862F3C711A177810861F30000E077A4
:1039600094F8210000F01F0084F820002078282817
:1039700026D129212046FFF7CDFB21E014E04007A6
:103980000AD5BDF8080004F10E0101F01CFB05008A
:103990000DD04D4510D100257F1CFFB2022010F044
:1039A0002DFA401CB842ACD8052D11D008E0A07FFC
:1039B00020F00400A07703E0112D00D0FFDF0025E8
:1039C000BDF806007086052D04D0284604B0C8E571
:1039D000A6F832800020F9E770B50646FFF732FD01
:1039E000054605F003FE040000D1FFDF6680207865
:1039F00020F00F00801C20F0F00020302070032009
:103A0000207295F83E006072BDE8704005F0F1BD8F
:103A10002DE9F04786B0040000D1FFDF2078B14DDA
:103A200020F00F00801C20F0F000703020706068E3
:103A30000178491F1B2933D2DFE801F0FE32323210
:103A400055FD320EFDFD42FC32323278FCFCFBFAB1
:103A500032FCFCF9F8FCFC00C6883046FFF7F2FCAB
:103A60000546304607F045FCE0B16068007A85F80D
:103A70003E0021212846FFF74DFB3046FEF75AFB5A
:103A8000304603F0D7FE3146012014F017F8A87F26
:103A900020F01000A877FFF726FF002800D0FFDFF6
:103AA00006B05EE5207820F0F00020302070032082
:103AB000207266806068007A607205F09AFDD8E72F
:103AC000C5882846FFF7BEFC00B9FFDF60680079B3
:103AD000012800D0FFDF6068017A06B02846BDE803
:103AE000F04707F0EBBDC6883046FFF7ABFC05009A
:103AF00000D1FFDF05F07DFD606831460089288137
:103B000060684089688160688089A881012013F01D
:103B1000D5FF0020A875A87F00F003000228BFD1C0
:103B2000FFF7E1FE0028BBD0FFDFB9E7007928B13D
:103B30000228B5D03C28B3D0FFDFB1E705F059FD2E
:103B40006668B6F806A0307A361D012806D0687E71
:103B5000814605F0D4FA070003D101E0E878F7E7E1
:103B6000FFDF00220221504610F097F9040000D137
:103B7000FFDF22212046FFF7CDFA3079012800D05F
:103B80000220A17F804668F30101A177308B20815C
:103B9000708B6081B08BA08184F822908DF80880B2
:103BA000B8680090F86801906A460321504610F00A
:103BB00074F900B9FFDFB888ADF81000B8788DF857
:103BC000120004AA0521504610F067F900B9FFDF82
:103BD000B888ADF80C00F8788DF80E0003AA04211F
:103BE000504610F05AF900B9FFDF062106F1120025
:103BF0000DF00EF940B37079800700D5FFDF7179C1
:103C0000E07D61F34700E075D6F80600A061708999
:103C1000A083062106F10C000DF0FAF8F0B195F83A
:103C200025004108607861F3470006E041E039E093
:103C300071E059E04EE02FE043E06070D5F82600D7
:103C4000C4F80200688D12E0E07D20F0FE00801CC8
:103C5000E075D6F81200A061F08AD9E7607820F00C
:103C6000FE00801C6070F068C4F80200308AE080BA
:103C7000B8F1010F04D0B8F1020F05D0FFDF0FE754
:103C80000320FFF7D3F90BE7287E122800D0FFDFCF
:103C90001120FFF7E3F903E706B02046BDE8F0473F
:103CA00001F092BD05F0A5FC15F8300F40F00200C0
:103CB00005E005F09EFC15F8300F40F00400287078
:103CC000EEE6287E13280AD01528D8D15FF016001A
:103CD000FFF7C4F906B0BDE8F04705F08ABC142030
:103CE000F6E70000F0010020A978052909D0042991
:103CF000C5D105F07EFC022006B0BDE8F047FFF715
:103D000095B900790028BAD0E87801F02DF905F0CE
:103D100070FC0320F0E7287E122802D1687E01F0B3
:103D200023F91120D4E72DE9F05F054600784FF024
:103D300000080009DFF8B8A891460C46464601285D
:103D40006ED002286DD007280BD00A286AD0FFDF7A
:103D5000A9F8006014B1A4F8008066800020BDE8D6
:103D6000F09F6968012704F108000B784FF0020BFF
:103D70005B1F4FF6FF721B2B7ED2DFE803F0647DE2
:103D80007D7D0E7D7D7D7D7D7D217D7D7D2BFDFC81
:103D9000FBFA7D14D2F9E7F8F700C8884FF0120853
:103DA000102621469AE14FF01C080A26BCB38888E9
:103DB000A0806868807920726868C0796072C7E7FF
:103DC0004FF01B08142654B30320207268688088C3
:103DD000A080BDE70A793C2ABAD00D1D4FF010082B
:103DE0002C26E4B16988A180298B6182298B2182EC
:103DF000698BA182A98BE1826B790246A91D1846C5
:103E0000FFF7EFFA2979002001290CD084F80FB0D0
:103E1000FF212176E06120626062A06298E70FE0F6
:103E20003BE15EE199E1E77320760AF1040090E856
:103E30000E00DAF81000C4E90930C4E9071287E778
:103E4000A9F800608AE72C264FF01D08002CF7D057
:103E5000A28005460F1D897B008861F30000288041
:103E6000B97A490861F341002880B97A890861F379
:103E700082002880B97A00E00CE1C90861F3C30030
:103E80002880B97AAA1C0911491C61F3041000F0BA
:103E90007F0028807878B91CFFF7A3FA387D05F1F8
:103EA000090207F11501FFF79CFA387B01F0A9F828
:103EB0002874787B01F0A5F86874F87EA874787A85
:103EC000E874387F2875B87B6875388AE882DAF834
:103ED0001C10A961B97A504697F808A0C1F34111A6
:103EE000012904D0008C504503D2824609E0FFDF4F
:103EF00010E0022903D0288820F0600009E0504536
:103F000004D1288820F06000403002E0288840F08A
:103F100060002880A4F824A0524607F11D01A8697A
:103F20009BE011264FF02008002C89D0A280686801
:103F300004F10A02007920726868007B6072696887
:103F40008B1D48791946FFF74CFA01E70A264FF016
:103F50002108002CE9D08888A080686880792072C8
:103F60006868C07960729AF8301006E078E06BE01B
:103F700052E07FE019E003E03AE021F00401A6E01E
:103F80000B264FF02208002CCFD0C888A08068688C
:103F9000007920726868007A01F033F8607268680E
:103FA000407A01F02EF8A072D2E61C264FF02608C7
:103FB000002CBAD0A2806868407960726868007A84
:103FC000A0720AF1040090E80E00DAF81000C4E9CB
:103FD0000530C4E90312686800793C2803D04328FF
:103FE00003D0FFDFB4E62772B2E684F808B0AFE68C
:103FF00010264FF02408002C97D08888A08068688D
:10400000807920816868807A608168680089A081F1
:1040100068688089E0819BE610264FF02308002C19
:1040200098D08888A0806868C088208168680089E6
:10403000608168684089A08168688089E0819AF819
:10404000301021F0020142E030264FF02508002C0C
:104050009AD0A2806968282249680AF0EEF977E6CA
:104060002A264FF02F08002C8ED0A28069682222C9
:10407000091DF2E714264FF01B08002C84D0A28003
:10408000686800790128B0D02772DAE90710C4E91E
:1040900003105DE64A46214660E0287A012803D0F5
:1040A000022817D0FFDF53E610264FF01F08002C20
:1040B000A2D06888A080A8892081E8896081288AA8
:1040C000A081688AE0819AF8301021F001018AF815
:1040D00030103DE64FF012081026688800F07EFF91
:1040E00036E6287AC8B3012838D0022836D003280B
:1040F00001D0FFDF2CE609264FF01108002C8FD0ED
:104100006F883846FFF79EF990F822A0A780687A5A
:104110002072042138460FF0DBFE052138460FF0EF
:10412000D7FE002138460FF0D3FE012138460FF0AC
:10413000CFFE032138460FF0CBFE022138460FF0A8
:10414000C7FE062138460FF0C3FE072138460FF0A0
:10415000BFFE504600F008FFFAE5FFE72846BDE83D
:10416000F05F01F0BBBC70B5012803D0052800D07A
:10417000FFDF70BD8DB22846FFF764F9040000D15F
:10418000FFDF20782128F4D005F030FA80B10178E3
:1041900021F00F01891C21F0F00110310170022182
:1041A000017245800020A075BDE8704005F021BA7D
:1041B00021462846BDE870401322FFF746B92DE995
:1041C000F04116460C00804600D1FFDF307820F029
:1041D0000F00801C20F0F000103030702078012893
:1041E00004D0022818D0FFDFBDE8F0814046FFF779
:1041F00029F9050000D1FFDF0320A87505F0F9F9C2
:1042000094E80F00083686E80F00F94810F8301FD0
:1042100041F001010170E7E74046FFF713F905009F
:1042200000D1FFDFA1884FF6FF700027814202D145
:10423000E288824203D0814201D1E08840B105F09A
:10424000D8F994E80F00083686E80F00AF75CBE781
:10425000A87D0128C8D178230022414613F084FBB1
:104260000220A875C0E738B50C4624285CD008DCCD
:1042700020280FD0212825D022284BD0232806D152
:104280004CE0252841D0262832D03F2851D00725A0
:10429000284638BD0021052013F0E6FB08B11120A7
:1042A00038BDA01C0EF0E1FA04F0BDFF0500EFD10F
:1042B000002208231146052013F056FB0528E7D0FD
:1042C000FFDFE5E76068FDF708F808B1102038BDAA
:1042D000618820886A460EF071FD04F0A4FF050095
:1042E000D6D160680028D3D0BDF800100180CFE798
:1042F000206820B1FCF7FAFF08B11025C8E7204676
:104300000EF03BFE1DE00546C2E7A17820880EF0C6
:1043100086FD16E0086801F08DFEF4E7087800F0ED
:1043200001000DF0B9FD0CE0618820880EF0C1FCA1
:1043300007E0087800F001008DF8000068460EF0F4
:10434000DFF804F070FFDEE770B505460C4608465E
:10435000FCF7A5FF08B1102070BD202D07D0212D3E
:104360000DD0222D0BD0252D09D0072070BD20881F
:10437000A11C0DF065FEBDE8704004F054BF06209E
:1043800070BD9B482530704708B5342200219848FD
:104390000AF07DF80120FEF749FE1120FEF75EFECF
:1043A00093496846263105F0B7F891489DF80020FA
:1043B00010F8251F62F3470121F00101017000216F
:1043C00041724FF46171A0F8071002218172FEF76B
:1043D0008FFE00B1FFDFFDF705F801F0BEF908BD63
:1043E00010B50C464022002120460AF050F8A07F6C
:1043F00020F00300A077202020700020A07584F812
:10440000230010BD70472DE9FC410746FCF721FF52
:1044100010B11020BDE8FC81754E06F12501D6F8DB
:1044200025000090B6F82950ADF8045096F82B40BE
:104430008DF806403846FEF7BDFF0028EAD1FEF7AA
:1044400057FE0028E6D0009946F8251FB580B471C4
:10445000E0E710B50446FCF722FF08B1102010BDBC
:1044600063486349224690F8250026314008FEF74C
:10447000B8FF002010BD3EB504460D460846FCF7C7
:104480000EFF08B110203EBD14B143F204003EBD42
:1044900057488078052803D0042801D008203EBD65
:1044A000694602A80AF012FC2A4669469DF80800EF
:1044B000FEF797FF00203EBDFEB50D4604004FF00D
:1044C000000712D00822FEF79FFE002812D1002616
:1044D00009E000BF54F826006946FEF720FF0028D7
:1044E00008D1761CF6B2AE42F4D30DF01CFC10B12C
:1044F00043F20320FEBD3E4E86F824700CB3002725
:104500001BE000BF54F8270002A9FEF708FF00B126
:10451000FFDF9DF808008DF8000054F8270050F8E0
:10452000011FCDF801108088ADF8050068460DF038
:104530001FFC00B1FFDF7F1CFFB2AF42E2D386F861
:1045400024500020FEBD2DE9F0418AB01546884672
:1045500004001ED00F4608222946FEF755FE00280B
:1045600011D1002613E000BF54F826006946103030
:1045700000F01FFD002806D13FB157F82600FCF7D8
:1045800068FE10B110200AB02EE6761CF6B2AE42DC
:10459000EAD3681EC6B217E0701CC7B212E000BFB3
:1045A00054F82600017C4A0854F827100B7CB2EB23
:1045B000530F05D106221130113109F011FF50B10E
:1045C0007F1CFFB2AF42EBD3761EF6B2E4D2464672
:1045D00024B1012003E043F20520D4E700200DF0D0
:1045E000ECFB10B90DF0F5FB20B143F20420CAE753
:1045F000F001002064B300270DF1170826E000BF8A
:1046000054F827006946103000F0D3FC00B1FFDFFA
:1046100054F82700102250F8111FCDF8011080889F
:10462000ADF8050054F827100DF1070009F005FF5B
:1046300096B156F827101022404609F0FEFE684653
:104640000DF07BFB00B1FFDF7F1CFFB2AF42D7D381
:10465000FEF713FF002096E7404601F0DFFCEEE78F
:1046600030B585B00446FDF7BDF830B906200FF02F
:10467000C5FB10B1062005B030BD2046FCF7E9FDB2
:1046800018B96068FCF732FE08B11020F3E76088C3
:104690004AF2B811884206D82078F94D28B101288D
:1046A00006D0022804D00720E5E7FEF721FD18E038
:1046B0006078022804D0032802D043F20220DAE70F
:1046C00085F82F00C1B200200090ADF80400022947
:1046D0002CD0032927D0FFDF68460DF009FC04F039
:1046E000A2FD0028C7D1606801F08BFC207858B18A
:1046F00001208DF800000DF1010001F08FFC6846EB
:104700000EF0FDFB00B1FFDF207885F82E00FEF7EC
:10471000B4FE608860B1A88580B20DF046FB00B1A0
:10472000FFDF0020A7E78DF80500D5E74020FAE776
:104730004FF46170EFE710B50446FCF7B0FD20B907
:10474000606838B1FCF7C9FD08B1102010BD606881
:1047500001F064FCCA4830F82C1F6180C178617098
:1047600080782070002010BD2DE9F843144689465A
:104770000646FCF794FDA0B94846FCF7B7FD80B9A2
:104780002046FCF7B3FD60B9BD4DA878012800D1E3
:104790003CB13178FF2906D049B143F20400BDE8AD
:1047A000F8831020FBE7012801D00420F7E7CCB301
:1047B000052811D004280FD069462046FEF776FE62
:1047C0000028ECD1217D49B1012909D0022909D065
:1047D000032909D00720E2E70820E0E7024604E0C9
:1047E000012202E0022200E003228046234617460F
:1047F00000200099FEF794FE0028D0D1A0892880DF
:10480000A07BE875BDF80000A882AF75BDF8001068
:10481000090701D5A18931B1A1892980C00704D038
:10482000032003E006E08021F7E70220FEF7FEFB0D
:1048300086F800804946BDE8F8430020FEF71EBF19
:104840007CB58F4C05460E46A078022803D003287D
:1048500001D008207CBD15B143F204007CBD0720C7
:104860000FF0D4FA10B9A078032806D0FEF70CFC9C
:1048700028B1A078032804D009E012207CBD1320C1
:104880007CBD304600F053FB0028F9D1E670FEF7FE
:104890006FFD0AF058F901208DF800008DF8010035
:1048A0008DF802502088ADF80400E07D8DF80600F8
:1048B00068460EF0C1F904F0B6FC0028E0D1A078FB
:1048C000032805D05FF00400FEF7B0FB00207CBD9C
:1048D000E07800F03CFB0520F6E71CB510B143F290
:1048E00004001CBD664CA078042803D0052801D024
:1048F00008201CBD00208DF8000001218DF801105A
:104900008DF8020068460EF097F904F08CFC002840
:10491000EFD1A078052805D05FF00200FEF786FBF6
:1049200000201CBDE07800F01FFB0320F6E72DE916
:10493000FC4180460E4603250846FCF7D7FC0028BC
:1049400066D14046FEF77EFD040004D02078222880
:1049500004D208205EE543F202005BE5A07F00F090
:1049600003073EB1012F0CD000203146FEF727FC93
:104970000500EFD1012F06D0022F1AD0FFDF284605
:1049800048E50120F1E7A07D3146022801D011B1B0
:1049900007E011203EE56846FCF758FE0028D9D113
:1049A0006946404606F04DFE0500E8D10120A0759D
:1049B000E5E7A07D032804D1314890F83000C00716
:1049C00001D02EB30EE026B1A07F40071ED40021F7
:1049D00000E00121404606F054FE0500CFD1A0754D
:1049E000002ECCD03146404600F0EDFA05461128A5
:1049F000C5D1A07F4107C2D4316844F80E1F716849
:104A0000616040F0040020740025B8E71125B6E786
:104A10001020FFE470B50C460546FEF713FD0100BB
:104A200005D022462846BDE87040FEF70EBD43F291
:104A3000020070BD10B5012807D1114B9B78012BE6
:104A400000D011B143F2040010BD0DF0E0F9BDE853
:104A5000104004F0E8BB012300F090BA00231A468E
:104A6000194600F08BBA70B506460C460846FCF7AE
:104A7000F0FB18B92068FCF712FC18B1102070BDCB
:104A8000F0010020F84D2A7E112A04D0132A00D309
:104A90003EB10820F3E721463046FEF77DFE60B1C7
:104AA000EDE70920132A0DD0142A0BD0A188FF2985
:104AB000E5D31520FEF7D2FA0020D4E90012C5E9AB
:104AC0000712DCE7A1881F29D9D31320F2E71CB510
:104AD000E548007E132801D208201CBD00208DF877
:104AE000000068460DF02AFC04F09DFB0028F4D17C
:104AF0001120FEF7B3FA00201CBD2DE9F04FDFF8BE
:104B000068A3814691B09AF818009B4615460C465A
:104B1000132803D3FFF7DBFF00281FD12046FCF743
:104B200098FBE8BB2846FCF794FBC8BB20784FF005
:104B30000107C0074FF0000102D08DF83A7001E084
:104B40008DF83A1020788846C0F3C1008DF8000037
:104B500060788DF80910C10803D0072011B0BDE8B6
:104B6000F08FB0B3C10701D08DF80970810705D56A
:104B70009DF8091041F002018DF80910400705D594
:104B80009DF8090040F004008DF809009DF8090027
:104B9000810703D540F001008DF80900002000E0F6
:104BA00015E06E4606EB400162884A81401CA288EF
:104BB000C0B20A820328F5D32078C0F3C1000128CF
:104BC00025D0032823D04846FCF743FB28B110200A
:104BD000C4E7FFE78DF80970D8E799F800004008AE
:104BE00008D0012809D0022807D0032805D043F2B5
:104BF0000220B3E78DF8028001E08DF8027048468C
:104C000050F8011FCDF803108088ADF80700FEF7BB
:104C1000AFFB8DF801000021424606EB41002B88D6
:104C2000C3826B888383AB884384EB880385491CEC
:104C3000C285C9B282860329EFD3E088ADF83C0073
:104C400068460DF053FC002887D19AF818005546A5
:104C5000112801D0082081E706200FF0D7F838B1DD
:104C60002078C0F3C100012804D0032802D006E058
:104C7000122073E795F8240000283FF46EAFFEF78A
:104C800003FA022801D2132068E7584600F04FF9D2
:104C900000289DD185F819B068460DF06DFD04F02F
:104CA000C2FA040094D1687E00F051F91220FEF798
:104CB000D5F9204652E770B56B4D287E122801D0F9
:104CC0000820DCE60DF05BFD04F0ADFA040005D130
:104CD000687E00F049F91120FEF7C0F92046CEE6C3
:104CE00070B5064615460C460846FCF7D8FA18B9C2
:104CF0002846FCF7D4FA08B11020C0E62A4621461F
:104D000030460EF03BF804F08EFA0028F5D12178F9
:104D10007F29F2D10520B2E67CB505460C4608464F
:104D2000FCF797FA08B110207CBD2846FEF78AFBF5
:104D300020B10078222804D208207CBD43F2020072
:104D40007CBD494890F83000400701D511207CBD5A
:104D50002078C00802D16078C00801D007207CBD4F
:104D6000ADF8005020788DF8020060788DF80300CF
:104D70000220ADF8040068460CF03BFE04F053FA44
:104D80007CBD70B586B014460D460646FEF75AFB4C
:104D900028B10078222805D2082006B06FE643F239
:104DA0000200FAE72846FCF7A1FA20B944B12046F0
:104DB000FCF793FA08B11020EFE700202060A080F4
:104DC000294890F83000800701D51120E5E703A9B4
:104DD00030460CF05EFE10B104F025FADDE7ADF8C8
:104DE0000060BDF81400ADF80200BDF81600ADF883
:104DF0000400BDF81000BDF81210ADF80600ADF8C3
:104E000008107DB1298809B1ADF80610698809B18B
:104E1000ADF80210A98809B1ADF80810E98809B108
:104E2000ADF80410DCB1BDF80610814201D9081AB2
:104E30002080BDF80210BDF81400814201D9081A83
:104E40006080BDF80800BDF80410BDF816200144CC
:104E5000BDF812001044814201D9081AA0806846AA
:104E60000CF0D5FEB8E70000F00100201CB56C493D
:104E70000968CDE9001068460DF03AFB04F0D3F95B
:104E80001CBD1CB500200090019068460DF030FB61
:104E900004F0C9F91CBD70B505460C460846FCF780
:104EA000FEF908B11020EAE5214628460DF012F976
:104EB000BDE8704004F0B7B93EB505460C4608465B
:104EC000FCF7EDF908B110203EBD002000900190E4
:104ED0000290ADF800502089ADF8080020788DF8D8
:104EE0000200606801902089ADF808006089ADF883
:104EF0000A0068460DF000F904F095F93EBD0EB5C4
:104F0000ADF800000020019068460DF0F5F804F0BF
:104F10008AF90EBD10800888508048889080C88823
:104F200010818888D080002050819081704710B512
:104F3000044604F0E4F830B1407830B1204604F083
:104F4000FCFB002010BD052010BD122010BD10B5C7
:104F500004F0D5F8040000D1FFDF607800B9FFDF6E
:104F60006078401E607010BD10B504F0C8F80400F1
:104F700000D1FFDF6078401C607010BD1CB5ADF83B
:104F800000008DF802308DF803108DF8042068467B
:104F90000DF0B7FE04F047F91CBD0CB521A2D2E913
:104FA0000012CDE900120079694601EB501000783B
:104FB0000CBD0278520804D0012A02D043F202202C
:104FC0007047FEF7ACB91FB56A46FFF7A3FF684606
:104FD0000DF008FC04F027F904B010BD70B50C000A
:104FE00006460DD0FEF72EFA050000D1FFDFA680A1
:104FF00028892081288960816889A081A889E08129
:105000003DE500B540B1012805D0022803D00328B2
:1050100004D0FFDF002000BDFF2000BD042000BD44
:1050200014610200070605040302010010B50446DE
:10503000FCF70FF908B1102010BD2078C0F3021062
:10504000042807D86078072804D3A178102901D84C
:10505000814201D2072010BDE078410706D42179B2
:105060004A0703D4000701D4080701D5062010BD64
:10507000002010BD10B513785C08837F64F3C7135C
:10508000837713789C08C37F64F30003C377107899
:10509000C309487863F34100487013781C090B7802
:1050A00064F347130B701378DB0863F30000487058
:1050B0005078487110BD10B5C4780B7864F30003C4
:1050C0000B70C478640864F341030B70C478A408BF
:1050D00064F382030B70C478E40864F3C3030B70B9
:1050E0000379117863F30001117003795B0863F3AE
:1050F0004101117003799B0863F3820111700079FB
:10510000C00860F3C301117010BD70B514460D46A0
:10511000064604F06BFA80B10178182221F00F01E5
:10512000891C21F0F001A03100F8081B214609F08C
:1051300084F9BDE8704004F05CBA29463046BDE809
:1051400070401322FEF781B92DE9F047064608A802
:10515000904690E8300489461F46142200212846D4
:1051600009F095F90021CAF80010B8F1000F03D03A
:10517000B9F1000F03D114E03878C00711D02068CE
:10518000FCF78DF8C0BBB8F1000F07D120681230D2
:1051900028602068143068602068A8602168CAF818
:1051A00000103878800724D56068FCF796F818BBA3
:1051B000B9F1000F21D0FFF7E4F80168C6F86811D3
:1051C0008188A6F86C11807986F86E0101F013FDD4
:1051D000F94FEF60626862B196F8680106F26911F2
:1051E00040081032FEF7FDF810223946606809F0D9
:1051F00024F90020BDE8F08706E0606820B1E8608F
:105200006068C6F86401F4E71020F3E730B505469E
:1052100008780C4620F00F00401C20F0F0011031FF
:1052200021700020607095F8230030B104280FD061
:10523000052811D0062814D0FFDF20780121B1EB1A
:10524000101F04D295F8200000F01F00607030BDE0
:1052500021F0F000203002E021F0F000303020702A
:10526000EBE721F0F0004030F9E7F0B591B002270C
:1052700015460C4606463A46ADF80870092103ABC0
:1052800005F063F80490002810D004208DF8040085
:105290008DF80170E034099605948DF818500AA92C
:1052A000684610F0FCFA00B1FFDF012011B0F0BD3C
:1052B00010B588B00C460A99ADF80000CBB118685B
:1052C000CDF80200D3F80400CDF80600ADF80A20AE
:1052D000102203A809F0B1F868460DF0F3FA03F0C4
:1052E000A2FF002803D1A17F41F01001A17708B0EF
:1052F00010BD0020CDF80200E6E72DE9F84F064684
:10530000808A0D4680B28246FEF79CF804463078CB
:10531000DFF8A48200274FF00209A8F120080F2827
:1053200070D2DFE800F06FF23708387D8CC8F1F0FA
:10533000EFF35FF3F300A07F00F00300022809D031
:105340005FF0000080F0010150460EF0AFFD050057
:1053500003D101E00120F5E7FFDF98F85C10C907F1
:1053600002D0D8F860000BE0032105F11D0012F017
:10537000BEF8D5F81D009149B0FBF1F201FB120017
:10538000C5F81D0070686867B068A8672078252890
:1053900000D0FFDFCAE0A07F00F00300022809D0A0
:1053A0005FF0000080F0010150460EF07FFD060026
:1053B00003D101E00120F5E7FFDF3078810702D556
:1053C0002178252904D040F001003070BDE8F88F25
:1053D00085F80090307F287106F11D002D36C5E953
:1053E0000206F3E7A07F00F00300022808D00020A7
:1053F00080F0010150460EF059FD040004D102E096
:105400000120F5E7A7E1FFDF2078C10604D50720DA
:1054100028703D346C60D9E740F008002070D5E773
:10542000E07F000700D5FFDF307CB28800F0010389
:1054300001B05046BDE8F04F092106F064B804B948
:10544000FFDF716821B1102204F1240008F0F5FF9C
:1054500028212046FDF75EFEA07F00F00300022811
:105460000ED104F12400002300901A462146504634
:10547000FFF71EFF112807D029212046FDF74AFE1D
:10548000307A84F82000A1E7A07F000700D5FFDF75
:1054900014F81E0F40F008002070E782A761E76152
:1054A000C109607861F34100014660F382016170D7
:1054B000307AE0708AE7A07F00F00300022809D06C
:1054C0005FF0000080F0010150460EF0EFFC040098
:1054D00003D101E00120F5E7FFDF022104F185009F
:1054E00012F005F80420287004F5B4706860B4F870
:1054F00085002882304810387C346C61C5E9028010
:1055000064E703E024E15BE02DE015E0A07F00F01C
:105510000300022807D0002080F0010150460EF061
:10552000C5FC18B901E00120F6E7FFDF324621464D
:105530005046BDE8F84FE8E504B9FFDF20782128A0
:10554000A1D93079012803D1E07F40F00800E0774D
:10555000324621465046FFF7D8FD2046BDE8F84FB9
:105560002321FDF7D7BD3279AA8005F1080309216F
:10557000504604F0EAFEE86010B10520287025E7E7
:10558000A07F00F00300022808D0002080F0010175
:1055900050460EF08BFC040003D101E00120F5E73A
:1055A000FFDF04F1620102231022081F0EF005FB49
:1055B00007703179417009E75002002040420F0026
:1055C000A07F00F00300022808D0002080F0010135
:1055D00050460EF06BFC050003D101E00120F5E719
:1055E000FFDF95F8840000F0030001287AD1A07F46
:1055F00000F00307E07F10F0010602D0022F04D173
:1056000033E095F8A000C0072BD0D5F8601121B386
:1056100095F88320087C62F387000874A17FCA098B
:10562000D5F8601162F341000874D5F8601166F393
:1056300000000874AEB1D5F86001102204F1240115
:10564000883508F0FAFE287E40F001002876287898
:1056500020F0010005F8880900E016B1022F04D0FF
:105660002DE095F88800C00727D0D5F85C1121B34C
:1056700095F88320087C62F387000874A17FCA092B
:10568000D5F85C1162F341000874D5F85C1166F33B
:10569000000008748EB1D5F85C01102204F12401D9
:1056A000883508F0CAFE287840F0010005F8180B8C
:1056B000287820F0010005F8A009022F44D000202E
:1056C00000EB400005EBC00090F88800800709D58A
:1056D00095F87C00D5F86421400805F17D01103271
:1056E000FDF77FFE8DF8009095F884006A4600F083
:1056F00003008DF8010095F888108DF8021095F8D8
:10570000A0008DF803002146504601F05DFA207894
:10571000252805D0212807D0FFDF2078222803D9AB
:1057200022212046FDF7F6FCA07F00F003000228AE
:105730000CD0002080F0010150460EF0C9FB00287B
:105740003FF44FAEFFDF41E60120B9E70120F1E76A
:10575000706847703AE6FFDF38E670B5FE4C00250A
:1057600084F85C50256610F066F804F110012046BC
:1057700003F0F8FE84F8305070BD70B50D46FDF7AB
:1057800061FE040000D1FFDF4FF4B872002128460B
:1057900008F07DFE04F124002861A07F00F00300E2
:1057A000022809D05FF0010105F1E00010F044F893
:1057B000002800D0FFDF70BD0221F5E70A46014650
:1057C00002F1E00010F059B870B50546406886B0A7
:1057D00001780A2906D00D2933D00E292FD0FFDFFA
:1057E00006B070BD86883046FDF72CFE040000D15F
:1057F000FFDF20782128F3D028281BD168680221F8
:105800000E3001F0D6F9A8B168680821801D01F0BA
:10581000D0F978B104F1240130460DF00FFA03F00D
:1058200002FD00B1FFDF06B02046BDE8704029212F
:10583000FDF770BC06B0BDE8704003F0DABE012190
:1058400001726868C6883046FDF7FCFD040000D18F
:10585000FFDFA07F00F00301022902D120F0100039
:10586000A077207821280AD06868017A09B10079E8
:1058700080B1A07F00F00300022862D0FFDFA07F8C
:1058800000F003000228ABD1FEF72DF80028A7D0C6
:10589000FFDFA5E703F0ADFEA17F08062BD5E07F73
:1058A000C00705D094F8200000F01F00102820D079
:1058B0005FF0050084F82300207829281DD02428D3
:1058C000DDD13146042012F0F9F822212046FDF7FF
:1058D00021FCA07F00F00300022830D05FF0000020
:1058E00080F0010130460EF0F3FA0028C7D0FFDF48
:1058F000C5E70620DEE70420DCE701F0030002280C
:1059000008D0002080F0010130460EF0CFFA0500EB
:1059100003D101E00120F5E7FFDF25212046FDF757
:10592000F9FB03208DF80000694605F1E0000FF057
:105930009BFF0228A3D00028A1D0FFDF9FE7012012
:10594000CEE703F056FE9AE72DE9F04387B099467B
:10595000164688460746FDF775FD04004BD02078B3
:10596000222848D3232846D0E07F000743D4A07FD5
:1059700000F00300022809D05FF0000080F0010170
:1059800038460EF093FA050002D00CE00120F5E74E
:10599000A07F00F00300022805D001210022384634
:1059A0000EF07BFA05466946284601F034F9009866
:1059B00000B9FFDF45B10098E03505612078222865
:1059C00006D0242804D007E000990020086103E0F5
:1059D00025212046FDF79EFB00980121417047627A
:1059E000868001A9C0E902890FF059FF022802D080
:1059F000002800D0FFDF07B0BDE8F08370B586B0A7
:105A00000546FDF71FFD017822291ED9807F00F091
:105A10000300022808D0002080F0010128460EF083
:105A200045FA04002FD101E00120F5E7FFDF2AE06D
:105A3000B4F85E0004F1620630440178427829B17E
:105A400021462846FFF711FCB0B9C9E6ADF804209D
:105A50000921284602AB04F078FC03900028F4D01A
:105A600005208DF80000694604F1E0000FF0FCFE0F
:105A7000022801D000B1FFDF02231022314604F1D9
:105A80005E000EF0D0F8B4F860000028D0D1A7E690
:105A900010B586B00446FDF7D5FC017822291BD944
:105AA000807F00F00300022808D0002080F0010170
:105AB00020460EF0FBF9040003D101E00120F5E7D8
:105AC000FFDF06208DF80000694604F1E0000FF0CA
:105AD000CBFE002800D0FFDF06B010BD2DE9F05F3F
:105AE00005460C4600270078904601093E4604F121
:105AF000080BBA4602297DD0072902D00A2909D10C
:105B000046E0686801780A2905D00D2930D00E29B1
:105B10002ED0FFDFBBE114271C26002C6BD0808821
:105B2000A080FDF78FFC5FEA000900D1FFDF99F844
:105B300017005A46400809F11801FDF752FC686841
:105B4000C0892082696851F8060FC4F812004868BD
:105B5000C4F81600A07E01E03002002020F006000C
:105B600040F00100A07699F81E0040F020014DE0C1
:105B70001A270A26002CD1D0C088A080FDF762FC2D
:105B8000050000D1FFDF59462846FFF73FFB7EE1C5
:105B90000CB1A88BA080287A0B287DD006DC0128C8
:105BA0007BD0022808D0032804D135E00D2875D019
:105BB0000E2874D0FFDF6AE11E270926002CADD025
:105BC000A088FDF73FFC5FEA000900D1FFDF287BDA
:105BD00000F003000128207A1BD020F00100207281
:105BE000297B890861F341002072297BC90861F390
:105BF000820001E041E1F2E02072297B090961F3B2
:105C0000C300207299F81E0040F0400189F81E1070
:105C10003DE140F00100E2E713270D26002CAAD059
:105C2000A088FDF70FFC8146807F00F0030002286A
:105C300008D0002080F00101A0880EF037F905009F
:105C400003D101E00120F5E7FFDF99F81E0000F025
:105C50000302022A50D0686F817801F00301012904
:105C6000217A4BD021F00101217283789B0863F3E4
:105C7000410121728378DB0863F38201217283780A
:105C80001B0963F3C3012172037863F306112172C8
:105C9000437863F3C71103E061E0A9E090E0A1E07D
:105CA000217284F809A0C178A172022A29D0027950
:105CB000E17A62F30001E1720279520862F3410174
:105CC000E1720279920862F38201E1720279D208EC
:105CD00062F3C301E1724279217B62F30001217317
:105CE0004279520862F3410121734279920862F3CA
:105CF00082012173407928E0A86FADE741F00101EE
:105D0000B2E74279E17A62F30001E1724279520826
:105D100062F34101E1724279920862F38201E17219
:105D20004279D20862F3C301E1720279217B62F306
:105D3000000121730279520862F341012173027953
:105D4000920862F3820121730079C00860F3C301F5
:105D5000217399F80000232831D9262140E0182723
:105D60001026E4B3A088FDF76DFB8346807F00F02A
:105D70000300022809D0002080F00101A0880EF065
:105D800095F85FEA000903D101E00120F4E7FFDFA5
:105D9000E868A06099F8000040F0040189F800105C
:105DA00099F80100800708D5012020739BF80000B6
:105DB00023286CD92721584651E084F80CA066E0CE
:105DC00015270F265CB1A088FDF73CFB8146062213
:105DD0005946E86808F0C7FB0120A073A0E041E045
:105DE00048463CE016270926E4B3287B20724EE0A3
:105DF000287B19270E26ACB3C4F808A0A4F80CA081
:105E0000012807D0022805D0032805D0042803D094
:105E1000FFDF0DE0207207E0697B042801F00F012D
:105E200041F0800121721ED0607A20F00300607280
:105E3000A088FDF707FB05460078212827D02328F6
:105E400000D0FFDFA87F00F00300022813D000205D
:105E500080F00101A0880EF03BF822212846FDF7D2
:105E600059F914E004E0607A20F00300401CDEE7FA
:105E7000A8F8006010E00120EAE70CB16888A08073
:105E8000287A68B301280AD002284FD0FFDFA8F88B
:105E900000600CB1278066800020BDE8F09F1527C8
:105EA0000F26002CE4D0A088FDF7CCFA807F00F00C
:105EB0000300022808D0002080F00101A0880DF026
:105EC000F5FF050003D101E00120F5E7FFDFD5F87C
:105ED0001D000622594608F046FB84F80EA0D6E7BE
:105EE00017270926002CC3D0A088FDF7ABFA8146FE
:105EF000807F00F00300022808D0002080F001011C
:105F0000A0880DF0D3FF050003D101E00120F5E7E3
:105F1000FFDF6878800701D5022000E001202072B1
:105F200099F800002328B2D9272159E719270E260E
:105F3000002C9DD0A088FDF785FA5FEA000900D10A
:105F4000FFDFC4F808A0A4F80CA084F808A0A07A89
:105F500040F00300A07299F81E10C90961F3820095
:105F6000A07299F81F2099F81E1012EAD11F05D0CF
:105F700099F8201001F01F0110292BD020F0080003
:105F8000A07299F81F10607A61F3C3006072697A99
:105F900001F003010129A2D140F00400607299F8D8
:105FA0001E0000F003000228E87A16D0217B60F37F
:105FB00000012173AA7A607B62F300006073EA7AC1
:105FC000520862F341012173A97A490861F3410043
:105FD00060735CE740F00800D2E7617B60F300018A
:105FE0006173AA7A207B62F300002073EA7A520878
:105FF00062F341016173A97A490861F3410020739A
:1060000045E710B5FE4C30B10146102204F12000E6
:1060100008F013FA012084F8300010BD10B50446D2
:1060200000F0E9FDF64920461022BDE8104020317D
:1060300008F003BA70B5F24D06004FF0000413D01B
:10604000FBF707F908B110240CE00621304608F0F0
:1060500071FA411C05D028665FF0010085F85C00EC
:1060600000E00724204670BD0020F7E7007810F01C
:106070000F0204D0012A05D0022A0CD110E0000939
:1060800009D10AE00009012807D0022805D0032819
:1060900003D0042801D00720704708700020704703
:1060A0000620704705282AD2DFE800F003070F1703
:1060B0001F00087820F0FF001EE0087820F00F0095
:1060C000401C20F0F000103016E0087820F00F009F
:1060D000401C20F0F00020300EE0087820F00F0087
:1060E000401C20F0F000303006E0087820F00F006F
:1060F000401C20F0F000403008700020704707205E
:1061000070472DE9F041804688B00D4600270846CB
:10611000FBF7ECF8A8B94046FDF794F9040003D06A
:106120002078222815D104E043F2020008B0BDE82F
:10613000F08145B9A07F410603D500F00300022895
:1061400001D01020F2E7A07FC10601D4010702D5DB
:106150000DB10820EAE7E17F090701D50D20E5E749
:1061600000F0030002280DD165B12846FEF75EFF5E
:106170000700DBD1FBF736FB20B9E878800701D5B3
:106180000620D3E7A07F00F00300022808D00020FB
:1061900080F0010140460DF089FE060002D00FE0BC
:1061A0000120F5E7A07F00F0030002280ED00020B8
:1061B00080F00101002240460DF06FFE060007D07E
:1061C000A07F00F00300022804D009E00120EFE7DF
:1061D0000420ABE725B12A4631462046FEF74AFFA8
:1061E0006946304600F017FD009800B9FFDF0099BE
:1061F000022006F1E0024870C1F824804A610022C2
:106200000A81A27F02F00302022A1CD00120087139
:10621000287800F00102087E62F3010008762A78EF
:10622000520862F3820008762A78920862F3C3006B
:1062300008762A78D20862F30410087624212046D2
:10624000FCF768FF33E035B30871301D88613078A2
:10625000400908777078C0F340004877287800F04C
:106260000102887F62F301008877A27FD20962F37E
:1062700082008877E27F62F3C3008877727862F3E6
:1062800004108877A878C87701F1210228462031C8
:10629000FEF711FF03E00320087105200876252191
:1062A0002046FCF737FFA07F20F04000A07701A92F
:1062B00000980FF0F4FA022801D000B1FFDF384651
:1062C00034E72DE9FF4F8DB09A4693460D460027DF
:1062D0000D98FDF7B7F8060006D03078262806D0CE
:1062E000082011B0BDE8F08F43F20200F9E7B07F5B
:1062F00000F00309B9F1020F11D04DB95846FEF76D
:1063000095FE0028EDD1B07F00F00300022806D0F2
:10631000BBF1000F11D0FBF765FA20B10DE0BBF126
:10632000000F50D109E006200DF068FD28B19BF860
:106330000300800701D50620D3E7B07F00F00300FB
:10634000022809D05FF0000080F001010D980DF0E7
:10635000ADFD040003D101E00120F5E7FFDF852D4D
:1063600027D007DCEDB1812D1DD0822D1DD0832DCE
:1063700008D11CE0862D1ED0882D1ED0892D1ED060
:106380008A2D1ED00F2020710F281CD003F02EF96B
:10639000D8B101208DF81400201D06902079B0B1ED
:1063A00056E10020EFE70120EDE70220EBE70320B4
:1063B000E9E70520E7E70620E5E70820E3E709200D
:1063C000E1E70A20DFE707208BE7112089E7B9F131
:1063D000020F03D0A56F03D1A06F02E0656FFAE74B
:1063E000606F804631D04FF0010001904FF0020005
:1063F00000905A4621463046FEF73CFE02E000007F
:10640000300200209BF8000000F00101A87861F341
:106410000100A870B17FC90961F38200A870F17F03
:1064200061F3C300A870617861F30410A87020784C
:10643000400928706078C0F3400068709BF8020043
:10644000E87000206871287103E0022001900120AB
:106450000090A87898F80210C0F3C000C1F3C00102
:10646000084003902CD05046FAF7F3FEC0BBDAF890
:106470000C00FAF7EEFE98BBDAF81C00FAF7E9FE1A
:1064800070BBDAF80C00A060DAF81C00E0606078FD
:1064900098F8012042EA500161F34100607098F8D9
:1064A0000210C0B200EA111161F300006070002018
:1064B0002077009906F11700022907D0012106E094
:1064C000607898F8012002EA5001E5E7002104EB2A
:1064D000810148610199701C022902D0012101E06B
:1064E00028E0002104EB81014861A87800F0030056
:1064F000012857D198F8020000F00300012851D17B
:10650000B9F1020F04D02A1D691D5846FEF7D3FDCC
:10651000287998F8041008408DF82C00697998F8CB
:10652000052011408DF8301008433BD05046FAF753
:1065300090FE08B11020D4E60AF110018B46B9F1A3
:10654000020F17D00846002104F18C03CDE90003A7
:1065500004F5AE7202920BAB2046039AFEF7F4FDEF
:106560000028E8D1B9F1020F08D0504608D14FF009
:10657000010107E050464FF00101E5E75846F5E715
:106580004FF0000104F1A403CDE9000304F5B0725B
:10659000029281F001010CAB2046039AFEF7D4FD74
:1065A0000028C8D16078800733D4A87898F8021002
:1065B000C0F38000C1F3800108432AD0297898F8FD
:1065C0000000F94AB9F1020F06D032F81120430059
:1065D000DA4002F003070AE032F810204B00DA40FC
:1065E00012F0030705D0012F0AD0022F0AD0032F83
:1065F00006D0039A6AB1012906D0042904D008E024
:106600000227F6E70127F4E7012801D0042800D18A
:106610000427B07F40F08000B077F17F039860F3EB
:106620000001F1776078800705D50320A0710398F9
:1066300070B9002029E00220022F18D0012F18D0B5
:10664000042F2AD00020A071B07F20F08000B07706
:1066500025213046FCF75EFD05A904F1E0000FF0AE
:1066600003F910B1022800D0FFDF002039E6A07145
:10667000DFE7A0710D22002104F1200007F007FFE1
:10668000207840F00200207001208DF8100004AA4C
:1066900031460D9800F098FADAE70120A071D7E7AB
:1066A0002DE9F04387B09046894604460025FCF763
:1066B000C9FE060006D03078272806D0082007B08B
:1066C000BDE8F08343F20200F9E7B07F00F0030079
:1066D000022809D05FF0000080F0010120460DF093
:1066E000E5FB040003D101E00120F5E7FFDFA77916
:1066F0005FEA090005D0012821D0B9F1020F26D1A7
:1067000010E0B8F1000F22D1012F05D0022F05D0E3
:10671000032F05D0FFDF2EE00C252CE001252AE019
:10672000022528E04046FAF794FDB0B9032F0ED1B8
:106730001022414604F11D0007F07FFE1BE0012FEF
:1067400002D0022F03D104E0B8F1000F13D00720CC
:10675000B5E74046FAF77DFD08B11020AFE71022FB
:10676000002104F11D0007F092FE0621404607F0CB
:10677000E1FEC4F81D002078252140F002002070C1
:106780003046FCF7C7FC2078C10713D020F0010089
:10679000207002208DF8000004F11D0002908DF899
:1067A00004506946C3300FF05FF8022803D010B1DF
:1067B000FFDF00E02577002081E730B587B00D4688
:1067C0000446FCF73FFE98B1807F00F003000228EA
:1067D00011D0002080F0010120460DF067FB04007D
:1067E0000ED02846FAF735FD38B1102007B030BD7D
:1067F00043F20200FAE70120ECE72078400701D4D9
:106800000820F3E7294604F13D002022054607F061
:1068100014FE207840F01000207001070FD520F002
:106820000800207007208DF80000694604F1E000A0
:1068300001950FF019F8022801D000B1FFDF002008
:10684000D4E770B50D460646FCF7FCFD18B101789B
:10685000272921D102E043F2020070BD807F00F0C1
:106860000300022808D0002080F0010130460DF01E
:106870001DFB040003D101E00120F5E7FFDFA07953
:10688000022809D16078C00706D02A462146304642
:10689000FEF7EBFC10B10FE0082070BDB4F860000B
:1068A0000E280BD204F1620102231022081F0DF002
:1068B00084F9012101704570002070BD112070BD68
:1068C00070B5064614460D460846FAF7C2FC18B9DC
:1068D0002046FAF7E4FC08B1102070BDA6F57F4011
:1068E000FF380ED03046FCF7ADFD38B14178224676
:1068F0004B08811C1846FCF774FD07E043F20200C8
:1069000070BD2046FDF7A5FD0028F9D11021E01D3E
:1069100010F0EDFDE21D294604F1170000F08BF99F
:10692000002070BD2DE9F04104468AB01546884626
:1069300000270846FAF7DAFC18B92846FAF7D6FC19
:1069400018B110200AB0BDE8F0812046FCF77AFDAE
:10695000060003D0307827281BD102E043F2020062
:10696000F0E7B07F00F00300022809D05FF00000DC
:1069700080F0010120460DF099FA040003D101E0F6
:106980000120F5E7FFDF2078400702D56078800717
:1069900001D40820D6E7B07F00F00300022805D01C
:1069A000A06F05D1A16F04E01C610200606FF8E7E1
:1069B000616F407800B19DB1487810B1B8F1000F17
:1069C0000ED0ADB1EA1D06A8E16800F034F910223E
:1069D00006A905F1170007F003FD18B1042707E029
:1069E0000720AFE71022E91D04F12D0007F025FD77
:1069F000B8F1000F06D0102208F1070104F11D00C4
:106A000007F01BFD2078252140F002002070304661
:106A1000FCF780FB2078C10715D020F00100207022
:106A200002208DF8000004F11D0002901030039048
:106A30008DF804706946B3300EF016FF022803D0BB
:106A400010B1FFDF00E0277700207BE7F8B515469F
:106A50000E460746FCF7F6FC040004D020782228F6
:106A600004D00820F8BD43F20200F8BDA07F00F07A
:106A70000300022802D043F20500F8BD3046FAF7C1
:106A8000E8FB18B92846FAF7E4FB08B11020F8BD76
:106A900000953288B31C21463846FEF709FC1128C0
:106AA00015D00028F3D1297C4A08A17F62F3C711D1
:106AB000A177297CE27F61F30002E277297C8908D3
:106AC00084F82010A17F21F04001A177F8BDA17FBB
:106AD0000907FBD4D6F80200C4F83600D6F8060041
:106AE000C4F83A003088A0861022294604F1240018
:106AF00007F0A3FC287C4108E07F61F34100E077C8
:106B0000297C61F38200E077287C800884F82100EA
:106B1000A07F40F00800A0770020D3E770B50D46B5
:106B200006460BB1072070BDFCF78CFC040007D0B3
:106B30002078222802D3A07F800604D4082070BDCC
:106B400043F2020070BDADB1294630460CF076F834
:106B500002F069FB297C4A08A17F62F3C711A17783
:106B6000297CE27F61F30002E277297C890884F8BE
:106B7000201004E030460CF084F802F054FBA17FB2
:106B800021F02001A17770BD70B50D46FCF75AFCCD
:106B9000040005D02846FAF782FB20B1102070BD12
:106BA00043F2020070BD29462046FEF72FFB00206D
:106BB00070BD04E010F8012B0AB100207047491E97
:106BC00089B2F7D20120704770B51546064602F02B
:106BD0000DFD040000D1FFDF207820F00F00801CA5
:106BE00020F0F0002030207066802868A060BDE8AA
:106BF000704002F0FEBC10B5134C94F83000002831
:106C000008D104F12001A1F110000EF06FFE012067
:106C100084F8300010BD10B190F8B9202AB10A48AC
:106C200090F8350018B1002003E0B83001E00648C4
:106C300034300860704708B50023009313460A46B5
:106C40000DF031FB08BD00003002002018B1817842
:106C5000012938D101E010207047018842F6011265
:106C6000881A914231D018DC42F60102A1EB0200F1
:106C700091422AD00CDC41B3B1F5C05F25D06FF44E
:106C8000C050081821D0A0F57060FF381BD11CE05F
:106C900001281AD002280AD117E0B0F5807F14D05D
:106CA00008DC012811D002280FD003280DD0FF28BE
:106CB00009D10AE0B0F5817F07D0A0F580700338D4
:106CC00003D0012801D0002070470F2070470A2808
:106CD0001FD008DC0A2818D2DFE800F0191B1F1F9C
:106CE000171F231D1F21102815D008DC0B2812D0D8
:106CF0000C2810D00D2816D00F2806D10DE0112831
:106D00000BD084280BD087280FD003207047002099
:106D1000704705207047072070470F2070470420F8
:106D20007047062070470C20704743F202007047FE
:106D300038B50C46050041D06946FFF797F90028A1
:106D400019D19DF80010607861F302006070694607
:106D5000681CFFF78BF900280DD19DF800106078B2
:106D600061F3C5006070A978C1F34101012903D026
:106D7000022905D0072038BD217821F0200102E04A
:106D8000217841F020012170410704D0A978C90879
:106D900061F386106070607810F0380F07D0A97822
:106DA000090961F3C710607010F0380F02D16078E4
:106DB000400603D5207840F040002070002038BD08
:106DC00070B504460020088015466068FFF7B0FFE4
:106DD000002816D12089A189884211D8606880785E
:106DE000C0070AD0B1F5007F0AD840F20120B1FBFC
:106DF000F0F200FB1210288007E0B1F5FF7F01D907
:106E00000C2070BD01F201212980002070BD10B559
:106E10000478137864F3000313700478640864F34F
:106E2000410313700478A40864F382031370047898
:106E3000E40864F3C30313700478240964F30413AF
:106E400013700478640964F34513137000788009A3
:106E500060F38613137031B10878C10701D1800740
:106E600001D5012000E0002060F3C713137010BDAE
:106E70004278530702D002F0070306E012F0380F01
:106E800002D0C2F3C20300E001234A7863F3020296
:106E90004A70407810F0380F02D0C0F3C20005E00D
:106EA000430702D000F0070000E0012060F3C502B4
:106EB0004A7070472DE9F04F95B00D00824613D00F
:106EC00012220021284607F0E2FA4FF6FF7B05AABE
:106ED0000121584607F0A3F80024264637464FF410
:106EE00020586FF4205972E0102015B0BDE8F08FE3
:106EF0009DF81E0001280AD1BDF81C1041450BD099
:106F000011EB09000AD001280CD002280CD0042C67
:106F10000ED0052C0FD10DE0012400E00224BDF8B5
:106F20001A6008E0032406E00424BDF81A7002E0A9
:106F3000052400E00624BDF81A10514547D12C74F1
:106F4000BEB34FF0000810AA4FF0070ACDE9028245
:106F5000CDE900A80DF13C091023CDF81090424670
:106F60003146584607F02BF908BBBDF83C002A46CD
:106F7000C0B210A90EF045FDC8B9AE81CFB1CDE9C0
:106F800000A80DF1080C0AAE40468CE8410213231C
:106F900000223946584607F012F940B9BDF83C00C6
:106FA000F11CC01EC0B22A1D0EF02BFD10B1032033
:106FB0009BE70AE0BDF82900E881062C05D19DF881
:106FC0001E00A872BDF81C00288100208DE705A8CE
:106FD00007F031F800288BD0FFF779FE85E72DE91F
:106FE000F0471C46DDE90978DDF8209015460E00D3
:106FF000824600D1FFDF0CB1208818B1D5B1112035
:10700000BDE8F087022D01D0012100E0002106F14A
:10701000140005F0CDFEA8F8000002463B462946C4
:10702000504603F092F9C9F8000008B9A41C3C606E
:107030000020E5E71320E3E7F0B41446DDE904524D
:107040008DB1002314B1022C09D101E0012306E027
:107050000D7CEE0703D025F0010501230D742146B8
:10706000F0BC04F050BA1A80F0BC70472DE9FE4F16
:1070700091461A881C468A468046FAB102AB4946B8
:1070800003F063F9050019D04046A61C27880DF0CF
:1070900050F83246072629463B4600960CF05FFC26
:1070A00020882346CDE900504A4651464046FFF726
:1070B000C3FF002020800120BDE8FE8F0020FBE7F9
:1070C0002DE9F04786B082460EA8904690E8B000C1
:1070D000894604AA05A903A88DE807001E462A468A
:1070E00021465046FFF77BFF039901B1012139701A
:1070F000002818D1FA4904F1140204AB086003987F
:1071000005998DE8070042464946504606F003FAC5
:10711000A8B1092811D2DFE800F005080510100A0F
:107120000C0C0E00002006B06AE71120FBE70720D8
:10713000F9E70820F7E70D20F5E70320F3E7BDF8AE
:1071400010100398CDE9000133462A4621465046E7
:10715000FFF772FFE6E72DE9F04389B01646DDE957
:1071600010870D4681461C461422002103A807F013
:107170008EF9012002218DF810108DF80C008DF889
:107180001170ADF8146064B1A278D20709D08DF8FF
:107190001600E088ADF81A00A088ADF81800A068C5
:1071A000079008A80095CDE90110424603A948467A
:1071B0006B68FFF785FF09B0BDE8F083F0B58BB0D1
:1071C00000240646069407940727089405A8099406
:1071D000019400970294CDE903400D461023224606
:1071E000304606F0ECFF78B90AA806A9019400978A
:1071F0000294CDE90310BDF8143000222946304630
:1072000006F07BFD002801D0FFF761FD0BB0F0BD5B
:1072100006F00CBC2DE9FC410C468046002602F02D
:10722000E5F9054620780D287ED2DFE800F0BC079E
:1072300013B325BD49496383AF959B00A8480068F7
:1072400020B1417841F010014170ADE0404602F0BC
:10725000FDF9A9E0042140460CF028FE070000D10A
:10726000FFDF07F11401404605F037FDA5BB1321F0
:107270004046FDF7CFFB97E0042140460CF016FE98
:10728000070000D1FFDFE088ADF800000020B881E2
:107290009DF80000010704D5C00602D5A088B8817A
:1072A00005E09DF8010040067ED5A088F88105B96B
:1072B000FFDF22462946404601F0ACFC022673E07F
:1072C000E188ADF800109DF8011009060FD50728D8
:1072D00003D006280AD00AE024E0042140460CF03E
:1072E000E5FD060000D1FFDFA088F0810226CDB9C0
:1072F000FFDF17E0042140460CF0D8FD070000D165
:10730000FFDF07F1140006F0C8FB90F0010F02D177
:10731000E079000648D5387C022640F00200387437
:1073200005B9FFDF224600E03DE02946404601F076
:1073300071FC39E0042140460CF0B8FD017C002DC1
:1073400001F00206C1F340016171017C21F00201EC
:107350000174E7D1FFDFE5E702260121404602F094
:10736000A7F921E0042140460CF0A0FD0546606825
:1073700000902089ADF8040001226946404602F0E1
:10738000B8F9287C20F0020028740DE0002DC9D146
:10739000FFDFC7E7022600214046FBF799F8002DE2
:1073A000C0D1FFDFBEE7FFDF3046BDE8FC813EB560
:1073B0000C0009D001466B4601AA002006F084FFAC
:1073C00020B1FFF784FC3EBD10203EBD0020208090
:1073D000A0709DF8050002A900F00700FEF762FE0C
:1073E00050B99DF8080020709DF8050002A9C0F36F
:1073F000C200FEF757FE08B103203EBD9DF808000D
:1074000060709DF80500C109A07861F30410A070B8
:107410009DF80510890961F3C300A0709DF8041060
:10742000890601D5022100E0012161F342009DF8A7
:10743000001061F30000A07000203EBD70B514463E
:1074400006460D4651EA040005D075B10846F9F725
:1074500044FF78B901E0072070BD2946304606F0A8
:107460009AFF10B1BDE8704031E454B12046F9F7FD
:1074700034FF08B1102070BD21463046BDE8704091
:1074800095E7002070BD2DE9FC5F0C46904605464F
:10749000002701780822007A3E46B2EB111F7DD109
:1074A00004F10A0100910A31821E4FF0020A04F130
:1074B000080B0191092A72D2DFE802F0EDE005F530
:1074C00028287BAACE00688804210CF0EFFC060077
:1074D00000D1FFDFB08928B152270726C3E00000A2
:1074E0009402002051271026002C7DD06888A080AF
:1074F0000120A071A88900220099FFF79FFF0028B2
:1075000073D1A8892081288AE081D1E0B5F8129052
:10751000072824D1E87B000621D5512709F1140062
:1075200086B2002CE1D0A88900220099FFF786FFDF
:1075300000285AD16888A08084F806A0A8892081F4
:107540000120A073288A2082A4F81290A88A0090B3
:1075500068884B46A969019A01F038FBA8E05027DA
:1075600009F1120086B2002C3ED0A88900225946AB
:10757000FFF764FF002838D16888A080A889E080E0
:10758000287A072813D002202073288AE081E87B1C
:10759000C0096073A4F81090A88A01E085E082E039
:1075A000009068884B4604F11202A969D4E70120D3
:1075B000EAE7B5F81290512709F1140086B2002CC1
:1075C00066D0688804210CF071FC83466888A0802E
:1075D000A88900220099FFF731FF00286ED184F8B6
:1075E00006A0A889208101E052E067E00420A07392
:1075F000288A2082A4F81290A88A009068884B46B6
:10760000A969019A01F0E2FAA989ABF80E104FE0DE
:107610006888FBF717FF0746688804210CF046FCD2
:10762000064607B9FFDF06B9FFDF687BC00702D057
:107630005127142601E0502712264CB36888A080F9
:10764000502F06D084F806A0287B594601F0CEFAC8
:107650002EE0287BA11DF9E7FE49A88949898142CE
:1076600005D1542706269CB16888A08020E05327C6
:107670000BE06888A080A889E08019E06888042170
:107680000CF014FC00B9FFDF55270826002CF0D1C0
:10769000A8F8006011E056270726002CF8D068886B
:1076A000A080002013E0FFDF02E0012808D0FFDF08
:1076B000A8F800600CB1278066800020BDE8FC9F20
:1076C00057270726002CE3D06888A080687AA0712D
:1076D000EEE7401D20F0030009B14143091D01EB15
:1076E0004000704713B5DB4A00201071009848B184
:1076F000002468460CF0F7F9002C02D1D64A009914
:1077000011601CBD01240020F4E770B50D4614463D
:10771000064686B05C220021284606F0B8FE04B971
:10772000FFDFA0786874A2782188284601F089FAE2
:107730000020A881E881228805F11401304605F077
:10774000B0FA6A460121304606F069FC1AE000BF33
:107750009DF80300000715D5BDF806103046FFF769
:107760002DFD9DF80300BDF8061040F010008DF8C7
:107770000300BDF80300ADF81400FF233046059A5E
:1077800006F0D1FD684606F056FC0028E0D006B0B1
:1077900070BD10B50C4601F1140005F0BAFA0146AF
:1077A000627C2046BDE8104001F080BA30B5044646
:1077B000A84891B04FF6FF75C18905AA284606F082
:1077C0002EFC30E09DF81E00A0422AD001282AD1CC
:1077D000BDF81C00B0F5205F03D042F601018842DD
:1077E00021D1002002AB0AAA0CA9019083E807006E
:1077F00007200090BDF81A1010230022284606F03A
:10780000DEFC38B9BDF828000BAAC0B20CA90EF0F6
:10781000F8F810B1032011B030BD9DF82E00A04241
:1078200001D10020F7E705A806F005FC0028C9D023
:107830000520F0E770B5054604210CF037FB040085
:1078400000D1FFDF04F114010C46284605F045FA8B
:1078500021462846BDE8704005F046BA70B58AB0AA
:107860000C460646FBF7EEFD050014D028782228CA
:1078700027D30CB1A08890B101208DF80C00032013
:107880008DF8100000208DF8110054B1A088ADF8DB
:107890001800206807E043F202000AB070BD09201A
:1078A000FBE7ADF818000590042130460CF0FEFA15
:1078B000040000D1FFDF04F1140005F040FA0007D6
:1078C00001D40820E9E701F091FE60B108A8022187
:1078D0000094CDE9011095F8232003A93046636890
:1078E000FFF7EEFBD9E71120D7E72DE9F04FB2F80B
:1078F00002A0834689B0154689465046FBF7A2FD93
:107900000746042150460CF0D1FA0026044605969D
:107910004FF002080696ADF81C6007B9FFDF04B906
:10792000FFDF4146504603F055FF50B907AA06A9AC
:1079300005A88DE807004246214650466368FFF7D8
:107940004EFB444807AB0660DDE9051204F1140064
:10795000CDF80090CDE90320CDE9013197F823203F
:10796000594650466B6805F033FA06000AD0022EDD
:1079700004D0032E14D0042E00D0FFDF09B030460F
:10798000BDE8F08FBDF81C000028F7D00599CDE9BF
:1079900000104246214650466368FFF74DFBEDE775
:1079A000687840F008006870E8E710B50C46FFF70B
:1079B000BFF900280BD1607800F00701012905D13B
:1079C00010F0380F02D02078810601D5072010BDB5
:1079D00040F0C8002070002010BD2DE9F04F99B094
:1079E00004464FF000081B48ADF81C80ADF820801D
:1079F000ADF82480A0F80880ADF81480ADF81880A8
:107A0000ADF82880ADF82C80007916460D46474623
:107A1000012808D0022806D0032804D0042802D068
:107A2000082019B0ACE72046F9F713FCF0BB284654
:107A3000F9F70FFCD0BB6068F9F758FCB0BB606881
:107A400068B160892189884202D8B1F5007F05D9E3
:107A50000C20E6E7940200201800002080460EAAC1
:107A600006A92846FFF7ACF90028DAD168688078C3
:107A7000C0F34100022808D19DF8190010F0380F1A
:107A800003D02869F9F729FC80B905A92069FFF717
:107A90004FF90028C5D1206950B1607880079DF862
:107AA000150000F0380002D5F0B301E011E0D8BBBA
:107AB0009DF8140080060ED59DF8150010F0380FC3
:107AC00003D06068F9F709FC18B96068F9F70EFC93
:107AD00008B11020A5E70BA906A8FFF7C9F99DF882
:107AE0002D000BA920F00700401C8DF82D006069C7
:107AF000FFF75BFF002894D10AA9A069FFF718F9E6
:107B000000288ED19DF8280080062BD4A06940B1B2
:107B10009DF8290000F00701012923D110F0380F4A
:107B200020D0E06828B100E01CE00078D0B11C282B
:107B300018D20FAA611C2046FFF769F901213846C7
:107B400061F30F2082468DF85210B94642F60300C9
:107B50000F46ADF850000DF13F0218A928680DF04E
:107B600052FF08B107205CE79DF8600015A9CDF829
:107B70000090C01CCDE9019100F0FF0B00230BF237
:107B80000122514614A806F075F9E8BBBDF854006F
:107B90000C90FB482A8929690092CDE901106B8974
:107BA000BDF838202868069906F064F9010077D1FD
:107BB00020784FF0020AC10601D4800616D58DF850
:107BC000527042F60210ADF85000CDF80C9008A9A2
:107BD00003AACDF800A0CDE90121002340F2032241
:107BE00014A80B9906F046F9010059D1E4484D4616
:107BF00008380089ADF83D000FA8CDE90290CDF816
:107C00000490CDF8109000E00CE04FF007095B46BF
:107C10000022CDF80090BDF854104FF6FF7006F02A
:107C20006CF810B1FFF753F8FBE69DF83C00000636
:107C300024D52946012060F30F218DF852704FF4AE
:107C400024500395ADF8500062789DF80C00002395
:107C500062F300008DF80C006278CDF800A05208A5
:107C600062F341008DF80C0003AACDE9012540F232
:107C7000032214A806F0FEF8010011D1606880B359
:107C80002069A0B905A906A8FFF7F2F86078800777
:107C900007D49DF8150020F038008DF8150006E097
:107CA00077E09DF8140040F040008DF814008DF846
:107CB000527042F60110ADF85000208940F20121C7
:107CC000B0FBF1F201FB1202606809ABCDF8008055
:107CD000CDE90103002314A8059906F0CBF80100B3
:107CE00057D12078C00728D00395A06950B90AA9B8
:107CF00006A8FFF7BDF89DF8290020F00700401CFA
:107D00008DF829009DF8280007A940F040008DF863
:107D100028008DF8527042F60310ADF8500003AA07
:107D2000CDF800A0CDE90121002340F2032214A8E0
:107D30000A9906F09FF801002BD1E06868B3294644
:107D4000012060F30F218DF8527042F60410ADF857
:107D50005000E068002302788DF8582040788DF8B4
:107D60005900E06816AA4088ADF85A00E06800792A
:107D70008DF85C00E068C088ADF85D00CDF800903B
:107D8000CDE901254FF4027214A806F073F8010042
:107D900003D00C9800F0B6FF43E679480321083879
:107DA000017156B100893080BDF824007080BDF8A3
:107DB0002000B080BDF81C00F080002031E670B5D6
:107DC00001258AB016460B46012802D0022816D19A
:107DD00004E08DF80E504FF4205003E08DF80E5063
:107DE00042F60100ADF80C005BB10024601C60F3AA
:107DF0000F2404AA08A918460DF005FE18B10720A3
:107E00004BE5102049E504A99DF820205C48CDE908
:107E10000021801E02900023214603A802F20122C5
:107E200006F028F810B1FEF752FF36E5544808383E
:107E30000EB1C1883180057100202EE5F0B593B0F8
:107E4000044601268DF83E6041F601000F46ADF86C
:107E50003C0011AA0FA93046FFF7B1FF002837D127
:107E60002000474C4FF00005A4F1080432D01C223A
:107E7000002102A806F00BFB9DF808008DF83E607B
:107E800040F020008DF8080042F60520ADF83C00D7
:107E900004200797ADF82C00ADF8300039480A905F
:107EA0000EA80D900E950FA80990ADF82E506A46B9
:107EB00009A902A8FFF791FD002809D1BDF800002B
:107EC0006081BDF80400A081401CE0812571002084
:107ED00013B0F0BD6581A581BDF84400F4E72DE93C
:107EE000F74F2749A0B00024083917940A79A14612
:107EF000012A04D0022A02D0082023B040E5CA8813
:107F0000824201D00620F8E721988A46824201D1B8
:107F10000720F2E70120214660F30F21ADF8480069
:107F20004FF6FF788DF86E000691ADF84A8042F664
:107F3000020B8DF872401CA9ADF86CB0ADF8704022
:107F40001391ADF8508012A806F0A4F800252E4633
:107F50002F460DAB072212A9404606F09EF898B1B5
:107F60000A2861D1B5B3AEB3ADF86450ADF8666020
:107F70009DF85E008DF8144019AC012868D06FE0C0
:107F80009C020020266102009DF83A001FB30128E0
:107F900059D1BDF8381059451FD118A809A9019425
:107FA0000294CDE9031007200090BDF8361010238D
:107FB0000022404606F003F9B0BBBDF8600004287B
:107FC00001D006284AD1BDF82410219881423AD127
:107FD0000F2092E73AE0012835D1BDF83800B0F51E
:107FE000205F03D042F6010188422CD1BAF8060086
:107FF000BDF83610884201D1012700E0002705B105
:108000009EB1219881421ED118A809AA0194029418
:10801000CDE90320072000900D46102300224046A2
:1080200006F0CDF800B902E02DE04E460BE0BDF8B9
:108030006000022801D0102810D1C0B217AA09A9E7
:108040000DF0DFFC50B9BDF8369082E7052054E70B
:1080500005A917A8221D0DF0D6FC08B103204CE796
:108060009DF814000023001DC2B28DF81420229840
:108070000092CDE901401BA8069905F0FBFE10B95E
:1080800002228AF80420FEF722FE36E710B50B46DE
:10809000401E88B084B205AA00211846FEF7B7FE3C
:1080A00000200DF1080C06AA05A901908CE8070034
:1080B000072000900123002221464FF6FF7005F0B3
:1080C0001CFE0446BDF81800012800D0FFDF204642
:1080D000FEF7FDFD08B010BDF0B5FF4F044687B0B8
:1080E00038790E46032804D0042802D0082007B0AF
:1080F000F0BD04AA03A92046FEF762FE0500F6D1F2
:1081000060688078C0F3410002280AD19DF80D0014
:1081100010F0380F05D02069F9F7DFF808B110200A
:10812000E5E7208905AA21698DE807006389BDF884
:1081300010202068039905F09DFE10B1FEF7C7FDE1
:10814000D5E716B1BDF814003080042038712846F8
:10815000CDE7F8B50C0006460BD001464FF6FF758B
:1081600000236A46284606F0AFF820B1FEF7AFFDBF
:10817000F8BD1020F8BD69462046FEF7D9FD00285D
:10818000F8D1A078314600F001032846009A06F0A5
:10819000CAF8EBE730B587B0144600220DF1080CA1
:1081A00005AD01928CE82C00072200920A46014698
:1081B00023884FF6FF7005F0A0FDBDF81410218054
:1081C000FEF785FD07B030BD70B50D4604210BF0FC
:1081D0006DFE040000D1FFDF294604F11400BDE864
:1081E000704004F0A5BD70B50D4604210BF05EFE95
:1081F000040000D1FFDF294604F11400BDE87040FF
:1082000004F0B9BD70B50D4604210BF04FFE04001B
:1082100000D1FFDF294604F11400BDE8704004F0EE
:10822000D1BD70B5054604210BF040FE040000D11D
:10823000FFDF214628462368BDE870400122FEF793
:1082400015BF70B5064604210BF030FE040000D1C6
:10825000FFDF04F1140004F05CFD401D20F0030575
:1082600011E0011D00880022431821463046FEF728
:10827000FDFE00280BD0607CABB2684382B2A068E0
:10828000011D0BF0D0FCA06841880029E9D170BD28
:1082900070B5054604210BF009FE040000D1FFDF94
:1082A000214628466368BDE870400222FEF7DEBE24
:1082B00070B50E46054601F099F9040000D1FFDFC4
:1082C0000120207266726580207820F00F00001D6A
:1082D00020F0F00040302070BDE8704001F089B916
:1082E00010B50446012900D0FFDF2046BDE810404C
:1082F0000121FAF7EDB82DE9F04F97B04FF0000AE1
:108300000C008346ADF814A0D04619D0E06830B117
:10831000A068A8B10188ADF81410A0F800A05846D4
:10832000FBF790F8070043F2020961D03878222861
:108330005CD3042158460BF0B9FD050005D103E0DC
:10834000102017B0BDE8F08FFFDF05F1140004F036
:10835000E0FC401D20F00306A078012803D002288D
:1083600001D00720EDE7218807AA584605F057FEFF
:1083700030BB07A805F05FFE10BB07A805F05BFE49
:1083800048B99DF82600012805D1BDF82400A0F5C4
:108390002451023902D04FF45050D2E7E068B0B116
:1083A000CDE902A00720009005AACDF804A0049210
:1083B000A2882188BDF81430584605F09EFC10B103
:1083C000FEF785FCBDE7A168BDF8140008809DF8A4
:1083D0001F00C00602D543F20140B2E70B9838B146
:1083E000A1780078012905D080071AD40820A8E7D1
:1083F0004846A6E7C007F9D002208DF83C00A868DF
:108400004FF00009A0B1697C4288714391420FD9B5
:108410008AB2B3B2011D0BF0BCFB8046A0F800A0ED
:1084200006E003208DF83C00D5F800804FF00109EC
:108430009DF8200010F0380F00D1FFDF9DF82000DC
:108440002649C0F3C200084497F8231010F8010C25
:10845000884201D90F2074E72088ADF8400014A9A4
:108460000095CDE90191434607220FA95846FEF732
:1084700027FE002891D19DF8500050B9A07801281E
:1084800007D1687CB3B2704382B2A868011D0BF0BB
:1084900094FB002055E770B5064615460C46084685
:1084A000FEF7D4FB002805D12A4621463046BDE818
:1084B000704084E470BD12E570B51E4614460D0090
:1084C0000ED06CB1616859B160B10349C98881426D
:1084D00008D0072070BD000094020020296102002E
:1084E0001020F7E72068FEF7B1FB0028F2D13246F2
:1084F00021462846BDE87040FFF76FBA70B51546B3
:108500000C0006D038B1FE490989814203D007200A
:10851000E0E71020DEE72068FEF798FB0028D9D1BD
:1085200029462046BDE87040D6E570B5064686B0BF
:108530000D4614461046F8F7B2FED0BB6068F8F757
:10854000D5FEB0BBA6F57F40FF3803D03046FAF722
:1085500079FF80B128466946FEF7ACFC00280CD1B3
:108560009DF810100F2008293DD2DFE801F0080621
:108570000606060A0A0843F2020006B0AAE703202C
:10858000FBE79DF80210012908D1BDF80010B1F5F4
:10859000C05FF2D06FF4C052D142EED09DF8061009
:1085A00001290DD1BDF80410A1F52851062907D2E3
:1085B00000E029E0DFE801F0030304030303DCE744
:1085C0009DF80A1001290FD1BDF80810B1F5245FFC
:1085D000D3D0A1F60211B1F50051CED00129CCD0F3
:1085E000022901D1C9E7FFDF606878B9002305AA35
:1085F0002946304605F068FE10B1FEF768FBBCE77F
:108600009DF81400800601D41020B6E76188224648
:1086100028466368FFF7BEFDAFE72DE9F0438146CA
:1086200087B0884614461046F8F739FE18B1102076
:1086300007B0BDE8F083002306AA4146484605F08E
:1086400043FE10B1FEF743FBF2E79DF81800C006A9
:1086500002D543F20140EBE70025072705A8019565
:1086600000970295CDE9035062884FF6FF734146AB
:10867000484605F0A4FD060013D16068F8F70FFE28
:1086800060B960680195CDE9025000970495238890
:1086900062884146484605F092FD0646BDF8140042
:1086A00020803046CEE739B1954B0A889B899A42A3
:1086B00002D843F2030070471DE610B586B0904C17
:1086C0000423ADF81430638943B1A4898C4201D2EC
:1086D000914205D943F2030006B010BD0620FBE726
:1086E000ADF81010002100910191ADF80030022189
:1086F0008DF8021005A9029104A90391ADF812208A
:108700006946FFF7F8FDE7E72DE9FC4781460D468E
:108710000846F8F79EFD88BB4846FAF793FE5FEAE5
:1087200000080AD098F80000222829D304214846DE
:108730000BF0BCFB070005D103E043F20200BDE8EB
:10874000FC87FFDF07F1140004F0F9FA06462878E9
:10875000012803D0022804D00720F0E7B0070FD586
:1087600002E016F01C0F0BD0A8792C1DC00709D011
:10877000E08838B1A068F8F76CFD18B11020DEE78A
:108780000820DCE721882A780720B1F5847F35D0DE
:108790001EDC40F20315A1F20313A94226D00EDC21
:1087A000B1F5807FCBD003DCF9B1012926D1C6E732
:1087B000A1F58073013BC2D0012B1FD113E0012B27
:1087C000BDD0022B1AD0032BB9D0042B16D112E046
:1087D000A1F20912082A11D2DFE802F00B040410FA
:1087E00010101004ABE7022AA9D007E0012AA6D096
:1087F00004E0320700E0F206002AA0DACDB200F071
:10880000F5FE50B198F82300CDE90005FA8923461A
:1088100039464846FEF79FFC91E711208FE72DE986
:10882000F04F8BB01F4615460C4683460026FAF7DC
:1088300009FE28B10078222805D208200BB081E576
:1088400043F20200FAE7B80801D00720F6E7032F49
:1088500000D100274FF6FF79CCB1022D71D320460D
:10886000F8F744FD30B904EB0508A8F10100F8F76A
:108870003DFD08B11020E1E7AD1E38F8028CAAB228
:108880002146484605F081FE40455AD1ADB21C490B
:10889000B80702D58889401C00E001201FFA80F843
:1088A000F80701D08F8900E04F4605AA4146584697
:1088B00005F0B5FB4FF0070A4FF00009FCB1204668
:1088C00008E0408810283CD8361D304486B2AE42BD
:1088D00037D2A01902884245F3D352E09DF8170021
:1088E00002074ED57CB304EB0608361DB8F80230FB
:1088F000B6B2102B25D89A19AA4222D802E040E03D
:1089000094020020B8F8002091421AD1C0061BD56D
:10891000CDE900A90DF1080C0AAAA11948468CE876
:108920000700B8F800100022584605F0E6F910B12B
:10893000FEF7CDF982E7B8F80200BDF828108842AA
:1089400002D00B207AE704E0B8F80200304486B287
:1089500006E0C00604D55846FEF730FC00288AD150
:108960009DF81700BDF81A1020F010008DF81700C0
:10897000BDF81700ADF80000FF235846009A05F037
:10898000D2FC05A805F057FB18B9BDF81A10B9427A
:10899000A4D9042158460BF089FA040000D1FFDF66
:1089A000A2895AB1CDE900A94D4600232146584677
:1089B000FEF7D1FB0028BDD1A5813FE700203DE7B0
:1089C0002DE9FF4F8BB01E4617000D464FF00004F7
:1089D00012D0B00802D007200FB0B3E4032E00D1AC
:1089E00000265DB10846F8F778FC28B93888691E7A
:1089F0000844F8F772FC08B11020EDE7C74AB00749
:108A000001D5D18900E00121F0074FF6FF7802D0AF
:108A1000D089401E00E0404686B206AA0B9805F0B9
:108A2000FEFA4FF000094FF0070B0DF1140A38E081
:108A30009DF81B00000734D5CDF80490CDF800B0A8
:108A4000CDF80890CDE9039A434600220B9805F033
:108A5000B6FB60BB05B3BDF814103A882144281951
:108A6000091D8A4230D3BDF81E2020F8022BBDF824
:108A7000142020F8022BCDE900B9CDE90290CDF801
:108A800010A0BDF81E10BDF8143000220B9805F0A0
:108A900096FB08B103209FE7BDF814002044001D99
:108AA00084B206A805F0C7FA20B10A2806D0FEF75E
:108AB0000EF991E7BDF81E10B142B9D934B17DB1BC
:108AC0003888A11C884203D20C2085E7052083E763
:108AD00022462946404605F058FD014628190180E6
:108AE000A41C3C80002077E710B50446F8F7D7FBBC
:108AF00008B1102010BD8948C0892080002010BD19
:108B0000F0B58BB00D4606461422002103A805F0EF
:108B1000BEFC01208DF80C008DF8100000208DF8AF
:108B20001100ADF814503046FAF78CFC48B10078CB
:108B3000222812D3042130460BF0B8F9040005D1E5
:108B400003E043F202000BB0F0BDFFDF04F11400BC
:108B5000074604F0F4F8800601D40820F3E7207CEF
:108B6000022140F00100207409A80094CDE9011011
:108B7000072203A930466368FEF7A2FA20B1217CE0
:108B800021F001012174DEE729463046F9F791FC16
:108B900008A9384604F0C2F800B1FFDFBDF8204054
:108BA000172C01D2172000E02046A84201D92C46FC
:108BB00002E0172C00D2172421463046FFF713FBA2
:108BC00021463046F9F799F90020BCE7F8B51C4674
:108BD00015460E46069F0BF09AFA2346FF1DBCB2BF
:108BE00031462A4600940AF086FEF8BD70B50C4660
:108BF00005460E220021204605F049FC0020208079
:108C00002DB1012D01D0FFDF64E4062000E0052036
:108C1000A0715FE410B548800878134620F00F007B
:108C2000001D20F0F00080300C4608701422194618
:108C300004F1080005F001FC00F0DBFC374804609B
:108C400010BD2DE9F047DFF8D890491D064621F008
:108C5000030117460C46D9F800000AF062FF050030
:108C600000D1FFDF4FF000083560A5F800802146F5
:108C7000D9F800000AF055FF050000D1FFDF75604C
:108C8000A5F800807FB104FB07F1091D0BD0D9F8CE
:108C900000000AF046FF040000D1FFDFB460C4F812
:108CA0000080BDE8F087C6F80880FAE72DE9F041BA
:108CB0001746491D21F00302194D06460168144666
:108CC00028680AF059FF2246716828680AF054FFA4
:108CD0003FB104FB07F2121D03D0B16828680AF007
:108CE0004BFF04200BF08AF8044604200BF08EF8AA
:108CF000201A012804D12868BDE8F0410AF006BF17
:108D0000BDE8F08110B50C4605F058F900B1FFDF61
:108D10002046BDE81040FDF7DABF000094020020B5
:108D20001800002038B50C468288817B19B1418932
:108D3000914200D90A462280C188121D90B26A462B
:108D40000AF0B2F8BDF80000032800D30320C1B236
:108D5000208801F020F838BD38B50C468288817B28
:108D600019B10189914200D90A462280C188121D99
:108D700090B26A460AF098F8BDF80000022800D3C5
:108D80000220C1B2208801F006F8401CC0B238BDF4
:108D90002DE9FF5F82468B46F74814460BF103022C
:108DA000D0E90110CDE9021022F0030201A84FF42E
:108DB000907101920AF097FEF04E002C02D1F0491A
:108DC000019A8A60019901440191B57F05F101057D
:108DD00004D1E8B20CF098FD00B1FFDF019800EB80
:108DE0000510C01C20F0030101915CB9707AB27AC1
:108DF0001044C2B200200870B08C80B204F03DFF75
:108E000000B1FFDF0198716A08440190214601A872
:108E100000F084FF80460198C01C20F00300019000
:108E2000B37AF27A717A04B100200AF052FF019904
:108E300008440190214601A800F0B8FFCF48002760
:108E40003D4690F801900CE0284600F04AFF0646A7
:108E500081788088F9F7E8F871786D1C00FB01775C
:108E6000EDB24D45F0D10198C01C20F003000190F7
:108E700004B100203946F9F7E2F8019900270844C7
:108E80000190BE483D4690F801900CE0284600F065
:108E900028FF0646C1788088FEF71BFC71786D1CA0
:108EA00000FB0177EDB24D45F0D10198C01C20F0D8
:108EB0000300019004B100203946FEF713FC01992C
:108EC0004FF0000908440190AC484D4647780EE049
:108ED000284600F006FF0646807B30B106F1080008
:108EE00002F09CF9727800FB02996D1CEDB2BD4254
:108EF000EED10198C01C20F00300019004B10020C5
:108F00009F494A78494602F08DF901990844019039
:108F1000214601A800F0B8FE0198C01D20F007000E
:108F20000190DAF80010814204D3A0EB0B01B1F5F7
:108F3000803F04DB4FF00408CAF8000004E0CAF8E0
:108F40000000B8F1000F03D0404604B0BDE8F09F28
:108F500084BB8C490020019A0EF044FEFBF714FA02
:108F6000864C207F0090607F012825D0002328B305
:108F70000022824800211030F8F73AFA00B1FFDFF2
:108F80007E49E07F2031FEF759FF00B1FFDF7B48CB
:108F90004FF4F6720021443005F079FA7748042145
:108FA000443080F8E91180F8EA11062180F8EB11CD
:108FB000032101710020C8E70123D8E702AAD8E7FE
:108FC00070B56E4C06464434207804EB4015E078CA
:108FD000083598B9A01990F8E80100280FD0A078BA
:108FE0000F2800D3FFDF20220021284605F04FFA8A
:108FF000687866F3020068700120E070284670BD52
:109000002DE9F04105460C460027007805219046E1
:109010003E46B1EB101F00D0FFDF287A50B1012887
:109020000ED0FFDFA8F800600CB12780668000201A
:10903000BDE8F0810127092674B16888A08008E0A6
:109040000227142644B16888A0802869E060A88AB5
:109050002082287B2072E5E7A8F80060E7E730B5BA
:10906000464C012000212070617020726072032242
:10907000A272E07261772177217321740521218327
:109080001F216183607440A161610A21A177E077AB
:1090900039483B4DB0F801102184C07884F8220093
:1090A0004FF4B06060626868C11C21F00301814226
:1090B00000D0FFDF6868606030BD30B5304C1568A7
:1090C000636810339D4202D20420136030BD2B4BE5
:1090D0005D785A6802EB0512107051700320D08041
:1090E000172090800120D0709070002090735878E5
:1090F000401C5870606810306060002030BD70B552
:1091000006461E480024457807E0204600F0E9FDA9
:109110000178B14204D0641CE4B2AC42F5D1002025
:1091200070BDF7B5074608780C4610B3FFF7E7FFA8
:109130000546A7F12006202F06D0052E19D2DFE81C
:1091400006F00F383815270000F0D6FD0DB169780C
:1091500000E00021401AA17880B20844FF2808D816
:10916000A07830B1A088022831D202E060881728A8
:109170002DD20720FEBD000030610200B0030020A8
:109180001C000020000000206E52463578000000D0
:10919000207AE0B161881729EBD3A1881729E8D399
:1091A000A1790029E5D0E1790029E2D0402804D94D
:1091B000DFE7242F0BD1207A48B161884FF6FB708E
:1091C000814202D8A188814201D90420D2E765B941
:1091D000207802AA0121FFF770FF0028CAD1207869
:1091E000FFF78DFF050000D1FFDF052E18D2DFE865
:1091F00006F0030B0E081100A0786870A088E880C4
:109200000FE06088A8800CE0A078A87009E0A07842
:10921000E87006E054F8020FA8606068E86000E0BB
:10922000FFDF0020A6E71A2835D00DDC132832D244
:10923000DFE800F01B31203131272723252D313184
:1092400029313131312F0F00302802D003DC1E28A4
:1092500021D1072070473A3809281CD2DFE800F0F6
:10926000151B0F1B1B1B1B1B07000020704743F225
:109270000400704743F202007047042070470D203D
:1092800070470F2070470820704711207047132047
:109290007047062070470320704710B5007800F033
:1092A000010009F0F3FDBDE81040BCE710B50078FF
:1092B00000F0010009F0F3FDBDE81040B3E70EB582
:1092C000017801F001018DF80010417801F00101F1
:1092D0008DF801100178C1F340018DF8021041783A
:1092E000C1F340018DF80310017889088DF804104E
:1092F000417889088DF8051081788DF80610C178BD
:109300008DF8071000798DF80800684608F0FDFD1B
:10931000FFF789FF0EBD2DE9FC5FDFF8F883FE4CF7
:1093200000264FF490771FE0012000F082FD01201D
:10933000FFF746FE05463946D8F808000AF0F1FB6B
:10934000686000B9FFDF686808F0AAFCB0B1284681
:10935000FAF75EFB284600F072FD28B93A466968C4
:10936000D8F808000AF008FC94F9E9010428DBDACF
:1093700002200AF043FD07460025AAE03A46696844
:10938000D8F808000AF0F8FBF2E7B8F802104046F7
:10939000491C89B2A8F80210B94201D300214180CA
:1093A0000221B8F802000AF081FD002866D0B8F862
:1093B0000200694609F0CFFCFFF735FF00B1FFDF7F
:1093C0009DF80000019078B1B8F802000AF0B1FEF3
:1093D0005FEA000900D1FFDF48460AF020F918B122
:1093E000B8F8020002F0E4F9B8F802000AF08FFEC3
:1093F0005FEA000900D1FFDF48460AF008F9E8BB40
:109400000321B8F802000AF051FD5FEA000B4BD1CE
:10941000FFDF49E0DBF8100010B10078FF284DD0E5
:10942000022000F006FD0220FFF7CAFD82464846F2
:109430000AF0F9F9CAF8040000B9FFDFDAF804000D
:109440000AF0C1FA002100900170B8F802105046ED
:10945000AAF8021002F0B2F848460AF0B6FA00B9CB
:10946000FFDF019800B10126504600F0E8FC18B972
:109470009AF80100000705D5009800E027E0CBF836
:10948000100011E0DBF8101039B10878401C10F022
:10949000FF00087008D1FFDF06E0002211464846B1
:1094A00000F0F0FB00B9FFDF94F9EA01022805DBC8
:1094B000B8F8020002F049F80028ABD194F9E901AC
:1094C000042804DB48460AF0E4FA00B101266D1CCA
:1094D000EDB2BD4204D294F9EA010228BFF655AFBD
:1094E000002E7FF41DAFBDE8FC5F032000F0A1BC9F
:1094F00010B5884CE06008682061AFF2E510F9F71C
:10950000E4FC607010BD844800214438017081483B
:10951000017082494160704770B505464FF0805038
:109520000C46D0F8A410491C05D1D0F8A810C943A6
:109530000904090C0BD050F8A01F01F0010129709B
:10954000416821608068A080287830B970BD06210C
:1095500020460DF0CCFF01202870607940F0C0005B
:10956000607170BD70B54FF080540D46D4F8801016
:10957000491C0BD1D4F88410491C07D1D4F88810A9
:10958000491C03D1D4F88C10491C0CD0D4F880109D
:109590000160D4F884104160D4F888108160D4F858
:1095A0008C10C16002E010210DF0A1FFD4F89000F2
:1095B000401C0BD1D4F89400401C07D1D4F898007B
:1095C000401C03D1D4F89C00401C09D054F8900FE3
:1095D000286060686860A068A860E068E86070BDA6
:1095E0002846BDE8704010210DF081BF4A4800793F
:1095F000E6E470B5484CE07830B3207804EB4010D6
:10960000407A00F00700204490F9E801002800DCCF
:10961000FFDF2078002504EB4010407A00F00700BF
:10962000011991F8E801401E81F8E8012078401CFA
:10963000C0B220700F2800D12570A078401CA07007
:109640000DF0D4FDE57070BDFFDF70BD3EB5054681
:1096500003210AF02BFC044628460AF058FD054673
:1096600004B9FFDF206918B10078FF2800D1FFDFBF
:1096700001AA6946284600F005FB60B9FFDF0AE051
:10968000002202A9284600F0FDFA00B9FFDF9DF88C
:10969000080000B1FFDF9DF80000411E8DF80010AA
:1096A000EED220690199884201D1002020613EBD9F
:1096B00070B50546A0F57F400C46FF3800D1FFDFAE
:1096C000012C01D0FFDF70BDFFF790FF040000D137
:1096D000FFDF207820F00F00401D20F0F000503018
:1096E000207065800020207201202073BDE870404A
:1096F0007FE72DE9F04116460D460746FFF776FF56
:10970000040000D1FFDF207820F00F00401D20F082
:10971000F00005E01C000020F403002048140020A5
:109720005030207067800120207228682061A8884E
:10973000A0822673BDE8F0415BE77FB5FFF7DFFC51
:10974000040000D1FFDF02A92046FFF7EBFA05462F
:1097500003A92046FFF700FB8DF800508DF80100AB
:10976000BDF80800001DADF80200BDF80C00001D9A
:10977000ADF80400E088ADF80600684609F070FB1B
:10978000002800D0FFDF7FBD2DE9F05FFC4E814651
:10979000307810B10820BDE8F09F4846F7F77FFD0C
:1097A00008B11020F7E7F74C207808B9FFF757FC0D
:1097B000A17A607A4D460844C4B200F09DFAA042F6
:1097C00007D2201AC1B22A460020FFF776FC0028F3
:1097D000E1D17168EB48C91C002721F003017160D9
:1097E000B3463E463D46BA463C4690F801800AE004
:1097F000204600F076FA4178807B0E4410FB01553C
:10980000641CE4B27F1C4445F2D10AEB870000EBF4
:10981000C600DC4E00EB85005C46F17A012200EBCD
:109820008100DBF80410451829464846FFF7B0FAD6
:10983000070012D00020FFF762FC05000BD005F1F5
:109840001300616820F00300884200D0FFDF7078C9
:10985000401E7070656038469DE7002229464846E4
:10986000FFF796FA00B1FFDFD9F8000060604FF60D
:10987000FF7060800120207000208CE72DE9F0410E
:109880000446BF4817460D46007810B10820BDE8D1
:10989000F0810846F7F7DDFC08B11020F7E7B94E74
:1098A000307808B9FFF7DBFB601E1E2807D8012CB3
:1098B00023D12878FE2820D8B0770020E7E7A4F14C
:1098C00020001F2805D8E0B23A462946BDE8F041FD
:1098D00027E4A4F140001F2805D829462046BDE80A
:1098E000F04100F0D4BAA4F1A0001F2805D8294601
:1098F0002046BDE8F04100F006BB0720C7E72DE990
:10990000F05F81460F460846F7F7C9FC48B948465C
:10991000F7F7E3FC28B909F1030020F003014945FA
:1099200001D0102037E797484FF0000B4430817882
:1099300069B14178804600EB411408343E883A46CC
:109940000021204600F089FA050004D027E0A7F89E
:1099500000B005201FE7B9F1000F24D03888B042CD
:1099600001D90C251FE0607800F00700824600F066
:1099700060FA08EB0A063A4696F8E8014946401CA8
:1099800086F8E801204600F068FA054696F8E801F6
:10999000401E86F8E801032000F04BFA2DB10C2D93
:1099A00001D0A7F800B02846F5E6754F5046BAF149
:1099B000010F25D002280DD0BAF1030F35D0FFDFFB
:1099C00098F801104046491CC9B288F801100F29C7
:1099D00037D038E0606828B16078000702D460882A
:1099E000FFF734FE98F8EA014446012802D178785E
:1099F000F9F78AFA94F9EA010428E1DBFFDFDFE7EF
:109A0000616821B14FF49072B8680AF0B5F898F81F
:109A1000E9014446032802D17878F9F775FA94F9F8
:109A2000E9010428CCDBFFDFCAE76078C00602D575
:109A30006088FFF70BFE98F9EB010628C0DBFFDF1B
:109A4000BEE780F801B08178491E88F8021096F8C8
:109A5000E801401C86F8E801A5E770B50C4605460C
:109A6000F7F7F7FB18B92046F7F719FC08B11020F3
:109A700070BD28460BF07FFF207008B1002070BD3C
:109A8000042070BD70B505460BF08EFFC4B22846A9
:109A9000F7F723FC08B1102070BD35B128782C7081
:109AA00018B1A04201D0072070BD2046FDF77EFE10
:109AB000052805D10BF07BFF012801D0002070BDE7
:109AC0000F2070BD70B5044615460E460846F7F7E0
:109AD000C0FB18B92846F7F7E2FB08B1102070BDAB
:109AE000022C03D0102C01D0092070BD2A4631462B
:109AF00020460BF086FF0028F7D0052070BD70B51A
:109B000014460D460646F7F7A4FB38B92846F7F782
:109B1000C6FB18B92046F7F7E0FB08B1102070BD6E
:109B20002246294630460BF06EFF0028F7D007206A
:109B300070BD3EB50446F7F7B2FB08B110203EBD3C
:109B4000684608F053F9FFF76EFB0028F7D19DF83F
:109B500006002070BDF808006080BDF80A00A080F3
:109B600000203EBD70B505460C460846F7F7B5FB2C
:109B700020B95CB12068F7F792FB28B1102070BDC6
:109B80001C000020B0030020A08828B121462846F0
:109B9000BDE87040FDF762BE0920F0E770B50546EC
:109BA0000C460846F7F755FBA0BB681E1E280ED8CA
:109BB000032D01D90720E2E705B9FFDFFE4800EBDE
:109BC000850050F8041C2046BDE870400847A5F108
:109BD00020001F2805D821462846BDE87040FAF726
:109BE00042BBA5F160001F2805D821462846BDE8E4
:109BF0007040F8F7DABCF02D0DD0F12D15D0BF2D47
:109C0000D8D1A078218800F0010001F08DFB98B137
:109C10000020B4E703E0A068F7F71BFB08B11020B1
:109C2000ADE7204609F081F902E0207809F0A0F9BB
:109C3000BDE87040FFF7F7BA0820A0E770B504460A
:109C40000D460846F7F72BFB30B9601E1E280FD8CB
:109C50002846F7F7FEFA08B1102090E7012C03D050
:109C6000022C01D0032C01D1062088E7072086E7CB
:109C7000A4F120001F28F9D829462046BDE87040ED
:109C8000FAF762BB09F092BC38B50446CB48007BBA
:109C900000F00105F9B904F01DFC0DB1226800E0E7
:109CA0000022C7484178C06807F06DFDC4481030F5
:109CB000C0788DF8000010B1012802D004E0012026
:109CC00000E000208DF80000684608F0FFF8BA4870
:109CD000243808F0B5FE002D02D02068283020601E
:109CE00038BD30B5B54D04466878A04200D8FFDFD6
:109CF000686800EB041030BD70B5B04800252C46F4
:109D0000467807E02046FFF7ECFF4078641C2844C3
:109D1000C5B2E4B2B442F5D1284630E72DE9F041AE
:109D20000C4607464FF0000800F01FF90646FF28D2
:109D300001D94FF013083868C01C20F003023A60C4
:109D400054EA080421D19D48F3B2072128300DF0D0
:109D5000DBFD09E0072C10D2DFE804F00604080858
:109D60000A040600974804E0974802E0974800E09C
:109D700097480DF0E9FD054600E0FFDFA54200D061
:109D8000FFDF641CE4B2072CE4D3386800EB061054
:109D9000386040467BE5021D5143452900D24521EC
:109DA0000844C01CB0FBF2F0C0B270472DE9FC5F64
:109DB000064682484FF000088B464746444690F8D6
:109DC000019022E02046FFF78CFF050000D1FFDF65
:109DD000687869463844C7B22846FEF7A3FF824632
:109DE00001A92846FEF7B8FF0346BDF80400524615
:109DF000001D81B2BDF80000001D80B20AF0D4F849
:109E00006A78641C00FB0288E4B24C45DAD1306801
:109E1000C01C20F003003060BBF1000F00D0002018
:109E2000424639460AF0CEF8316808443060BDE851
:109E3000FC9F6249443108710020C87070475F4937
:109E40004431CA782AB10A7801EB421108318142C3
:109E500001D001207047002070472DE9F0410646EF
:109E60000078154600F00F0400201080601E0F4699
:109E7000052800D3FFDF50482A46183800EB84003D
:109E8000394650F8043C3046BDE8F04118472DE90A
:109E9000F0414A4E0C46402806D0412823D04228A3
:109EA0002BD0432806D123E0A07861780D18E17803
:109EB000814201D90720EAE42078012801D9132042
:109EC000E5E4FF2D08D80BF009FF07460DF046F931
:109ED000381A801EA84201DA1220D8E42068B06047
:109EE000207930730DE0BDE8F041084600F078B805
:109EF00008780228DED8307703E008780228D9D81D
:109F000070770020C3E4F8B500242C4DA02805D0BC
:109F1000A12815D0A22806D00720F8BD087800F0A7
:109F20000100E8771FE00E4669463046FDF73DFD2B
:109F30000028F2D130882884B07885F8220012E019
:109F400008680921F82801D3820701D00846F8BD26
:109F50006A7C02F00302012A04D16A8BD73293B2E1
:109F60008342F3D868622046F8BD2DE9F047DFF858
:109F70004C900026344699F8090099F80A2099F87F
:109F800001700244D5B299F80B20104400F0FF088C
:109F900008E02046FFF7A5FE817B407811FB0066B4
:109FA000641CE4B2BC42F4D199F8091099F80A0093
:109FB0002944294441440DE054610200B0030020CB
:109FC0001C0000206741000045B30000DD2F0000A9
:109FD000FB56010000B1012008443044BDE8F08781
:109FE00038B50446407800F00300012803D0022869
:109FF0000BD0072038BD606858B1F7F777F9D0B9B2
:10A000006068F7F76AF920B915E06068F7F721F999
:10A0100088B969462046FCF729F80028EAD160781B
:10A0200000F00300022808D19DF8000028B1606804
:10A03000F7F753F908B1102038BD6189F8290DD818
:10A04000208988420AD8607800F003020A48012A71
:10A0500006D1D731426A89B28A4201D2092038BD7D
:10A0600094E80E0000F1100585E80E000AB9002101
:10A070000183002038BD0000B00300202DE9F0412D
:10A08000074614468846084601F08AFD064608EB56
:10A0900088001C22796802EBC0000D18688C58B14A
:10A0A0004146384601F08BFD014678680078C200D1
:10A0B000082305F120000CE0E88CA8B141463846A1
:10A0C00001F084FD0146786808234078C20005F15C
:10A0D000240009F0A8FD38B1062121726681D0E97B
:10A0E0000010C4E9031009E0287809280BD00520E6
:10A0F000207266816868E060002028702046BDE814
:10A10000F04101F02EBD072020726681F4E72DE9B1
:10A11000F04116460D460746406801EB85011C22BA
:10A1200002EBC1014418204601F072FD40B100214C
:10A13000708865F30F2160F31F4106200DF0BEFC0F
:10A1400009202070324629463846BDE8F04195E79F
:10A150002DE9F0410E46074600241C21F07816E058
:10A1600004EB8403726801EBC303D25C6AB1FFF7AE
:10A170003DFA050000D1FFDF6F802A4621463046B8
:10A18000FFF7C5FF0120BDE8F081641CE4B2A042E6
:10A19000E6D80020F7E770B5064600241C21C078F9
:10A1A0000AE000BF04EB8403726801EBC303D51817
:10A1B0002A782AB1641CE4B2A042F3D8402070BDD2
:10A1C00028220021284604F062F9706880892881DD
:10A1D000204670BD70B5034600201C25DC780CE0DD
:10A1E00000EB80065A6805EBC6063244167816B1B5
:10A1F000128A8A4204D0401CC0B28442F0D8402067
:10A2000070BDF0B5044600201C26E5780EE000BFC6
:10A2100000EB8007636806EBC7073B441F788F425B
:10A2200002D15B78934204D0401CC0B28542EFD883
:10A230004020F0BD0078032801D0002070470120A5
:10A2400070470078022801D0002070470120704735
:10A250000078072801D000207047012070472DE9C1
:10A26000F041064688461078F1781546884200D3BA
:10A27000FFDF2C781C27641CF078E4B2A04201D8E0
:10A28000201AC4B204EB8401706807EBC1010844D2
:10A29000017821B14146884708B12C7073E72878CE
:10A2A000A042E8D1402028706DE770B514460B88B5
:10A2B0000122A240134207D113430B8001230A223B
:10A2C000011D09F07AFC047070BD2DE9FF4F81B0CB
:10A2D0000878DDE90E7B9A4691460E4640072CD45D
:10A2E000019809F026FF040000D1FFDF07F1040800
:10A2F00020461FFA88F109F065F8050000D1FFDF5C
:10A30000204629466A4609F0B0FA0098A0F8037082
:10A31000A0F805A0284609F056FB017869F306016C
:10A320006BF3C711017020461FFA88F109F08DF810
:10A3300000B9FFDF019807F094F906EB0900017FEF
:10A34000491C017705B0BDE8F08F2DE9F84F0E46A6
:10A350009A4691460746032109F0A8FD0446008D60
:10A36000DFF8B885002518B198F80000B0421ED17A
:10A37000384609F0DEFE070000D1FFDF09F10401D5
:10A38000384689B209F01EF8050010D03846294633
:10A390006A4609F06AFA009800210A460180817035
:10A3A00007F01CFA0098C01DCAF8000021E098F8D8
:10A3B0000000B04216D104F1260734F8341F012002
:10A3C00000FA06F911EA090F00D0FFDF2088012307
:10A3D00040EA090020800A22391D384609F008FCAD
:10A3E000067006E0324604F1340104F12600FFF75E
:10A3F0005CFF0A2188F800102846BDE8F88FFEB5FA
:10A4000015460C46064602AB0C220621FFF79DFFBF
:10A41000002827D00299607812220A70801C4870A8
:10A4200008224A80A07002982988052381806988C3
:10A43000C180A9880181E988418100250C20CDE9EE
:10A440000005062221463046FFF73FFF294600223D
:10A4500066F31F41F02310460DF086FA6078801CE9
:10A4600060700120FEBDFEB514460D46062206466C
:10A4700002AB1146FFF769FF002812D0029B1320A0
:10A4800000211870A8785870022058809C800620FF
:10A49000CDE900010246052329463046FFF715FFA6
:10A4A0000120FEBD2DE9FE430C46804644E002AB90
:10A4B0000E2207214046FFF748FF002841D0606880
:10A4C0001C2267788678BF1C06EB860102EBC1016F
:10A4D000451802981421017047700A214180698A49
:10A4E0000181E98A4181A9888180A98981813046D9
:10A4F00001F056FB029905230722C8806F700420E3
:10A50000287000250E20CDE9000521464046FFF7C2
:10A51000DCFE294666F30F2168F31F41F023002279
:10A5200006200DF021FA6078FD49801C6070626899
:10A530002046921CFFF793FE606880784028B6D1D1
:10A540000120BDE8FE83FEB50D46064638E002ABAD
:10A550000E2207213046FFF7F8FE002835D0686844
:10A560001C23C17801EB810203EBC202841802981C
:10A5700015220270627842700A224280A2894281CA
:10A58000A2888281084601F00BFB01460298818077
:10A59000618AC180E18A0181A088B8B10020207061
:10A5A00000210E20CDE9000105230722294630466F
:10A5B000FFF78BFE6A68DB492846D21CFFF74FFE87
:10A5C0006868C0784028C2D10120FEBD0620E6E7B9
:10A5D0002DE9FE430C46814644E0204601F002FB93
:10A5E000D0B302AB082207214846FFF7AEFE002891
:10A5F000A7D060681C2265780679AD1C06EB860141
:10A6000002EBC10147180298B7F8108006210170CB
:10A61000457004214180304601F0C2FA014602989B
:10A6200005230722C180A0F804807D7008203870BF
:10A630000025CDE9000521464846FFF746FE29469C
:10A6400066F30F2169F31F41F023002206200DF06D
:10A650008BF96078801C60706268B3492046121DD7
:10A66000FFF7FDFD606801794029B6D1012068E758
:10A670002DE9F34F83B00D4691E0284601F0B2FA80
:10A6800000287DD068681C2290F806A00AEB8A0199
:10A6900002EBC10144185146284601F097FAA1780F
:10A6A000CB0069684978CA00014604F1240009F02A
:10A6B000D6FA07468188E08B4FF00009091A8EB25E
:10A6C00008B1C84607E04FF00108504601F053FAC0
:10A6D00008B9B61CB6B2208BB04200D80646B346C5
:10A6E00002AB324607210398FFF72FFE060007D082
:10A6F000B8F1000F0BD0504601F03DFA10B106E062
:10A7000000201FE60299B8884FF0020908800196E0
:10A71000E28B3968ABEB09001FFA80F80A44039812
:10A720004E46009209F005FDDDE90021F61D434685
:10A73000009609F014F9E08B404480B2E083B988B8
:10A74000884201D1012600E00026CDE900B6238A27
:10A75000072229460398FFF7B8FD504601F00BFA8F
:10A7600010B9E089401EE08156B1A078401CA0706D
:10A770006868E978427811FB02F1CAB2012300E06F
:10A7800007E081690E3009F018FA80F800A0002077
:10A79000E0836A6865492846921DFFF760FD686896
:10A7A000817940297FF469AF0120CBE570B5064679
:10A7B00048680D4614468179402910D104EB840184
:10A7C0001C2202EBC101084401F043FA002806D024
:10A7D0006868294684713046BDE8704048E770BD1E
:10A7E000FEB50C460746002645E0204601F0FAF982
:10A7F000D8B360681C22417901EB810102EBC101F1
:10A800004518688900B9FFDF02AB082207213846E6
:10A81000FFF79BFD002833D00299607816220A705A
:10A82000801C4870042048806068407901F0B8F9C5
:10A83000014602980523072281806989C18008208A
:10A84000CDE9000621463846FFF73FFD6078801CC1
:10A850006070A88969890844B0F5803F00D3FFDFA4
:10A86000A88969890844A8816E81626830492046B8
:10A87000521DFFF7F4FC606841794029B5D10120F1
:10A88000FEBD30B5438C458BC3F3C704002345B1EF
:10A89000838B641EED1AC38A6D1E1D4495FBF3F372
:10A8A000E4B22CB1008918B1A04200D8204603447C
:10A8B0004FF6FF70834200D3034613800C7030BD07
:10A8C0002DE9FC41074616460D46486802EB860115
:10A8D0001C2202EBC10144186A4601A92046FFF779
:10A8E000D0FFA089618901448AB2BDF8001091426D
:10A8F00012D0081A00D5002060816868407940288D
:10A900000AD1204601F09BF9002805D06868294645
:10A9100046713846FFF764FFBDE8FC813000002037
:10A9200035A2000043A2000051A2000053BC000069
:10A930003FBC00002DE9FE4F0F468146154650886A
:10A94000032109F0B3FA0190B9F8020001F01BF9F4
:10A9500082460146019801F045F9002824D001986B
:10A960001C2241680AEB8A0002EBC0000C1820464A
:10A9700001F04EF9002817D1B9F80000E18A8842A9
:10A980000ED8A18961B1B8420ED100265146019876
:10A9900001F015F9218C01EB0008608B30B114E057
:10A9A000504601F0E8F8A0B3BDE8FE8F504601F034
:10A9B000E2F808B1678308E0022FF5D3B9F8040084
:10A9C0006083618A884224D80226B81B87B2B8F80F
:10A9D0000400A28B801A002814DD874200DA384672
:10A9E0001FFA80FB688869680291D8F800100A4451
:10A9F000009209F08CFBF61D009A5B4602990096C6
:10AA000008F079FFA08B384480B2A083618B884224
:10AA100007D96888019903B05246BDE8F04F01F0AC
:10AA200035B91FD14FF009002872B9F802006881CA
:10AA3000D8E90010C5E90410608BA881284601F010
:10AA400090F85146019801F0BAF8014601980823A0
:10AA500040680078C20004F1200009F0E4F800200A
:10AA6000A0836083504601F086F810B9A089401E8B
:10AA7000A0816888019903B00AF0FF02BDE8F04F99
:10AA80001EE72DE9F041064615460F461C461846BE
:10AA9000F6F7DFFB18B92068F6F701FC10B11020BB
:10AAA000BDE8F0817168688C0978B0EBC10F01D303
:10AAB0001320F5E73946304601F081F80146706809
:10AAC00008230078C20005F1200009F076F8D4E9E7
:10AAD0000012C0E900120020E2E710B5044603218D
:10AAE00009F0E4F90146007800F00300022805D0DF
:10AAF0002046BDE8104001F1140280E48A8A204615
:10AB0000BDE81040AFE470B50446032109F0CEF96A
:10AB1000054601462046FFF75BFD002816D0294672
:10AB20002046FFF75DFE002810D029462046FFF79B
:10AB30000AFD00280AD029462046FFF7B3FC00286A
:10AB400004D029462046BDE8704091E570BD2DE94E
:10AB5000F0410C4680461EE0E178427811FB02F19C
:10AB6000CAB2816901230E3009F05DF80778606888
:10AB70001C22C179491EC17107EB8701606802EB95
:10AB8000C10146183946204601F02CF818B130466C
:10AB900001F037F820B16068C1790029DCD17FE786
:10ABA000FEF724FD050000D1FFDF0A202872384699
:10ABB00000F0F6FF68813946204601F007F80146AB
:10ABC000606808234078C20006F1240009F02BF8E1
:10ABD000D0E90010C5E90310A5F80280284600F06E
:10ABE000C0FFB07800B9FFDFB078401EB07057E703
:10ABF00070B50C460546032109F058F90146406836
:10AC0000C2792244C2712846BDE870409FE72DE911
:10AC1000FE4F8246507814460F464FF00008002839
:10AC20004FD0012807D0022822D0FFDF2068B8606B
:10AC30006068F860B8E602AB0E2208215046FFF7C4
:10AC400084FB0028F2D00298152105230170217899
:10AC500041700A214180C0F80480C0F80880A0F843
:10AC60000C80628882810E20CDE90008082221E054
:10AC7000A678304600F094FF054606EB86012C22AC
:10AC8000786802EBC1010822465A02AB11465046D1
:10AC9000FFF75BFB0028C9D00298072101702178DB
:10ACA00041700421418008218580C680CDE90018CB
:10ACB00005230A4639465046FFF707FB87F8088008
:10ACC00072E6A678022516B1022E13D0FFDF2A1DE8
:10ACD000914602AB08215046FFF737FB0028A5D06C
:10ACE00002980121022E01702178417045808680F2
:10ACF00002D005E00625EAE7A188C180E18801814C
:10AD0000CDE900980523082239465046D4E710B50E
:10AD10000446032109F0CAF8014600F10802204662
:10AD2000BDE8104073E72DE9F04F0F4605468DB0A2
:10AD300014465088032109F0B9F84FF000088DF847
:10AD400014800646ADF81680042F7BD36A78002A5B
:10AD500078D028784FF6FF794FF01C0A132834D0AA
:10AD600008DC012871D006284AD007286ED01228A6
:10AD70000ED106E014286AD0152869D0162807D10C
:10AD8000AAE10C2F04D1307800F00301022907D08A
:10AD9000CDF80880CDF80C8068788DF808004CE07C
:10ADA00040F0080030706878B07001208DF8140011
:10ADB000A888ADF81800E888ADF81A002889ADF821
:10ADC0001C006889ADF81E0011E1B078904239D1BD
:10ADD0003078010736D5062F34D120F008003070C6
:10ADE0006088414660F31F4100200CF067FE02209E
:10ADF0008DF81400ADF81890A888ADF81A00F6E0A8
:10AE0000082F1FD1A888EF88814600F0BCFE80463D
:10AE10000146304600F0E6FE18B1404600F0ABFEB9
:10AE2000B8B1FC48D0E90010CDE902106878ADF85F
:10AE30000C908DF80800ADF80E70608802AA3146BB
:10AE4000FFF7E5FE0DB0BDE8F08FB6E01EE041E093
:10AE5000ECE0716808EB88002C2202EBC000085A75
:10AE6000B842EFD1EB4802AAD0E90210CDE90210B6
:10AE700068788DF8080008F0FF058DF80A506088A2
:10AE80003146FFF7C4FE224629461FE0082FD9D1DC
:10AE9000B5F80480E88800F076FE074601463046A3
:10AEA00000F0A0FE0028CDD007EB870271680AEB06
:10AEB000C2000844028A4245C4D101780829C1D1A0
:10AEC000407869788842BDD1F9B222463046FFF712
:10AED0001EF9B7E70E2F7FF45BAFE9886F898B46C9
:10AEE000B5F808903046FFF775F9ABF140014029FD
:10AEF00001D309204AE0B9F1170F01D3172F01D26E
:10AF00000B2043E040280ED000EB800271680AEB72
:10AF1000C20008440178012903D140786978884249
:10AF200090D00A2032E03046FFF735F9014640283C
:10AF30002BD001EB810372680AEBC30002EB00081F
:10AF4000012288F800206A7888F801207068AA88B1
:10AF50004089B84200D93846AD8903232372A282C2
:10AF6000E7812082A4F80C906582084600F018FE64
:10AF70006081A8F81490A8F81870A8F80E50A8F8E6
:10AF800010B0204600F0EDFD5CE7042005212172A1
:10AF9000A4F80A80E081012121739E49D1E90421AE
:10AFA000CDE9022169788DF80810ADF80A006088B3
:10AFB00002AA3146FFF72BFEE3E7062F89D3B078CC
:10AFC00090421AD13078010717D520F00800307070
:10AFD0006088414660F31F4100200CF06FFD0220A5
:10AFE0008DF81400A888ADF81800ADF81A906088A4
:10AFF000224605A9F9F7E3F824E704213046FFF7D4
:10B0000000F905464028BFD0022083030090224665
:10B010002946304600F003FE4146608865F30F2163
:10B0200060F31F4106200CF049FD0BE70E2FABD15A
:10B0300004213046FFF7E5F881464028A4D0414678
:10B04000608869F30F2160F31F4106200CF036FD84
:10B05000A8890B906889099070682F894089B84247
:10B0600000D938468346B5F80680A8880A90484635
:10B0700000F096FD60810B9818B1022000900B9BA8
:10B0800024E0B8F1170F1ED3172F1CD30420207211
:10B0900009986082E781A4F810B0A4F80C8009EB4D
:10B0A000890271680AEBC2000D18DDE90913A5F8E1
:10B0B0001480A5F818B0E9812B82204600F051FDDC
:10B0C00006202870BEE601200B2300902246494648
:10B0D000304600F0A4FDB5E6082F8DD1A988304692
:10B0E000FFF778F80746402886D000F044FD002896
:10B0F0009BD107EB870271680AEBC20008448046C7
:10B1000000F086FD002890D1ED88B8F80E002844A4
:10B11000B0F5803F05D360883A46314600F0B6FD71
:10B1200090E6002DCED0A8F80E0060883A46314651
:10B13000FFF73CFB08202072384600F031FD6081AB
:10B14000A5811EE72DE9F05F0C4601281FD09579F7
:10B1500092F8048092F8056005EB85011F2202EB4E
:10B16000C10121F0030B08EB060111FB05F14FF6BD
:10B17000FF7202EAC10909F1030115FB0611264F0E
:10B1800021F0031ABB6840B101283ED125E0616877
:10B19000E57891F800804E78DEE75946184608F0C9
:10B1A000C0FC606000B9FFDF5A460021606803F010
:10B1B0006EF9E5705146B86808F0B3FC6168486103
:10B1C00000B9FFDF6068426902EB090181616068D4
:10B1D00080F800806068467017E0606852464169F8
:10B1E000184608F0C9FC5A466168B86808F0C4FC03
:10B1F000032008F003FE0446032008F007FE201A8F
:10B20000012802D1B86808F081FC0BEB0A00BDE808
:10B21000F09F000060610200300000200246002123
:10B2200002208FE7F7B5FF4C0A20164620700098E1
:10B2300060B100254FEA0D0008F055FC0021A17017
:10B240006670002D01D10099A160FEBD012500208E
:10B25000F2E770B50C46154638220021204603F06F
:10B2600016F9012666700A22002104F11C0003F081
:10B270000EF905B9FFDF297A207861F3010020700B
:10B28000A87900282DD02A4621460020FFF75AFF32
:10B2900061684020E34A88706168C870616808711D
:10B2A000616848716168887161682888088161688F
:10B2B00068884881606886819078002811D061682C
:10B2C0000620087761682888C885616828884886CC
:10B2D00060680685606869889288018681864685EF
:10B2E000828570BDC878002802D00022012029E79D
:10B2F000704770B50546002165F31F4100200CF032
:10B30000DDFB0321284608F0D1FD040000D1FFDF5A
:10B3100021462846FEF71CFF002804D0207840F084
:10B3200010002070012070BD70B505460C4603204A
:10B3300008F056FD08B1002070BDBA4885708480C1
:10B34000012070BD2DE9FF4180460E460F0CFEF72F
:10B350004DF9050007D06F800321384608F0A6FD9F
:10B36000040008D106E004B03846BDE8F0411321DE
:10B37000F9F750BBFFDF5FEA080005D0B8F1060F10
:10B3800018D0FFDFBDE8FF8120782A4620F00800B2
:10B3900020700020ADF8020002208DF800004FF66A
:10B3A000FF70ADF80400ADF8060069463846F8F7BE
:10B3B00006FFE7E7C6F3072101EB81021C23606863
:10B3C00003EBC202805C042803D008280AD0FFDF08
:10B3D000D8E7012000904FF440432A46204600F071
:10B3E0001EFCCFE704B02A462046BDE8F041FEF738
:10B3F0008EBE2DE9F05F05464089002790460C4639
:10B400003E46824600F0BFFB8146287AC01E0828CF
:10B410006BD2DFE800F00D04192058363C47722744
:10B420001026002C6CD0D5E90301C4E902015CE0D0
:10B4300070271226002C63D00A2205F10C0104F1BA
:10B44000080002F0FAFF50E071270C26002C57D0BC
:10B45000E868A06049E0742710269CB3D5E9030191
:10B46000C4E902016888032108F020FD8346FEF745
:10B47000BDF802466888508049465846FEF7FEFDF2
:10B4800033E075270A26ECB1A88920812DE07627C4
:10B490001426BCB105F10C0004F1080307C883E8C9
:10B4A000070022E07727102664B1D5E90301C4E93B
:10B4B00002016888032108F0F9FC01466888FFF75B
:10B4C00046FB12E01CE073270826CCB168880321F4
:10B4D00008F0ECFC01460078C00606D56888FEF747
:10B4E00037FE10B96888F8F777FAA8F800602CB131
:10B4F0002780A4F806A066806888A080002086E6E1
:10B50000A8F80060FAE72DE9FC410C461E461746F4
:10B510008046032108F0CAFC05460A2C0AD2DFE85F
:10B5200004F005050505050509090907042303E0DD
:10B53000062301E0FFDF0023CDE9007622462946FD
:10B540004046FEF7C2FEBDE8FC81F8B50546A0F511
:10B550007F40FF382BD0284608F0D9FD040000D1E9
:10B56000FFDF204608F05FF9002821D001466A4637
:10B57000204608F07AF900980321B0F805602846C3
:10B5800008F094FC0446052E13D0304600F0FBFA78
:10B5900005460146204600F025FB40B1606805EBFA
:10B5A00085013E2202EBC101405A002800D0012053
:10B5B000F8BD007A0028FAD00020F8BDF8B504469E
:10B5C000408808F0A4FD050000D1FFDF6A46284648
:10B5D000616800F0C4FA01460098091F8BB230F888
:10B5E000032F0280428842800188994205D1042AB3
:10B5F00008D0052A20D0062A16D022461946FFF781
:10B6000099F9F8BD001D0E46054601462246304612
:10B61000F6F739FF0828F4D1224629463046FCF7D0
:10B6200064F9F8BD30000020636864880A46011D93
:10B630002046FAF789F9F4E72246001DFFF773FB6D
:10B64000EFE770B50D460646032108F02FFC040015
:10B6500004D02078000704D5112070BD43F2020009
:10B6600070BD2A4621463046FEF7C9FE18B9286843
:10B6700060616868A061207840F0080020700020B8
:10B6800070BD70B50D460646032108F00FFC04009E
:10B6900004D02078000704D4082070BD43F20200D3
:10B6A00070BD2A4621463046FEF7DDFE00B9A58270
:10B6B000207820F008002070002070BD2DE9F04FA8
:10B6C0000E4691B08046032108F0F0FB0446404648
:10B6D00008F02FFD07460020079008900990ADF86C
:10B6E00030000A9002900390049004B9FFDF0DF13E
:10B6F0000809FFB9FFDF1DE038460BA9002207F05B
:10B7000055FF9DF82C0000F07F050A2D00D3FFDFC8
:10B710006019017F491E01779DF82C00000609D5AC
:10B720002A460CA907A8FEF7C0FD19F80510491C08
:10B7300009F80510761EF6B2DED204F13400F84D99
:10B7400004F1260BDFF8DCA304F12A07069010E0D1
:10B750005846069900F08CFA064628700A2800D34D
:10B76000FFDF5AF8261040468847E08CC05DB042A3
:10B7700002D0208D0028EBD10A202870E94D4E46DA
:10B7800028350EE00CA907A800F072FA0446375DD0
:10B7900055F8240000B9FFDF55F82420394640460B
:10B7A0009047BDF81E000028ECD111B0BDE8F08F25
:10B7B00010B5032108F07AFB040000D1FFDF0A2254
:10B7C000002104F11C0002F062FE207840F0040029
:10B7D000207010BD10B50C46032108F067FB204413
:10B7E000007F002800D0012010BD2DE9F84F8946C8
:10B7F00015468246032108F059FB070004D028466D
:10B80000F5F727FD40B903E043F20200BDE8F88FE9
:10B810004846F5F744FD08B11020F7E7786828B1ED
:10B8200069880089814201D90920EFE7B9F8000051
:10B830001C2488B100F0A7F980460146384600F084
:10B84000D1F988B108EB8800796804EBC000085C86
:10B8500001280BD00820D9E73846FEF79CFC80462B
:10B86000402807D11320D1E70520CFE7FDF7BEFE22
:10B8700006000BD008EB8800796804EBC0000C18B8
:10B88000B9F8000020B1E88910B113E01120BDE73C
:10B890002888172802D36888172801D20720B5E71F
:10B8A000686838B12B1D224641463846FFF7E9F853
:10B8B0000028ABD104F10C0269462046FEF7E1FFF7
:10B8C000288860826888E082B9F8000030B10220E0
:10B8D0002070E889A080E889A0B12BE003202070C7
:10B8E000A889A08078688178402905D180F80280F5
:10B8F00039465046FEF7D6FD404600F051F9A9F80A
:10B90000000021E07868218B4089884200D90846F0
:10B910002083A6F802A004203072B9F800007081DC
:10B92000E0897082F181208B3082A08AB08130461C
:10B9300000F017F97868C178402905D180F80380B4
:10B9400039465046FEF7FFFD00205FE770B50D4613
:10B950000646032108F0AAFA04000ED0284600F09B
:10B9600012F905460146204600F03CF918B1284678
:10B9700000F001F920B1052070BD43F2020070BD56
:10B9800005EB85011C22606802EBC101084400F050
:10B990003FF908B1082070BD2A462146304600F024
:10B9A00075F9002070BD2DE9F0410C461746804620
:10B9B000032108F07BFA0546204600F0E4F804462F
:10B9C00095B10146284600F00DF980B104EB8401E1
:10B9D0001C22686802EBC1014618304600F018F9D5
:10B9E00038B10820BDE8F08143F20200FAE70520F3
:10B9F000F8E73B46324621462846FFF742F8002842
:10BA0000F0D1E2B229464046FEF75AFF708C083862
:10BA1000082803D242484078F7F776FA0020E1E799
:10BA20002DE9F0410D4617468046032108F03EFA05
:10BA30000446284600F0A7F8064624B13846F5F734
:10BA400008FC38B902E043F20200CBE73868F5F7AA
:10BA500000FC08B11020C5E73146204600F0C2F8CE
:10BA600060B106EB86011C22606802EBC10145183B
:10BA7000284600F0CDF818B10820B3E70520B1E75B
:10BA8000B888A98A884201D90C20ABE76168E88CA4
:10BA90004978B0EBC10F01D31320A3E7314620460C
:10BAA00000F094F80146606808234078C20005F170
:10BAB000240008F082F8D7E90012C0E90012F2B2BF
:10BAC00021464046FEF772FE00208BE72DE9F04745
:10BAD0000D461F4690468146032108F0E7F90446CB
:10BAE000284600F050F806463CB14DB13846F5F70F
:10BAF000F4FB50B11020BDE8F08743F20200FAE7F2
:10BB0000606858B1A0F80C8027E03146204600F06C
:10BB100069F818B1304600F02EF828B10520EAE7A0
:10BB2000300000207861020006EB86011C2260686C
:10BB300002EBC1014518284600F06AF808B1082058
:10BB4000D9E7A5F80880F2B221464846FEF7B8FECC
:10BB50001FB1A8896989084438800020CBE707F025
:10BB600084BE017821F00F01491C21F0F001103151
:10BB70000170FDF73EBD20B94E48807808B1012024
:10BB80007047002070474B498988884201D10020C6
:10BB90007047402801D2402000E0403880B2704712
:10BBA00010B50446402800D9FFDF2046FFF7E3FF29
:10BBB00010B14048808810BD4034A0B210BD40682C
:10BBC00042690078484302EBC0007047C278406881
:10BBD000037812FB03F24378406901FB032100EB79
:10BBE000C1007047C2788A4209D9406801EB8101DF
:10BBF0001C2202EBC101405C08B10120704700200B
:10BC000070470078062801D901207047002070474E
:10BC10000078062801D00120704700207047F0B45A
:10BC200001EB81061C27446807EBC6063444049DDB
:10BC300005262670E3802571F0BCFEF71FBA10B50B
:10BC4000418911B1FFF7DDFF08B1002010BD0120CF
:10BC500010BD10B5C18C8278B1EBC20F04D9C18977
:10BC600011B1FFF7CEFF08B1002010BD012010BDBB
:10BC700010B50C4601230A22011D07F0D4FF0078FD
:10BC80002188012282409143218010BDF0B402EB53
:10BC900082051C264C6806EBC505072363554B68D7
:10BCA0001C79402C03D11A71F0BCFEF791BCF0BC9A
:10BCB000704700003000002010B5EFF3108000F056
:10BCC000010472B6FC484178491C41704078012853
:10BCD00001D10BF0B3FA002C00D162B610BD70B5E3
:10BCE000F54CA07848B90125A570FFF7E5FF0BF0EA
:10BCF000B6FA20B100200BF080FA002070BD4FF0A2
:10BD00008040E570C0F80453F7E770B5EFF310809A
:10BD100000F0010572B6E84C607800B9FFDF60788A
:10BD2000401E6070607808B90BF08CFA002D00D1CD
:10BD300062B670BDE04810B5817821B10021C170B4
:10BD40008170FFF7E2FF002010BD10B504460BF034
:10BD500086FAD9498978084000D001202060002067
:10BD600010BD10B5FFF7A8FF0BF079FA02220123EE
:10BD7000D149540728B1D1480260236103200872D9
:10BD800002E00A72C4F804330020887110BD2DE966
:10BD9000F84FDFF824934278817889F80420002650
:10BDA00089F80510074689F806600078DFF810B3B7
:10BDB000354620B1012811D0022811D0FFDF0BF049
:10BDC00060FA4FF0804498B10BF062FAB0420FD1A4
:10BDD00030460BF061FA0028FAD042E00126EEE787
:10BDE000FFF76AFF58460168C907FCD00226E6E75C
:10BDF0000120E060C4F80451B2490E600107D1F897
:10BE00004412B04AC1F3423124321160AD49343199
:10BE100008604FF0020AC4F804A3A060AA480168B1
:10BE2000C94341F3001101F10108016841F010011B
:10BE3000016001E019F0A8FFD4F804010028F9D04E
:10BE400030460BF029FA0028FAD0B8F1000F04D1DF
:10BE50009D48016821F010010160C4F808A3C4F8EE
:10BE6000045199F805004E4680B1387870B90BF04E
:10BE7000F6F980460BF006FC6FF00042B8F1000FB7
:10BE800002D0C6E9032001E0C6E90302DBF80000A6
:10BE9000C00701D00BF0DFF9387810B13572BDE87A
:10BEA000F88F4FF01808C4F808830127A7614FF4F2
:10BEB0002070ADF8000000BFBDF80000411EADF8D5
:10BEC0000010F9D2C4F80C51C4F810517A48C01DC2
:10BED0000BF06CFA3570FFF744FF676179493079F0
:10BEE00020310860C4F80483D9E770B5050000D19B
:10BEF000FFDF4FF080424FF0FF30C2F8080300210F
:10BF0000C2F80011C2F80411C2F80C11C2F81011E5
:10BF1000694C61700BF0AFF910B10120A070607036
:10BF200067480068C00701D00BF095F92846BDE8C6
:10BF300070402CE76048007A002800D0012070474C
:10BF40002DE9F04F61484FF0000A85B0D0F800B0FD
:10BF5000D14657465D4A5E49083211608406D4F8DE
:10BF6000080110B14FF0010801E04FF000080BF09C
:10BF7000F0F978B1D4F8240100B101208246D4F858
:10BF80001C0100B101208146D4F8200108B101272D
:10BF900000E00027D4F8000100B101200490D4F89B
:10BFA000040100B101200390D4F80C0100B101207C
:10BFB0000290D4F8100100B101203F4D0190287883
:10BFC00000260090B8F1000F04D0C4F808610120E9
:10BFD0000BF013F9BAF1000F04D0C4F82461092062
:10BFE0000BF00BF9B9F1000F04D0C4F81C610A2062
:10BFF0000BF003F927B1C4F820610B200BF0FDF81A
:10C000002D48C01D0BF0DAF900B1FFDFDFF8AC807E
:10C010000498012780B1C4F80873E87818B1EE706D
:10C0200000200BF0EAF8287A022805D103202872B4
:10C030000221C8F800102761039808B1C4F8046110
:10C04000029850B1C4F80C61287A032800D0FFDFB1
:10C05000C8F800602F72FFF758FE019838B1C4F895
:10C060001061287A012801D100F05CF8676100981E
:10C0700038B12E70287A012801D1FFF772FEFFF740
:10C0800044FE0D48C01D0BF0AFF91049091DC1F861
:10C0900000B005B0BDE8F08F074810B5C01D0BF02B
:10C0A0008DF90549B0B1012008704FF0E021C1F8C9
:10C0B0000002BDE81040FFE544000020340C0040C1
:10C0C0000C0400401805004010ED00E0100502408F
:10C0D00001000001087A012801D1FFF742FEBDE806
:10C0E000104024480BF080B970B5224CE41FA078B2
:10C0F00008B90BF0A7F801208507A861207A00266F
:10C10000032809D1D5F80C0120B900200BF0C4F8A0
:10C110000028F7D1C5F80C6126724FF0FF30C5F842
:10C12000080370BD70B5134CE41F6079F0B10128AD
:10C1300003D0A179401E814218DA0BF090F8054631
:10C140000BF0A0FA6179012902D9A179491CA171EA
:10C150000DB1216900E0E168411A022902DA11F10A
:10C16000020F06DC0DB1206100E0E060BDE8704028
:10C17000F7E570BD4B0000200F4A12680D498A4256
:10C180000CD118470C4A12680A4B9A4206D101B5E5
:10C190000BF04AFA0BF01DFDBDE8014007490968A4
:10C1A0000958084706480749054A064B70470000EA
:10C1B00000000000BEBAFECA5C000020040000209F
:10C1C000C8130020C8130020F8B51D46DDE9064756
:10C1D0000E000AD007F0ADFF2346FF1DBCB231466A
:10C1E0002A46009407F0BBFBF8BDD0192246194639
:10C1F00002F023F92046F8BD70B50D460446102222
:10C20000002102F044F9258117206081A07B40F0D5
:10C210000A00A07370BD4FF6FF720A80014602202B
:10C220000BF04CBC704700897047827BD30701D16B
:10C23000920703D48089088000207047052070474A
:10C24000827B920700D581817047014600200988D2
:10C2500041F6FE52114200D00120704700B503465E
:10C26000807BC00701D0052000BD59811846FFF72B
:10C27000ECFFC00703D0987B40F004009873987BD4
:10C2800040F001009873002000BD827B520700D56A
:10C2900009B14089704717207047827B61F3C30260
:10C2A000827370472DE9FC5F0E460446017896467E
:10C2B000012000FA01F14DF6FF5201EA020962681D
:10C2C0004FF6FF7B1188594502D10920BDE8FC9F3C
:10C2D000B9F1000F05D041F6FE55294201D00120E9
:10C2E000F4E741EA090111801D0014D000232B70EE
:10C2F00094F800C0052103221F464FF0020ABCF14A
:10C300000E0F76D2DFE80CF0F909252F47646B7722
:10C31000479193B4D1D80420D8E7616820898B7BFA
:10C320009B0767D517284AD30B89834247D389894E
:10C33000172901D3814242D185F800A0A5F8010058
:10C340003280616888816068817B21F0020181739D
:10C35000C6E0042028702089A5F801006089A5F8AE
:10C3600003003180BCE0208A3188C01D1FFA80F8AC
:10C37000414524D3062028702089A5F80100608952
:10C38000A5F80300A089A5F805000721208ACDE9BA
:10C390000001636941E00CF0FF00082810D008207C
:10C3A00028702089A5F801006089A5F80300318074
:10C3B0006A1D694604F10C0009F025FB10B15EE02E
:10C3C0001020EDE730889DF800100844308087E0A9
:10C3D0000A2028702089A5F80100328044E00C2052
:10C3E00028702089A5F801006089A5F80300318034
:10C3F0003AE082E064E02189338800EB41021FFAD1
:10C4000082F843453BD3B8F1050F38D30E222A708A
:10C410000BEA4101CDE90010E36860882A467146C5
:10C42000FFF7D2FEA6F800805AE04020287060890D
:10C430003188C01C1FFA80F8414520D32878714606
:10C4400020F03F00123028702089A5F80100608993
:10C45000CDE9000260882A46E368FFF7B5FEA6F83A
:10C460000080287840063BD461682089888037E0C6
:10C47000A0893288401D1FFA80F8424501D2042766
:10C480003DE0162028702089A5F801006089A5F8F4
:10C490000300A089CDE9000160882A46714623691E
:10C4A000FFF792FEA6F80080DEE718202870207AB9
:10C4B0006870A6F800A013E061680A88920401D4AD
:10C4C00005271CE0C9882289914201D0062716E081
:10C4D0001E21297030806068018821F4005101809C
:10C4E000B9F1000F0BD061887823002202200BF0F5
:10C4F0003BFA61682078887006E033800327606823
:10C50000018821EA090101803846DFE62DE9FF4F65
:10C5100085B01746129C0D001E461CD03078C1070E
:10C5200003D000F03F00192801D9012100E00021CB
:10C530002046FFF7AAFEA8420DD32088A0F57F4130
:10C54000FF3908D03078410601D4000605D508200F
:10C5500009B0BDE8F08F0720FAE700208DF8000051
:10C560008DF8010030786B1E00F03F0C0121A81EF1
:10C570004FF0050A4FF002094FF0030B9AB2BCF1DD
:10C58000200F75D2DFE80CF08B10745E7468748C29
:10C59000749C74B574BA74C874D474E1747474F10E
:10C5A00074EF74EE74ED748B052D78D18DF80090D6
:10C5B000A0788DF804007088ADF8060030798DF809
:10C5C0000100707800F03F000C2829D00ADCA0F1AF
:10C5D0000200092863D2DFE800F0126215621A62D5
:10C5E0001D622000122824D004DC0E281BD0102845
:10C5F000DBD11BE016281FD01828D6D11FE02078E9
:10C60000800701E020784007002848DAEEE0207833
:10C610000007F9E72078C006F6E720788006F3E700
:10C6200020784006F0E720780006EDE72088C00576
:10C63000EAE720884005E7E720880005E4E720884E
:10C64000C004E1E72078800729D5032D27D18DF894
:10C6500000B0B6F8010081E0217849071FD5062D0A
:10C660001DD381B27078012803D0022817D102E0CF
:10C67000C9E0022000E0102004228DF8002072782A
:10C680008DF80420801CB1FBF0F2ADF8062092B2C8
:10C6900042438A4203D10397ADF80890A6E079E0BF
:10C6A0002078000776D598B282088DF800A0ADF802
:10C6B0000420B0EB820F6DD10297ADF8061095E023
:10C6C0002178C90666D5022D64D381B206208DF883
:10C6D0000000707802285DD3B1FBF0F28DF8040001
:10C6E000ADF8062092B242438A4253D1ADF8089089
:10C6F0007BE0207880064DD5072003E020784006B7
:10C700007FD508208DF80000A088ADF80400ADF8B2
:10C710000620ADF8081068E02078000671D50920E1
:10C72000ADF804208DF80000ADF8061002975DE02A
:10C730002188C90565D5022D63D381B20A208DF801
:10C740000000707804285CD3C6E72088400558D5DF
:10C75000012D56D10B208DF80000A088ADF8040003
:10C7600044E021E026E016E0FFE72088000548D5F8
:10C77000052D46D30C208DF80000A088ADF80400EC
:10C78000B6F803006D1FADF80850ADF80600ADF81F
:10C790000AA02AE035E02088C00432D5012D30D12E
:10C7A0000D208DF8000021E02088800429D4B6F8FF
:10C7B0000100E080A07B000723D5032D21D3307832
:10C7C00000F03F001B2818D00F208DF800002088B3
:10C7D00040F40050A4F80000B6F80100ADF80400E1
:10C7E000ED1EADF80650ADF808B003976946059800
:10C7F000F5F792FB050008D016E00E208DF800003A
:10C80000EAE7072510E008250EE0307800F03F0049
:10C810001B2809D01D2807D0022005990BF04EF9DE
:10C82000208800F400502080A07B400708D52046D7
:10C83000FFF70BFDC00703D1A07B20F00400A0731D
:10C84000284685E61FB5022806D101208DF8000094
:10C8500088B26946F5F760FB1FBD0000F8B51D46BC
:10C86000DDE906470E000AD007F063FC2346FF1DF2
:10C87000BCB231462A46009407F071F8F8BDD019D1
:10C880002246194601F0D9FD2046F8BD2DE9FF4F9B
:10C890008DB09B46DDE91B57DDF87CA00C46082BCC
:10C8A00005D0E06901F0FEF850B11020D2E02888F0
:10C8B000092140F0100028808AF80010022617E0B5
:10C8C000E16901208871E2694FF420519180E169AA
:10C8D0008872E06942F601010181E06900218173FB
:10C8E0002888112140F0200028808AF800100426B2
:10C8F00038780A900A2038704FF0020904F11800C5
:10C900004D460C9001F0C6FBB04681E0BBF1100F24
:10C910000ED1022D0CD0A9EB0800801C80B20221A0
:10C92000CDE9001005AB52461E990D98FFF796FF12
:10C93000BDF816101A98814203D9F74800790F9074
:10C9400004E003D10A9808B138702FE04FF00201DB
:10C95000CDE900190DF1160352461E990D98FFF707
:10C960007DFF1D980088401B801B83B2C6F1FF002D
:10C97000984200D203461E990BA8D9B15FF000027D
:10C98000DDF878C0CDE9032009EB060189B2CDE9D5
:10C9900001C10F980090BDF8161000220D9801F00B
:10C9A0000EFC387070B1C0B2832807D0BDF81600F5
:10C9B00020833AE00AEB09018A19E1E7022011B06D
:10C9C000BDE8F08FBDF82C00811901F0FF08022DA1
:10C9D0000DD09AF80120424506D1BDF820108142C1
:10C9E00007D0B8F1FF0F04D09AF801801FE08AF851
:10C9F0000180C94800680178052902D1BDF81610E8
:10CA0000818009EB08001FFA80F905EB080085B268
:10CA1000DDE90C1005AB0F9A01F03FFB28B91D981A
:10CA20000088411B4145BFF671AF022D13D0BBF109
:10CA3000100F0CD1A9EB0800801C81B20220CDE9B7
:10CA4000000105AB52461E990D98FFF707FF1D9890
:10CA50000580002038700020B1E72DE9F8439C469E
:10CA6000089E13460027B26B9AB3491F8CB2F18F10
:10CA7000A1F57F45FF3D05D05518AD882944891D96
:10CA80008DB200E000252919B6F83C8008314145F7
:10CA900020D82A44BCF8011022F8021BBCF803106D
:10CAA00022F8021B984622F8024B914607F02FFB12
:10CAB0004FF00C0C41464A462346CDF800C006F024
:10CAC0001AFFF587B16B00202944A41D214408807A
:10CAD00003E001E0092700E083273846BDE8F8833A
:10CAE00010B50B88848F9C420CD9846BE0180488A5
:10CAF00044B1848824F40044A41D23440B801060B6
:10CB0000002010BD0A2010BD2DE9F0478AB0002595
:10CB1000904689468246ADF8185007274BE00598A5
:10CB200006888088000446D4A8F8006007A801950C
:10CB300000970295CDE903504FF40073002231466F
:10CB4000504601F03CFB04003CD1BDF81800ADF8A4
:10CB50002000059804888188B44216D10A0414D4B0
:10CB600001950295039521F400410097049541F445
:10CB7000804342882146504601F0BFF804000BD1A3
:10CB80000598818841F40041818005AA08A948469A
:10CB9000FFF7A6FF0400DCD00097059802950195E9
:10CBA000039504950188BDF81C300022504601F021
:10CBB000A4F80A2C06D105AA06A94846FFF790FF5B
:10CBC0000400ACD0ADF8185004E00598818821F439
:10CBD0000041818005AA06A94846FFF781FF002889
:10CBE000F3D00A2C03D020460AB0BDE8F08700201D
:10CBF000FAE710B50C46896B86B051B10C218DF85F
:10CC00000010A18FADF80810A16B01916946FAF7E9
:10CC100001FB00204FF6FF71A063E187A08706B0FB
:10CC200010BD2DE9F0410D460746896B0020069E98
:10CC30001446002911D0012B0FD13246294638461F
:10CC4000FFF762FF002808D1002C06D032462946A3
:10CC50003846BDE8F04100F034BFBDE8F0812DE971
:10CC6000FC411446DDE9087C0E46DDE90A15521D3B
:10CC7000BCF800E092B2964502D20720BDE8FC81E4
:10CC8000ACF8002017222A70A5F80160A5F803303F
:10CC90000522CDE900423B462A46FFF7DFFD002092
:10CCA000ECE770B50C46154648220021204601F0FD
:10CCB000EEFB04F1080044F81C0F00204FF6FF7152
:10CCC000E06161842084A5841720E08494F82A0020
:10CCD00040F00A0084F82A0070BD4FF6FF720A8007
:10CCE000014603200AF0EABE30B585B00C46054681
:10CCF000FFF77FFFA18E284629B101218DF8001092
:10CD00006946FAF787FA0020E0622063606305B0A5
:10CD100030BDB0F8400070476000002090F8462019
:10CD2000920703D4408808800020F4E70620F2E749
:10CD300090F846209207EED5A0F84410EBE70146A4
:10CD4000002009880A0700D5012011F0F00F01D05A
:10CD500040F00200CA0501D540F004008A0501D563
:10CD600040F008004A0501D540F010000905D2D571
:10CD700040F02000CFE700B5034690F84600C0071A
:10CD800001D0062000BDA3F842101846FFF7D7FFD8
:10CD900010F03E0F05D093F8460040F0040083F8F1
:10CDA000460013F8460F40F001001870002000BD47
:10CDB00090F84620520700D511B1B0F84200AAE71A
:10CDC0001720A8E710F8462F61F3C3020270A2E70C
:10CDD0002DE9FF4F9BB00E00DDE92B34DDE929780A
:10CDE000289D24D02878C10703D000F03F001928DF
:10CDF00001D9012100E000212046FFF7D9FFB04210
:10CE000015D32878410600F03F010CD41E290CD020
:10CE1000218811F47F6F0AD13A8842B1A1F57F428F
:10CE2000FF3A04D001E0122901D1000602D5042006
:10CE30001FB0C5E5FA491D984FF0000A08718DF83A
:10CE400018A08DF83CA00FAA0A60ADF81CA0ADF8A0
:10CE500050A02978994601F03F02701F5B1C04F135
:10CE6000180C4FF0060E4FF0040BCDF858C01F2AD7
:10CE70007ED2DFE802F07D7D107D267DAC7DF47DE5
:10CE8000F37DF27DF17DF47DF07D7D7DEF7DEE7DA6
:10CE90007D7D7D7DED0094F84610B5F80100890791
:10CEA00001D5032E02D08DF818B01EE34FF40061B7
:10CEB000ADF85010608003218DF83C10ADF84000B3
:10CEC000D4E2052EEFD1B5F801002083ADF81C00A7
:10CED000B5F80310618308B1884201D9012079E1D6
:10CEE0000020A07220814FF6FF702084169801F078
:10CEF000D1F8052089F800000220029083460AAB91
:10CF00001D9A16991B9801F0C8F890BB9DF82E0049
:10CF1000012804D0022089F80100102003E001203C
:10CF200089F8010002200590002203A90BA808F04F
:10CF30006AFDE8BB9DF80C00059981423DD1398816
:10CF4000801CA1EB0B01814237DB02990220CDE965
:10CF500000010DF12A034A4641461B98FFF77EFC6B
:10CF600002980BF1020B801C81B217AA029101E01A
:10CF70009CE228E003A90BA808F045FD02999DF862
:10CF80000C00CDE9000117AB4A4641461B98FFF75C
:10CF900065FC9DF80C000AAB0BEB00011FFA81FB4E
:10CFA00002991D9A084480B2029016991B9800E0DD
:10CFB00003E001F072F80028B6D0BBF1020F02D0F6
:10CFC000A7F800B04FE20A208DF818004BE20021CC
:10CFD0000391072EFFF467AFB5F801002083ADF889
:10CFE0001C00B5F80320628300283FF477AF90421D
:10CFF0003FF674AF0120A072B5F805002081002033
:10D00000A073E06900F04EFD78B9E16901208871F4
:10D01000E2694FF420519180E1698872E16942F63A
:10D0200001000881E06900218173F01F20841E98AF
:10D03000606207206084169801F02CF8072089F8B8
:10D0400000000120049002900020ADF82A0028E0A2
:10D0500019E29FE135E1E5E012E2A8E080E043E07B
:10D060000298012814D0E0698079012803D1BDF825
:10D070002800ADF80E00049803ABCDE900B04A4695
:10D0800041461B98FFF7EAFB0498001D80B204900C
:10D09000BDF82A00ADF80C00ADF80E00059880B27E
:10D0A00002900AAB1D9A16991B9800F0F6FF28B95A
:10D0B00002983988001D05908142D1D2029801283A
:10D0C00081D0E0698079012803D1BDF82800ADF84E
:10D0D0000E00049803ABCDE900B04A4641461B98C8
:10D0E000FFF7BCFB0298BDE1072E02D0152E7FF49E
:10D0F000DAAEB5F801102183ADF81C10B5F80320A5
:10D10000628300293FF4EAAE91423FF6E7AE012187
:10D11000A1724FF0000BA4F808B084F80EB0052EF1
:10D1200007D0C0B2691DE26908F06BFC00287FF4EB
:10D130004AAF4FF6FF70208401A906AA14A8CDF8C3
:10D1400000B081E885032878214600F03F031D9A4E
:10D150001B98FFF79BFB8246208BADF81C0082E1F9
:10D160000120032EC3D14021ADF85010B5F80110B5
:10D170002183ADF81C100AAAB8F1000F00D00023DB
:10D18000CDE9020304921D98CDF804800090388800
:10D190000022401E83B21B9801F011F88DF8180090
:10D1A00090BB0B2089F80000BDF8280035E04FF057
:10D1B000010C052E9BD18020ADF85000B5F8011070
:10D1C0002183B5F803002084ADF81C10B0F5007F72
:10D1D00003D907208DF8180087E140F47C422284AF
:10D1E0000CA8B8F1000F00D00023CDE90330CDE941
:10D1F000018C1D9800903888401E83B21B9800F067
:10D20000DEFF8DF8180018B18328A8D10220BFE0F6
:10D210000D2189F80010BDF83000401C22E100000B
:10D2200060000020032E04D248067FF53CAE0020AB
:10D2300018E1B5F80110ADF81C102878400602D5A9
:10D240008DF83CE002E007208DF83C004FF000082C
:10D250000320CDE902081E9BCDF810801D98019394
:10D26000A6F1030B00901FFA8BF342461B9800F0C7
:10D2700044FD8DF818008DF83C80297849060DD5BD
:10D280002088C00506D5208BBDF81C10884201D12E
:10D29000C4F8248040468DF81880E3E0832801D14B
:10D2A0004FF0020A4FF48070ADF85000BDF81C003A
:10D2B0002083A4F820B01E986062032060841321AC
:10D2C000CDE0052EFFF4EFADB5F80110ADF81C1060
:10D2D000A28F6AB3A2F57F43FE3B29D008228DF8C6
:10D2E0003C2000BF4FF0000B0523CDE9023BDDF8E9
:10D2F00078C0CDF810B01D9A80B2CDF804C040F4CB
:10D3000000430092B5F803201B9800F0F6FC8DF85E
:10D310003CB04FF400718DF81800ADF85010832820
:10D3200010D0F8B1A18FA1F57F40FE3807D0DCE026
:10D330000B228DF83C204FF6FE72A287D2E7A4F8AC
:10D340003CB0D2E000942B4631461E9A1B98FFF762
:10D3500084FB8DF8180008B183284BD1BDF81C0060
:10D36000208353E700942B4631461E9A1B98FFF703
:10D3700074FB8DF81800E8BBE18FA06B0844831D97
:10D380008DE888034388828801881B98FFF767FC33
:10D39000824668E095F80180022E70D15FEA0800AD
:10D3A00002D0B8F1010F6AD109208DF83C0007A81E
:10D3B00000908DF840804346002221461B98FFF7DD
:10D3C00030FC8DF842004FF0000B8DF843B050B99F
:10D3D000B8F1010F12D0B8F1000F04D1A18FA1F55F
:10D3E0007F40FF380AD0A08F40B18DF83CB04FF499
:10D3F000806000E037E0ADF850000DE00FA91B9809
:10D40000F9F708FF82468DF83CB04FF48060ADF824
:10D410005000BAF1020F06D0FC480068C07928B16C
:10D420008DF8180027E0A4F8188044E0BAF1000F46
:10D4300003D081208DF818003DE007A800904346F6
:10D44000012221461B98FFF7ECFB8DF818002146BE
:10D450001B98FFF7CEFB9DF8180020B9192189F819
:10D460000010012038809DF83C0020B10FA91B98C6
:10D47000F9F7D0FE8246BAF1000F33D01BE018E076
:10D480008DF818E031E02078000712D5012E10D178
:10D490000A208DF83C00E088ADF8400003201B997D
:10D4A0000AF00CFB0820ADF85000C0E648067FF5F6
:10D4B000FAAC4FF0040A2088BDF8501008432080D1
:10D4C000BDF8500080050BD5A18FA1F57F40FE3837
:10D4D00006D11E98E06228982063A6864FF0030AC2
:10D4E0005046A5E49DF8180078B1012089F80000A5
:10D4F000297889F80110BDF81C10A9F802109DF8D0
:10D50000181089F80410052038802088BDF85010C4
:10D5100088432080E4E72DE9FF4F8846087895B0DE
:10D52000012181404FF20900249C0140ADF82010F8
:10D530002088DDF88890A0F57F424FF0000AFF3A7E
:10D5400006D039B1000705D5012019B0BDE8F08F2C
:10D550000820FAE7239E4FF0000B0EA886F800B0D3
:10D5600018995D460988ADF83410A8498DF81CB0AB
:10D57000179A0A718DF838B0086098F800000128F1
:10D580003BD0022809D003286FD1307820F03F002B
:10D590001D303070B8F80400E08098F800100320C7
:10D5A000022904D1317821F03F011B31317094F808
:10D5B0004610090759D505ABB9F1000F13D000216A
:10D5C00002AA82E80B000720CDE90009BDF834006B
:10D5D000B8F80410C01E83B20022159800F0EFFDC9
:10D5E0000028D1D101E0F11CEAE7B8F80400A6F860
:10D5F0000100BDF81400C01C04E198F805108DF876
:10D600001C1098F80400012806D04FF4007A022874
:10D610002CD00328B8D16CE12188B8F8080011F4A7
:10D620000061ADF8201020D017281CD3B4F84010AA
:10D63000814218D3B4F84410172901D3814212D182
:10D64000317821F03F01C91C3170A6F80100032197
:10D65000ADF83410A4F8440094F8460020F002001D
:10D6600084F8460065E105257EE177E1208808F130
:10D67000080700F4FE60ADF8200010F0F00F1BD09A
:10D6800010F0C00F03D03888228B9042EBD199B9AB
:10D69000B878C00710D0B9680720CDE902B1CDF83D
:10D6A00004B00090CDF810B0FB88BA88398815987E
:10D6B00000F023FB0028D6D12398BDF82010401C91
:10D6C00080294ED006DC10290DD020290BD040290E
:10D6D00087D124E0B1F5807F6ED051457ED0B1F581
:10D6E000806F97D1DEE0C80601D5082000E0102049
:10D6F00082460DA907AA0520CDE902218DF8380040
:10D70000ADF83CB0CDE9049608A93888CDE9000110
:10D710005346072221461598FFF7B8F8A8E09DF870
:10D720001C2001214FF00A0A002A9BD105ABB9F158
:10D73000000F00D00020CDE902100720CDE900093C
:10D74000BDF834000493401E83B2218B002215984B
:10D7500000F035FD8DF81C000B203070BDF8140072
:10D7600020E09DF81C2001214FF00C0A002A22D154
:10D7700013ABB9F1000F00D00020CDE90210072053
:10D78000CDE900090493BDF83400228C401E83B219
:10D79000218B159800F013FD8DF81C000D203070C2
:10D7A000BDF84C00401CADF8340005208DF8380061
:10D7B000208BADF83C00BCE03888218B88427FF498
:10D7C00052AF9DF81C004FF0120A00281CD1606A6D
:10D7D000A8B1B878C0073FF446AF00E018E0BA68D7
:10D7E0000720CDE902B2CDF804B00090CDF810B01A
:10D7F000FB88BA88159800F080FA8DF81C00132079
:10D8000030700120ADF8340093E00000600000208B
:10D810003988208B8142D2D19DF81C004FF0160A26
:10D820000028A06B08D0E0B34FF6FF7000215F46E0
:10D83000ADF808B0019027E068B1B978C907BED14A
:10D84000E18F0DAB0844821D03968DE80C024388DE
:10D850008288018809E0B878C007BCD0BA680DABEF
:10D8600003968DE80C02BB88FA881598FFF7F7F944
:10D8700005005ED0072D72D076E0019005AA02A9BE
:10D880002046FFF72DF90146E28FBDF808008242DD
:10D8900001D00029F1D0E08FA16B084407800198E6
:10D8A000E08746E09DF81C004FF0180A40B1208B3D
:10D8B000C8B13888208321461598FFF79AF938E0D7
:10D8C00004F118000090237E012221461598FFF7ED
:10D8D000A8F98DF81C000028EDD119203070012026
:10D8E000ADF83400E7E7052521461598FFF781F9E3
:10D8F0003AE0208800F40070ADF8200050452DD1AA
:10D90000A08FA0F57F41FE3901D006252CE0D8F884
:10D9100008004FF0160A48B1A063B8F80C10A187B0
:10D920004FF6FF71E187A0F800B002E04FF6FF70FC
:10D93000A087BDF8200030F47F611AD07823002240
:10D94000032015990AF010F898F80000207120883B
:10D95000BDF82010084320800EE000E00725208855
:10D96000BDF8201088432080208810F47F6F1CD0E1
:10D970003AE02188814321809DF8380020B10EA92A
:10D980001598F9F747FC05469DF81C000028EBD0D8
:10D9900086F801A001203070208B70809DF81C005B
:10D9A00030710520ADF83400DEE7A18EE1B11898A2
:10D9B0000DAB0088ADF834002398CDE90304CDE920
:10D9C0000139206B0090E36A179A1598FFF700FA67
:10D9D000054601208DF838000EA91598F9F71AFCB4
:10D9E00000B10546A4F834B094F8460040070AD5C3
:10D9F0002046FFF7A4F910F03E0F04D114F8460FAB
:10DA000020F0040020701898BDF8341001802846DA
:10DA10009BE500B585B0032806D102208DF80000F3
:10DA200088B26946F9F7F6FB05B000BD10B5384C71
:10DA30000B782268012B02D0022B2AD111E0137837
:10DA40000BB1052B01D10423137023688A889A80B7
:10DA50002268CB88D38022680B8913814989518140
:10DA60000DE08B8893802268CB88D38022680B8955
:10DA700013814B8953818B899381096911612168D5
:10DA8000F9F7C8FB226800210228117003D0002892
:10DA900000D0812010BD832010BD806B002800D0F5
:10DAA000012070478178012909D10088B0F5205FF5
:10DAB00003D042F60101884201D1002070470720BF
:10DAC0007047F0B587B0002415460E460746ADF8FE
:10DAD000184011E005980088288005980194811D60
:10DAE000CDE902410721049400918388428801888E
:10DAF000384600F002F930B905AA06A93046FEF70B
:10DB0000EFFF0028E6D00A2800D1002007B0F0BDC2
:10DB10006000002010B58B7883B102789A4205D15D
:10DB20000B885BB102E08B79091D4BB18B789A426F
:10DB3000F9D1B0F801300C88A342F4D1002010BD17
:10DB4000812010BD072826D012B1012A27D103E079
:10DB5000497801F0070102E04978C1F3C2010529C3
:10DB60001DD2DFE801F00318080C12000AB10320EF
:10DB700070470220704704280DD250B10DE00528EF
:10DB800009D2801E022808D303E0062803D0032808
:10DB900003D005207047002070470F207047812078
:10DBA0007047C0B282060BD4000607D5FA48807AC7
:10DBB0004143C01D01EBD00080B27047084670475A
:10DBC0000020704770B513880B800B781C0625D594
:10DBD000F14CA47A844204D843F01000087000206D
:10DBE00070BD956800F0070605EBD0052D78F5406F
:10DBF00065F304130B701378D17803F0030341EA43
:10DC0000032140F20123B1FBF3F503FB15119268E8
:10DC1000E41D00FB012000EBD40070BD906870BDD6
:10DC200037B51446BDF804101180117841F0040195
:10DC300011709DF804100A061ED5D74AA368C1F3D7
:10DC40000011927A824208D8FE2811D1D21DD20842
:10DC50004942184600F01BFC0AE003EBD00200F03A
:10DC60000703012510789D40A84399400843107090
:10DC7000207820F0100020703EBD2DE9F0410746CD
:10DC8000C81C0E4620F00300B04202D08620BDE83A
:10DC9000F081C14D002034462E60AF802881AA72E9
:10DCA000E8801AE0E988491CE980810614D4E1780B
:10DCB00000F0030041EA002040F20121B0FBF1F244
:10DCC00001FB12012068FFF76CFF2989084480B22C
:10DCD0002881381A3044A0600C3420784107E1D400
:10DCE0000020D4E7AC4801220189C08800EB400045
:10DCF00002EB8000084480B270472DE9FF4F89B0E5
:10DD00001646DDE9168A0F46994623F44045084633
:10DD100000F054FB040002D02078400703D4012017
:10DD20000DB0BDE8F08F099806F086F802902078D3
:10DD3000000606D59848817A0298814201D887204A
:10DD4000EEE7224601A90298FFF73CFF8346002038
:10DD50008DF80C004046B8F1070F1AD00122214679
:10DD6000FFF7F0FE0028DBD12078400611D5022015
:10DD70008DF80C00ADF81070BDF80400ADF812007D
:10DD8000ADF814601898ADF81650CDF81CA0ADF899
:10DD900018005FEA094004D500252E46A846012751
:10DDA0000CE02178E07801F0030140EA012040F224
:10DDB0000121B0FBF1F2804601FB12875FEA494086
:10DDC00009D5B84507D1A178207901F0030140EACF
:10DDD0000120B04201D3BE4201D90720A0E7A81913
:10DDE0001FFA80F9B94501D90D2099E79DF80C007B
:10DDF00028B103A90998F9F70BFA002890D1B84582
:10DE000007D1A0784FEA192161F30100A07084F8CE
:10DE100004901A9800B10580199850EA0A0027D09A
:10DE2000199830B10BEB06002A46199900F005FB52
:10DE30000EE00BEB06085746189E099806F067F9A6
:10DE40002B46F61DB5B239464246009505F053FD06
:10DE5000224601A90298FFF7B5FE9DF8040022466C
:10DE600020F010008DF80400DDE90110FFF7D8FE66
:10DE7000002055E72DE9FF4FDFF81C91824685B061
:10DE8000B9F80610D9F8000001EB410100EB81045C
:10DE900040F20120B2FBF0F1174600FB1175DDE9FD
:10DEA000138B4E4629460698FFF77BFE0346FFF785
:10DEB00019FF1844B1880C30884202D9842009B077
:10DEC0002FE70698C6B2300603D5B00601D5062066
:10DED000F5E7B9F80620521C92B2A9F80620BBF16A
:10DEE000000F01D0ABF80020B00602D5C4F80880BE
:10DEF0000AE0B9F808201A4492B2A9F80820D9F823
:10DF00000000891A0844A0602246FE200699FFF707
:10DF100087FEE77025712078390A61F301002A0A2B
:10DF2000A17840F0040062F30101A17020709AF81A
:10DF300002006071BAF80000E08000252573300609
:10DF400002D599F80A7000E00127B00601D54FF01C
:10DF500000084E4600244FF007090FE0CDE90258B3
:10DF60000195CDF800900495F1882046129B089AFF
:10DF7000FFF7C3FE0028A2D1641CE4B2BC42EDD37B
:10DF800000209CE700B5FFF7ADFE03490C308A88FE
:10DF9000904203D9842000BD00060020CA8808688A
:10DFA00002EB420300EB8300521C037823F00403CE
:10DFB0000370CA80002101730846ECE72DE9F047A1
:10DFC000804600F0FBF9070005D000264446F74DD7
:10DFD00040F2012916E00120BDE8F087204600F05C
:10DFE000EDF90278C17802F0030241EA0222B2FBA5
:10DFF000F9F309FB13210068FFF7D3FD3044641CDB
:10E0000086B2A4B2E988601E8142E7DCA8F1010073
:10E01000E8802889801B288100203870DCE710B553
:10E02000144631B1491E218005F006FFA070002082
:10E0300010BD012010BD70B50446DC48C1880368DE
:10E0400001E0401C20802088884207D200EB40027B
:10E0500013EB820202D015786D07F2D580B28842A8
:10E0600016D2AAB15079A072D08820819178107907
:10E0700001F0030140EA0120A081A078E11CFFF734
:10E08000A1FD20612088401C2080E080002070BD20
:10E090000A2070BD0121018270472DE9FF4F85B034
:10E0A0004FF6FF798246A3F8009048681E460D4659
:10E0B00080788DF8060048680088ADF804000020DC
:10E0C0008DF80A00088A0C88A04200D304462C82EE
:10E0D00051E03878400708D4641C288AA4B2401C58
:10E0E000288208F10100C0B246E0288A401C28823C
:10E0F000781D6968FFF70EFDD8BB3188494501D10D
:10E10000601E30803188A1EB080030806888A04212
:10E1100038D3B878397900F0030041EA002801A922
:10E12000781DFFF7F7FC20BB298949452ED0002236
:10E1300039460798FFF706FDD8B92989414518D116
:10E14000E9680391B5F80AC0D7F808B05046CDF891
:10E1500000C005F0DCFFDDF800C05A460CF1070CEA
:10E160001FFA8CFC43460399CDF800C005F08DFBE7
:10E1700060B1641CA4B200208046204600F01EF965
:10E180000700A6D1641E2C820A2098E67480787954
:10E19000B071F888B0803978F87801F0030140EA6E
:10E1A00001207081A6F80C80504605F045FE3A46E5
:10E1B00006F10801FFF706FD306100207FE62DE93A
:10E1C000FF4F87B081461C469246DDF860B0DDF80F
:10E1D0005480089800F0F2F8050002D02878400733
:10E1E00002D401200BB09CE5484605F025FE2978B5
:10E1F000090605D56D49897A814201D88720F1E762
:10E20000CAF309062A4601A9FFF7DCFC0746149861
:10E2100007281CD000222946FFF794FC0028E1D1F2
:10E220002878400613D501208DF808000898ADF82D
:10E230000C00BDF80400ADF80E00ADF81060ADF8AC
:10E24000124002A94846F8F7E3FF0028CAD129780E
:10E25000E87801F0030140EA0121AA78287902F068
:10E26000030240EA0220564507D0B1F5007F04D9E9
:10E27000611E814201DD0B20B4E7864201D90720EF
:10E28000B0E7801B85B2A54200D92546BBF1000F3F
:10E2900001D0ABF80050179818B1B9192A4600F010
:10E2A000CCF8B8F1000F0DD03E4448464446169FC6
:10E2B00005F03FFF2146FF1DBCB232462B460094BD
:10E2C00005F04DFB00208DE72DE9F04107461D4686
:10E2D0001646084600F072F8040002D02078400785
:10E2E00001D40120D3E4384605F0A6FD21780906C3
:10E2F00005D52E49897A814201D88720C7E4224674
:10E300003146FFF75FFC65B12178E07801F0030149
:10E3100040EA0120B0F5007F01D8012000E0002094
:10E3200028700020B3E42DE9F04107461D4616464B
:10E33000084600F043F8040002D02078400701D4DA
:10E340000120A4E4384605F077FD2178090605D5BB
:10E350001649897A814201D8872098E422463146BD
:10E36000FFF75EFCFF2D14D02178E07801F0030266
:10E3700040EA022040F20122B0FBF2F302FB13005C
:10E3800015B900F2012080B2E070000A60F30101CB
:10E39000217000207BE410B50C4600F00FF810B19E
:10E3A0000178490704D4012010BD000000060020B8
:10E3B000C18821804079A0700020F5E70749CA880C
:10E3C000824209D340B1096800EB40006FF00B02B4
:10E3D00002EB8000084470470020704700060020D0
:10E3E00070B504460D4621462B460AB9002070BD83
:10E3F00001E0491C5B1C501E021E03D008781E78E9
:10E40000B042F6D008781E78801BF0E730B50C4695
:10E4100001462346051B954206D202E0521E9D5C32
:10E420008D54002AFAD107E004E01D780D70491CD4
:10E430005B1C521E002AF8D130BDF0B50E460146D5
:10E44000334680EA030404F00304B4B906E002B9D9
:10E45000F0BD13F8017B01F8017B521E01F00307A8
:10E46000002FF4D10C461D4602E080CD80C4121F5F
:10E47000042AFAD221462B4600BF04E013F8014BD0
:10E4800001F8014B521E002AF8D100BFE0E7F0B5B9
:10E490000C460146E6B204E002B9F0BD01F8016B9A
:10E4A000521E01F00307002FF6D10B46E5B245EAF4
:10E4B000052545EA054501E020C3121F042AFBD2C9
:10E4C000194602E001F8016B521E002AFAD100BF82
:10E4D000E3E7000010B509F0A0FDF4F7F9F909F041
:10E4E000E7FBBDE8104009F0AFBC302834BF012085
:10E4F00000207047202834BF4FF0A0420C4A01236F
:10E5000000F01F0003FA00F0002914BFC2F80C0548
:10E51000C2F808057047202834BF4FF0A0410449D5
:10E5200000F01F00012202FA00F0C1F81805704740
:10E530000003005070B50346002002466FF02F051F
:10E540000EE09C5CA4F130060A2E02D34FF0FF309F
:10E5500070BD00EB800005EB4000521C2044D2B29D
:10E560008A42EED370BD30B50A230BE0B0FBF3F462
:10E5700003FB1404B0FBF3F08D183034521E05F881
:10E58000014CD2B2002AF1D130BD30B500234FF694
:10E59000FF7510E0040A44EA002084B2C85C6040C1
:10E5A000C0F30314604005EA00344440E0B25B1C51
:10E5B00084EA40109BB29342ECD330BD2DE9F04188
:10E5C000FE4B0026012793F864501C7893F868C02E
:10E5D000B8B183F89140A3F8921083F8902083F8A3
:10E5E0008E70BCF1000F0CBF83F8946083F89450D8
:10E5F000F3488068008805F08AFDBDE8F04105F029
:10E6000021BA4FF6FF7083F89140A3F8920083F887
:10E61000902083F88E70BCF1000F14BF83F89450E3
:10E6200083F89460BDE8F0812DE9F041E44D29685C
:10E6300091F89C200024012A23D091F89620012AE9
:10E6400030D091F86C301422DC4E0127012B32D0EF
:10E6500091F88E30012B4FD091F8A620012A1CBFD3
:10E660000020BDE8F08144701F2200F8042B222214
:10E67000A731FFF7E2FE286880F8A6400120BDE838
:10E68000F08144701B220270D1F89D204260D1F8C5
:10E69000A120826091F8A520027381F89C4001209E
:10E6A000BDE8F081447007220270D1F898204260E2
:10E6B00081F89640E2E78046447000F8042B20225F
:10E6C0006E31FFF7BAFE88F80870286880F86C4051
:10E6D00090F86E000028D1D1B6F87000A6F8980026
:10E6E000A868417B86F89A1086F89670008805F035
:10E6F0000EFD05F0B6F9C1E791F86C30012B0BD097
:10E70000447017220270D1F890204260B1F8942032
:10E71000028181F88E40B1E78046447000F8042BF6
:10E7200020226E31FFF789FE88F80870286880F88B
:10E730006C4090F86E000028A0D1CDE7A04800689A
:10E7400090F86C10002914BFB0F870004FF6FF70FD
:10E75000704770B59A4C06462068002808BFFFDF56
:10E760000025206845706660002808BFFFDF20682C
:10E77000417800291CBFFFDF70BDCC220021FFF7CC
:10E7800086FE2068FF2101707F2180F83810132158
:10E790004184282180F86910012180F85C1080F8FC
:10E7A00061500AF0C1F9BDE8704009F0AEBA844981
:10E7B0000968097881420CBF012000207047804819
:10E7C000006890F82200C0F3400070477C48006861
:10E7D00090F8220000F0010070477948006890F836
:10E7E0002200C0F3001070472DE9F0437448002464
:10E7F000036893F82400B3F822C0C0F38001C0F38B
:10E800004002114400F001000844CCF3001121B390
:10E81000BCF1100F02BF6B4931F81000BDE8F08366
:10E82000BCF1120F18BFBCF1130F0ED0BCF1150FC5
:10E830001EBFFFDF2046BDE8F0830021624A32F8A8
:10E84000102010FB0120BDE8F083604A002132F85F
:10E85000102010FB0120BDE8F08393F85E2093F8B0
:10E860005F102E264FF47A774FF014084FF04009CE
:10E87000022A04BF4AF2D745B5FBF7F510D0012AAA
:10E8800004BF4AF22F75B5FBF7F510D04AF62315F1
:10E89000B5FBF7F5082A08BF4E4613D0042A18D056
:10E8A0002646082A0ED0042A13D0022A49D004F1A1
:10E8B0002806042A0FD0082A1CBF4FF01908082286
:10E8C00004D00AE04FF0140806F5A8764FF0400295
:10E8D00003E006F5A8764FF0100218FB026212FB67
:10E8E0000052C0EB00103A4D00EB800005EB8000B9
:10E8F00010441CF0010F4FF4C8724FF4BF7504BFF1
:10E90000CCF34006002E65D0CCF3400600F5A57090
:10E91000EEB1082904BF174640260CD0042904BFD5
:10E920002F46102607D0022907BF04F11807042636
:10E9300004F12807082606EB860808EB86163E44F5
:10E940001BE004F118064FF019080422C5E7082956
:10E9500004BF164640270CD0042904BF2E461027BA
:10E9600007D0022907BF04F11806042704F128067E
:10E97000082707EB871706EB8706304400F19C0653
:10E9800093F8690001F00C07002F08BF0020304405
:10E9900018BF00F5416027D1082904BF164640275B
:10E9A0001BD0042904BF2E46102716D0022906BF0B
:10E9B00004F11806042704F128060CE00C060020D8
:10E9C00068000020DC610200E4610200D461020002
:10E9D000D4FEFFFF64E018BF0827C7EBC70707EBAB
:10E9E000470706EB4706304498301CF0010F17D05C
:10E9F000082908BF40210CD0042904BF2A46102151
:10EA000007D0022907BF04F11802042104F12802EB
:10EA1000082101EB410303EB0111114408443BE0E1
:10EA2000082904BF944640260CD0042904BFAC46F4
:10EA3000102607D0022907BF04F1180C042604F1A0
:10EA4000280C082606EB8616B3F840300CEB860C33
:10EA50006044EB2B20D944F2552C0B3303FB0CF311
:10EA60009B0D082907D0042902D0022905D008E00F
:10EA70002A46102108E0402106E004F11802042192
:10EA800002E004F12802082101EB811102EB81016F
:10EA900001F5A57103FB010000F5B470BDE8F0833A
:10EAA00000F5A570082904BF944640260CD004291F
:10EAB00004BFAC46102607D0022907BF04F1180C8A
:10EAC000042604F1280C082606EB8616B3F8483015
:10EAD0000CEB860C6044EB2BDED944F2552C0B3347
:10EAE00003FB0CF39B0D0829C5D00429C0D00229D3
:10EAF000C7D1C2E7FE4840F271210068806A4843EE
:10EB00007047FB48006890F83700002818BF0120C4
:10EB1000704710B5F74C207B022818BF032808D196
:10EB2000207D04F115010EF0E6FE08281CBF01202F
:10EB300010BD207B002816BF022800200120BDE860
:10EB400010400AF021BDEB4908737047E849096895
:10EB500081F8300070472DE9F047E54C2168087BCB
:10EB6000002816BF022800200120487301F10E0181
:10EB70000AF0F4FC2168087B022816BF0328012252
:10EB8000002281F82F204FF0080081F82D00487BEB
:10EB900001F10E034FF001064FF00007012804BFFA
:10EBA0005B7913F0C00F0AD001F10E03012804D1E4
:10EBB000587900F0C000402801D0002000E001207A
:10EBC00081F82E00002A04BF91F8220010F0040FF3
:10EBD00007D0087D01F115010EF08DFE216881F846
:10EBE0002D002068476007F0BFFA2168C14D4FF043
:10EBF0000009886095F82D000EF089FE804695F892
:10EC00002F00002818BFB8F1000F04D095F82D0090
:10EC10000EF0B1FC68B195F8300000281CBF95F8E3
:10EC20002E0000281DD0697B05F10E0001290ED0B1
:10EC300012E06E734A4605F10E0140460AF0E4FC0C
:10EC400095F82D1005F10E000EF063FF09E04079F4
:10EC500000F0C000402831D0394605F10E000AF01E
:10EC60000BFD2068C77690F8220010F0040F08BF53
:10EC7000BDE8F087002795F82D000EF017FD050080
:10EC800008BFBDE8F087102102F0C2F8002818BFC5
:10EC9000BDE8F08720683A4600F11C01C676284698
:10ECA0000AF0B2FC206800F11C0160680FF08EF8D9
:10ECB0006068BDE8F04701210FF0A3B80EF066FFD1
:10ECC0004A4605F10E010AF09FFCCAE7884A12681D
:10ECD000137B0370D2F80E000860508A888070475A
:10ECE00078B584490446824E407B087332682078A8
:10ECF00010706088ADF8000080B200F00101C0F330
:10ED0000400341EA4301C0F3800341EA8301C0F3B9
:10ED1000C00341EAC301C0F3001341EA0311C0F389
:10ED2000401341EA4311C0F3801041EA801050843F
:10ED3000E07D012808BF012507D0022808BF022571
:10ED400003D0032814BFFFDF0825306880F85E5029
:10ED5000607E012808BF012507D0022808BF0225D0
:10ED600003D0032814BFFFDF0825316881F85F5006
:10ED700091F83500012829D0207B81F82400488CA7
:10ED80001D280CBF002060688862607D81F8370014
:10ED9000A07B002816BF0228002001200875D4F8A7
:10EDA0000F00C1F81500B4F81300A1F81900A07EF7
:10EDB00091F86B2060F3071281F86B20E07E012848
:10EDC00018BF002081F83400002078BD91F85E2043
:10EDD0000420082A08BF81F85E00082D08BF81F8CA
:10EDE0005F00C9E742480068408CC0F3001131B1B0
:10EDF000C0F38000002804BF1F20704702E0C0F36A
:10EE0000400109B10020704710F0010F14BFEE203F
:10EE1000FF20704736480068408CC0F3001119B1DC
:10EE2000C0F3800028B102E0C0F3400008B1002028
:10EE30007047012070472E49002209684A664B8CB2
:10EE40001D2B0CBF81F8682081F8680070470023F3
:10EE5000274A126882F85D30D164A2F85000012080
:10EE600082F85D007047224A0023126882F85C3005
:10EE7000A2F858000120516582F85C0070471C49D7
:10EE8000096881F8360070471949096881F86100FE
:10EE900070471748006890F961007047144800688F
:10EEA00090F82200C0F3401070471148006890F8B5
:10EEB0002200C0F3C0007047012070470C48006872
:10EEC00090F85F00704770B509F018FE09F0F7FD83
:10EED00009F0C0FC09F06CFD054C2068416E491C2E
:10EEE000416690F83300002558B109F01DFE03E09B
:10EEF000680000200C06002008F007FF206880F85A
:10EF000033502068457090F8391021B1BDE8704049
:10EF100004200AF0AEBF90F86810D9B1406E81426B
:10EF200018D804200AF0A5FF206890F8220010F0FD
:10EF3000010F07D0A06843220188BDE8704001207E
:10EF4000FFF73CBBBDE8704043224FF6FF71002045
:10EF5000FFF734BBBDE8704000200AF08ABF2DE9FE
:10EF6000F04782B00F468146FE4E4FF000083068F1
:10EF7000458C15F0030F10D015F0010F05F00200BD
:10EF800005D0002808BF4FF0010806D004E0002893
:10EF900018BF4FF0020800D1FFDF4FF0000A5446BF
:10EFA00015F0010F05F002000DD080B915F0040F27
:10EFB0000DD04AF00800002F1CBF40F0010040F0C7
:10EFC00002044DD09EE010B115F0040F0DD015F0E5
:10EFD000070F10D015F0010F05F0020043D00028F4
:10EFE00008BF15F0040F34D04AE0002F18BF4AF0D4
:10EFF000090444D141E037B14AF00800044615F055
:10F00000200F1BD07EE0316805F02002B1F84800E7
:10F01000104308BF4AF0010474D04AF018000446B7
:10F0200015F0200F6ED191F85E1011F00C0118BF91
:10F030000121C94361F30000044663E0316891F89F
:10F040005E1011F00C0118BF012161F300000446AD
:10F0500058E04AF00800002F18BF40F0010451D1D9
:10F0600040F010044EE0002818BF15F0040F07D040
:10F07000002F18BF4AF00B0444D14AF0180441E0B5
:10F0800015F0030F3DD115F0040F3AD077B1306879
:10F090004AF0080490F85E0010F00C0118BF01213E
:10F0A00061F3410415F0200F24D02BE0306805F007
:10F0B0002002B0F84810114308BF4AF0030421D0E1
:10F0C0004AF0180415F0200F0AD000BF90F85E0037
:10F0D00010F00C0018BF0120C04360F3410411E0A0
:10F0E00090F85E1011F00C0118BF0121C94361F3C3
:10F0F0000004EBE710F00C0018BF012060F30004DF
:10F1000000E0FFDF15F0400F1CD0CFB93168B1F837
:10F110004800002804BF488C10F0010F0BD110F0FC
:10F12000020F08BF10F0200F05D115F0010F08BF26
:10F1300015F0020F04D091F85E0010F00C0F01D111
:10F1400044F040047068A0F800A0017821F020018C
:10F1500001704FF007010EF005FE414670680EF099
:10F16000F8FF214670680FF000F814F0010F0CD082
:10F170004FF006034FF000027B4970680EF0CFFF9E
:10F180003068417B70680EF02FFE14F0020F18D02B
:10F19000D6E90010B9F1000F4FF006034FF001025D
:10F1A00007D01C310EF0BBFF012170680EF029FE64
:10F1B00007E015310EF0B3FF3068017D70680EF086
:10F1C00020FE14F0040F18BFFFDF14F0080F19D051
:10F1D000CDF800A03068BDF800200223B0F86A1016
:10F1E00061F30B02ADF8002090F86B0003220109D7
:10F1F0009DF8010061F307108DF801006946706801
:10F200000EF08DFF012F62D13068B0F84810E1B3E5
:10F2100090F82200C0F34000B8BB70680EF095FF74
:10F22000401CC7B23068C7F1FF05B0F84820B0F8FD
:10F230005A10511AA942B8BF0D46AA423BD990F8BC
:10F24000220010F0010F36D144F0100421467068FE
:10F250000EF08BFFF81CC0B2ED1E284482B230685D
:10F26000B0F86A10436EC1F30B0151FA83F190F8C4
:10F2700060303E4F1944BC460023E1FB07C31B0925
:10F280006FF0240C03FB0C1100E020E080F860100C
:10F2900090F85F00012101F01FF90090BDF8000017
:10F2A0009DF80210032340EA01400190042201A9C5
:10F2B00070680EF034FF3068AAB2416C70680EF0CE
:10F2C00082FF3068B0F85A102944A0F85A1014F0A0
:10F2D000400F06D0D6E900100123062261310EF05E
:10F2E0001EFF14F0200F18BFFFDF0020002818BFFA
:10F2F000FFDF02B0BDE8F0872DE9F043194C89B07B
:10F300002068002808BFFFDF20684178002944D129
:10F310000178FF2941D0002680F83160A0F85A60BA
:10F32000867080F83960304609F062FB104802AD03
:10F3300000F1240191E80E1085E80E10D0E90D10BF
:10F34000CDE9061002A809F041FB08F0BCFF2068D7
:10F3500090F9610009F090F8064809F093F8064822
:10F360000CE00000680000201A06002053E4B36E91
:10F37000C8610200D0610200CD61020009F012FBF9
:10F38000606809F038FB206890F8240010F0010F45
:10F3900007D0252009F07EF80AE009B00C20BDE86E
:10F3A000F08310F0020F18BF262069D009F072F820
:10F3B000206890F85E10252008F043FF206880F850
:10F3C0002C6009F00FFB206890F85E10002009F017
:10F3D00028F90F21052008F0F8FF206890F82E107A
:10F3E000002901BF90F82F10002990F8220010F09A
:10F3F000040F74D006F0B8FE0546206829468068E0
:10F4000007F0AAFBDFF82884074690FBF8F008FB1A
:10F4100010704142284606F08EFB2168886097FBF9
:10F42000F8F04A68104448600EF062FA014620681D
:10F43000426891426ED8C0E90165FE4D4FF0010867
:10F4400095F82D000EF063FA814695F82F000127FC
:10F45000002818BFB9F1000F04D095F82D000EF068
:10F460008AF8A0B195F8300000281CBF95F82E004E
:10F47000002824D0687B05F10E01012815D019E081
:10F4800010F0040F14BF2720FFDF8FD190E73A461A
:10F490006F7305F10E0148460AF0B6F895F82D1085
:10F4A00005F10E000EF035FB09E0487900F0C000D0
:10F4B000402815D0414605F10E000AF0DDF820681D
:10F4C00090F8220010F0040F24D095F82D000EF0D3
:10F4D000EDF805001ED0102101F09AFC40B119E0B2
:10F4E0000EF054FB3A4605F10E010AF08DF8E6E7FE
:10F4F00020683A4600F11C01C77628460AF084F8D5
:10F50000206800F11C0160680EF060FC0121606859
:10F510000EF077FC2068417B0E3008F038FF206841
:10F5200090F85C1061B3B0F85810A0F84810416D25
:10F53000416490F82210C1F30011F1B9B0F86A00EB
:10F540000221C0F30B05ADF80050684607F0B0FF8C
:10F5500028B1BDF80000C0F30B00A84204D1BDF8EB
:10F560000000401CADF800002168BDF80000B1F8B3
:10F570006A2060F30B02A1F86A20206880F85C60C2
:10F58000206890F85D1039B1B0F85010A0F8401024
:10F59000C16CC16380F85D60B0F86A10426EC1F35F
:10F5A0000B0151FA82F190F86020DFF88CC211440F
:10F5B00063460022E1FB0C3212096FF0240302FBC8
:10F5C000031180F860100EF00CFA032160680EF051
:10F5D00090FA216881F8330009B00020BDE8F0837B
:10F5E0009649886070472DE9F043944C83B02268B7
:10F5F00092F831303BB1508C1D2808BFFFDF03B0BB
:10F60000BDE8F0435FE401260027F1B1054692F81A
:10F61000600008F03FFF206890F85F10FF2008F0BE
:10F6200010FE20684FF4A57190F85F20002009F0CB
:10F63000D4F8206890F8221011F0030F00F02C810C
:10F64000002D00F0238100F027B992F822108046A7
:10F65000D07EC1F30011002956D0054660680780AE
:10F66000017821F020010170518C132937D01FDC63
:10F67000102908BF022144D0122908BF062140D01A
:10F68000FFDF6C4D606805F10E010EF091FB697BA8
:10F6900060680EF0A9FB2068418C1D2918BF152950
:10F6A00063D0B0F84820416C60680EF0B6FB5CE0B7
:10F6B000152918BF1D29E3D14FF001010EF052FBAF
:10F6C0006068017841F020010170216885B11C312A
:10F6D0000EF07CFB012160680EF093FBD1E7002166
:10F6E0000EF040FB6068017841F020010170C8E72E
:10F6F00015310EF06BFB2068017D60680EF081FB18
:10F70000BFE70EF02FFBBCE70021FFF728FC606885
:10F71000C17811F03F0F28D0017911F0100F24D0DB
:10F720000EF01EFB2368024693F82410C1F38000FC
:10F73000C1F3400C604401F00101084493F82C101F
:10F74000C1F3800CC1F34005AC4401F001016144F8
:10F75000401AC1B293F85E0000F0BEFE0090032391
:10F760000422694660680EF0DAFC2068002590F8F3
:10F77000241090F82C0021EA000212F0010F18BFAB
:10F7800001250ED111F0020F04D010F0020F08BFB6
:10F79000022506D011F0040F03D010F0040F08BFAB
:10F7A0000425B8F1000F2BD0012D1BD0022D08BF6E
:10F7B00026201BD0042D14BFFFDF272016D0206881
:10F7C00090F85E10252008F03CFD206890F822108B
:10F7D000C1F3001169B101224FF49671002008F0C5
:10F7E000FCFF0DE0252008F055FEE8E708F052FE8A
:10F7F000E5E790F85E204FF49671002008F0EDFFE9
:10F80000206890F82C10294380F82C1090F82420C0
:10F8100032EA01011CD04670418C13292BD026DC22
:10F82000102904BF03B0BDE8F083122923D007E0FC
:10F8300040420F000C06002053E4B36E6800002025
:10F84000C1F30010002818BFFFDF03B0BDE8F0834C
:10F85000418C1D2908BF80F82C70DCD0C1F3001149
:10F86000002914BF80F8316080F83170D3E7152982
:10F8700018BF1D29DBD190F85E2003B04FF00101C5
:10F88000BDE8F043084609F094B900BF90F85F2046
:10F890000121084609F08DF92168002DC87E7CD031
:10F8A0004A8C3D46C2F34000002808BF47F00805D7
:10F8B00012F0400F18BF45F04005002819BFD1F8DD
:10F8C0003C90B1F84080D1F84490B1F8488060682D
:10F8D000072107800EF046FA002160680EF039FC1F
:10F8E000294660680EF041FC15F0080F17D020681B
:10F8F000BDF800100223B0F86A2062F30B01ADF8E6
:10F90000001090F86B00032201099DF8010061F3DB
:10F9100007108DF80100694660680EF000FC606811
:10F920000EF0DCFA2168C0F1FE00B1F85A20A8EB15
:10F9300002018142A8BF0146CFB2D019404544D24E
:10F9400045F0100160680EF010FC60680EF0C6FA19
:10F950002168C0F1FE00B1F85A10A8EB0101814204
:10F96000A8BF0146CFB260680EF0EFFB3844421CDE
:10F970002068B0F86A10436EC1F30B0151FA83F1AD
:10F9800090F86030FE4D1944AC460023E1FB05C3FE
:10F990004FEA131C6FF0240300E03CE00CFB031162
:10F9A00080F8601090F85F00012100F095FD009054
:10F9B000BDF800009DF80210032340EA01400190C9
:10F9C000042201A960680EF0AAFB216891F82200C8
:10F9D00010F0400F05D001230622613160680EF05F
:10F9E0009EFB20683A46B0F85A0000EB09016068B7
:10F9F0000EF0E9FB2068B0F85A103944A0F85A100C
:10FA000009F0BFFC002818BFFFDF20684670867031
:10FA100003B0BDE8F0830121FFF7A1FAF0E7D94870
:10FA200010B50068417841B90078FF2805D0002161
:10FA30000846FFF7D8FD002010BD09F05FF809F077
:10FA40003EF808F007FF08F0B3FF0C2010BD2DE9C9
:10FA5000F041CC4D0446174628680E4690F86C00DD
:10FA6000002818BFFFDF2868002F80F86E7018BFCD
:10FA7000BDE8F0812188A0F870106188A0F8861098
:10FA8000A188A0F88810E188A0F88A1094F888115D
:10FA900080F88C1090F82F10002749B1427B00F1BC
:10FAA0000E01012A04D1497901F0C001402935D065
:10FAB00090F8301041B1427B00F10E01012A04BFE1
:10FAC000497911F0C00F29D000F17A00F3F794FAC8
:10FAD0006868FF2E0178C1F380116176D0F80310B9
:10FAE000C4F81A10B0F80700E08328681ED0C0F8E8
:10FAF0008010E18BA0F8841000F17402511E304692
:10FB00000DF014FF002808BFFFDF286890F873107D
:10FB100041F0020180F87310BDE8F081D0F80E10BA
:10FB2000C0F87A10418AA0F87E10D1E7C0F8807042
:10FB3000A0F88470617E80F87310D4F81A104167C1
:10FB4000E18BA0F87810BDE8F08170B58D4C0125EF
:10FB5000206890F82200C0F3C00038B13C22FF2199
:10FB6000A068FFF774FF206880F86C50206890F858
:10FB7000220010F0010F1CBFA06801884FF03C026A
:10FB800012BF01204FF6FF710020FEF717FD20681D
:10FB900080F8395070BD7B49096881F832007047A0
:10FBA0002DE9F041774C0026206841780127354641
:10FBB000012906D0022901D003297DD0FFDFBDE84D
:10FBC000F081817802250029418C46D0C1F34002A2
:10FBD000002A08BF11F0010F6FD090F85F204FF09E
:10FBE00001014FF0000008F0E4FF216891F82200C5
:10FBF000C0F34000002814BF0C20222091F85F10B1
:10FC000008F01FFB2068457090F8330058B108F0E9
:10FC100068F8206890F85F0010F00C0F0CBF4020CF
:10FC2000452008F077FF206890F83400002818BFBE
:10FC300008F08FFF216891F85F0091F8691010F0CB
:10FC40000C0F08BF0021962008F0F6FE09F090FB8B
:10FC5000002818BFFFDFBDE8F081C1F3001282B1B8
:10FC600010293FD090F8330020B108F03AF8402036
:10FC700008F050FF206890F8221011F0040F36D0E1
:10FC800043E090F8242090F82C309A422AD1B0F822
:10FC90004800002808BF11F0010F05D111F0020F34
:10FCA00008BF11F0200F6FD04FF001014FF000009E
:10FCB000FFF799FC206801E041E035E0418C11F04C
:10FCC000010F04BFC1F34001002907D1B0F85A1059
:10FCD000B0F84820914218BFBDE8F08180F831703B
:10FCE000BDE8F081BDE8F041002101207BE490F8FF
:10FCF0003710012914BF0329102646F00E0190F891
:10FD00005E204FF0000008F054FF206890F83400A7
:10FD1000002818BF08F01DFF0021962008F08CFE77
:10FD200020684570BDE8F081B0F85A10B0F848007E
:10FD3000814242D0BDE8F0410121084653E4817878
:10FD4000D9B1418C11F0010F22D080F86C7090F87D
:10FD50006E20B0F870100120FEF730FC206845706E
:10FD600008F0CCFE08F0ABFE08F074FD08F020FEB1
:10FD7000BDE8F04103200AF07CB88178012004E05E
:10FD800053E4B36E6800002017E0BDE8F0412AE4B8
:10FD900011F0020F04BFFFDFBDE8F081B0F85A1088
:10FDA000B0F84000814208D001210846FFF71BFC53
:10FDB000216803204870BDE8F081BDE8F041FFF7FD
:10FDC00082B8FFF780B810B5FE4C206890F8341068
:10FDD00049B1383008F0CCFE18B921687F2081F88D
:10FDE000380008F0ACFE206890F8330018B108F035
:10FDF0009BFE07F08AFF0AF02EFCA8B1206890F85D
:10FE00002210C1F3001179B14078022818BFFFDF3A
:10FE100000210120FFF7E7FB2068417800291EBF81
:10FE200040780128FFDF10BDBDE81040FFF74BB858
:10FE30002DE9F047E34C0F4680462168B8F1030FE7
:10FE4000488C08BFC0F3400508D000F0010591F8C8
:10FE50003200002818BF4FF0010901D14FF000090E
:10FE600008F00CFB0646B8F1030F0CBF4FF0020878
:10FE70004FF0010835EA090008BFBDE8F0872068A7
:10FE800090F8330068B10DF08FFD38700146FF28FF
:10FE900007D06068C01C0DF060FD38780DF091FD52
:10FEA000064360680178C1F3801221680B7D9A4295
:10FEB00008D10622C01C1531FEF792FA002808BFAF
:10FEC000012000D000203978FF2906D0C8B9206869
:10FED00090F82D00884216D113E0A0B1616811F8A6
:10FEE000030BC0F380100DF006FD05460DF061FE1A
:10FEF00038B128460DF0DAFB18B1102100F088FF68
:10FF000008B1012000E00020216891F8221011F0D2
:10FF1000040F01D0F0B11AE0CEB9AB4890F8370029
:10FF2000002818BF404515D1616811F8030BC0F3D4
:10FF300080100DF0E0FC04460DF03BFE38B1204689
:10FF40000DF0B4FB18B1102100F062FF10B10120D8
:10FF5000BDE8F0870020BDE8F0872DE9F04F994D0E
:10FF6000044683B0286800264078022818BFFFDFC7
:10FF700028684FF07F0B90F8341049B1383008F002
:10FF8000F7FD002804BF286880F838B008F0D7FDD6
:10FF900068680DF009FF8046002C00F0458208F0EB
:10FFA00010FA002800F04082012400274FF0FF09DA
:10FFB000B8F1050F1ED1686890F8240000F01F000A
:10FFC000102817D9286890F8360098B18DF800905D
:10FFD00069460520FFF72CFF002800F025822868DD
:10FFE00080F8A64069682222A730C91CFEF725FACE
:10FFF00000F01ABA68680EF062F8002800F0148267
:020000040001F9
:100000004046DFF8C4814FF0030A062880F02182C1
:10001000DFE800F0FCFCFC03FCFB8DF80090694677
:100020000320FFF705FF002800F0F180296891F810
:10003000340010B191F89C00D8B12868817801296A
:100040004DD06868042107800DF08CFE08F10E0188
:1000500068680DF0ADFE98F80D1068680DF0C4FEEC
:100060002868B0F84020C16B68680DF0FAFE00F017
:1000700063B99DF8000081F89C400A7881F89D20C2
:10008000FF280FD001F19F029E310DF04FFC002898
:1000900008BFFFDF286890F89E1041F0020180F849
:1000A0009E100DE068680278C2F3801281F89E20ED
:1000B000D0F80320C1F89F20B0F80700A1F8A300F2
:1000C000286800F1A50490F838007F2808BFFFDFFA
:1000D000286890F83810217080F838B0ADE790F8B3
:1000E00022000721C0F3801938480479686869F351
:1000F000861407800DF036FE002168680EF029F89E
:10010000214668680EF031F80623002208F10E013E
:1001100068680EF004F82868417B68680DF064FE9A
:1001200068680DF0DBFE2968B1F84020C0F1FE01DF
:100130008A42B8BF1146CFB2BA423CD9F81EC7B204
:1001400044F0100B594668680EF00FF868680DF01F
:10015000FCFF384400F101082868B0F86A10426ECC
:10016000C1F30B0151FA82F190F86020184C0A4457
:10017000A4460023E2FB04C319096FF0240301FB2A
:10018000032180F8601090F85F004246012100F0E2
:10019000A3F90190BDF804009DF80610032340EA7E
:1001A00001400290042202A968680DF0B8FF594688
:1001B00068680DF0DAFFB9F1000F0FD0D5E9001033
:1001C000012307E0680000200C060020C86102003F
:1001D00053E4B36E062261310DF0A1FF28683A4660
:1001E000C16B68680DF0EFFF2868A0F85A70B0F88E
:1001F00040108F420CBF0121002180F8311009F01E
:10020000C0F8002818BFFFDF96E007E021E128686A
:100210008078002840F00A8100F006B98DF800903F
:1002200068680178C1F38019D0F803100191B0F823
:100230000700ADF8080069460520FFF7F9FD002822
:1002400028687DD0817800297CD090F85FB0D5E90E
:100250000104D0F80F10C4F80E10B0F8131061822A
:10026000417D2175817D6175B0F81710E182B0F88C
:1002700019106180B0F81B10A180B0F81D10E1804A
:1002800000F11F0104F1080015F085FE686890F880
:10029000241001F01F01217690F82400400984F811
:1002A000880184F864B084F865B01BF00C0F0CBFB3
:1002B0000021012104F130000EF0ABF92868002282
:1002C00090F8691084F8661090F8610084F867006F
:1002D0009DF80010A868FFF7BAFB022009F0C9FDDD
:1002E000B2480DF1040B08210468686807800DF01E
:1002F00039FD002168680DF02CFF214668680DF07B
:1003000034FF0623002208F10E0168680DF007FF94
:100310002868417B68680DF067FD494668680DF004
:1003200070FD06230122594668680DF0F8FE09F0B9
:1003300028F8002818BFFFDF286880F801A077E0C0
:100340006DE0FFE76868D5F808804FF00109027892
:1003500098F80D10C2F34012114088F80D10D0F833
:100360000F10C8F80E10B0F81310A8F81210417D45
:1003700088F81410817D88F81510B0F81710A8F8C7
:100380001610B0F81910A8F80210B0F81B10A8F851
:100390000410B0F81D10A8F8061000F11F0108F1B4
:1003A000080015F0F8FD686890F8241001F01F01AE
:1003B00088F8181090F824000021400988F8880176
:1003C00088F8649088F8659008F130000EF021F903
:1003D0002868002290F8691088F8661090F861008B
:1003E00088F867009DF80010A868FFF730FB2868C0
:1003F00080F86C4090F86E20B0F870100120FEF785
:10040000DDF82868477008F079FB08F058FB08F021
:1004100021FA08F0CDFA012009F02BFD08E090F850
:100420002200C0F3001008B1012601E0FEF74BFDE9
:10043000286890F8330018B108F076FB07F065FCE7
:1004400096B10AF008F960B100210120FFF7CBF85E
:1004500013E0286890F82200C0F300100028E5D0CF
:10046000E2E7FEF730FD08E028688178012904D131
:1004700090F85F10FF2007F0E4FE2868417800291B
:1004800019BF4178012903B0BDE8F08F40780328F7
:1004900018BFFFDF03B0BDE8F08F70B5444C0646CF
:1004A0000D462068807858B107F0F2FD21680346B8
:1004B000304691F85F202946BDE870400AF085BAC1
:1004C00007F0E6FD21680346304691F85E20294694
:1004D000BDE870400AF079BA78B50C460021009169
:1004E000082804BF4FF4C87040210DD0042804BF71
:1004F0004FF4BF70102107D0022807BF01F1180088
:10050000042101F128000821521D02FB01062848A0
:100510009DF80010006890F8602062F3050141F03A
:1005200040058DF8005090F85F00012829D002287E
:100530002ED004281CBF0828FFDF2FD025F0800014
:100540008DF80000C4EB041000EB80004FF01E019A
:1005500001EB800006FB04041648844228BFFFDF3D
:100560001548A0FB0410BDF80110000960F30C0150
:10057000ADF80110BDF800009DF8021040EA0140FE
:1005800078BD9DF8020020F0E0008DF80200D5E76C
:100590009DF8020020F0E000203004E09DF8020009
:1005A00020F0E00040308DF80200C7E7C86102008B
:1005B00068000020C4BF0300898888880023C383A3
:1005C000428401EBC202521EB2FBF1F1018470477A
:1005D0002DE9F04104460026D9B3552333224FF4C8
:1005E000FA4501297DD0022900F01481032918BFA2
:1005F000BDE8F08104F17001207B00F01F00207342
:1006000084F889605FF0000004EB000C9CF808C0DF
:1006100003EA5C05ACEB050C0CF0FF0C0CF03305A9
:1006200002EA9C0CAC440D180CEB1C1C0CF00F0CDB
:1006300085F814C04D7E401CAC44C0B281F819C08E
:100640000528E1D30CF0FF00252898BFBDE8F08114
:10065000DCE0FFE704F17005802200212846FDF769
:1006600016FFAE71EE712E736E73EE732E746E7193
:10067000AE76EE76212085F84000492085F84100CD
:10068000FE2085F874002588702200212046FDF7A1
:10069000FEFE2580012584F8645084F865502820EA
:1006A00084F86600002104F130000DF0B2FF1B2237
:1006B000A4F84E20A4F85020A4F85220A4F8542006
:1006C0004FF4A470A4F85600A4F8580065734FF4D2
:1006D00048606080A4F8F060A4F8F260A4F8F460C8
:1006E00000E023E0A4F8F660A4F8F86084F8FA606B
:1006F00084F8FD60A4F8066184F80461A4F8186128
:10070000A4F81A6184F8B66184F8B76184F8C0610E
:1007100084F8C16184F88C6184F88F6184F8A861E1
:10072000C4F8A061C4F8A461BDE8F081A4F8066132
:1007300084F8FB606088FE490144B1FBF0F1A4F845
:1007400090104BF68031A4F89210B4F806C0A4F8CB
:100750009860B4F89C704FEACC0C4743BCFBF0FCAB
:1007600097FBF0F70CF1010CA4F89C701FFA8CFCBD
:100770000CFB00F704F17001A4F89AC0B7F5C84F5C
:10078000C4BFACF1010CA1F82AC0B5FBF0FC0CF120
:10079000010CA1F830C000F5802C0CF5EE3CACF15A
:1007A0000105B5FBF0FCA1F820C0CD8B05FB00FCDA
:1007B000BCFBF0F0C8830846217B01F01F012173C8
:1007C0004676002104EB010C9CF808C003EA5C05A6
:1007D000ACEB050C0CF0FF0C0CF0330502EA9C0CA2
:1007E000AC4445180CEB1C1C0CF00F0C85F814C025
:1007F000457E491CAC44C9B280F819C00529E1D333
:100800000CF0FF00252898BFBDE8F081FFDFBDE8B0
:10081000F08100BFB4F8B011B4F8B4316288A4F824
:100820009860B4F89CC0DB000CFB02FCB3FBF1F356
:100830009CFBF1FC5B1CA4F89CC09BB203FB01FC7D
:1008400004F17000A4F89A30BCF5C84FC4BF5B1E19
:100850004385B5FBF1F35B1C0386438C01EBC303BB
:100860005B1EB3FBF1F30384C38B5A43B2FBF1F17C
:10087000C183BDE8F0812DE9F04104460025A1B314
:1008800055234FF4FA464FF0330C01297DD002294D
:1008900000F0E080032918BFBDE8F08104F170008A
:1008A000217B01F01F01217384F889500021621817
:1008B000127A03EA5205521BD2B202F033050CEA57
:1008C00092022A44451802EB121202F00F022A7516
:1008D000457E491C2A44C9B242760529E7D3D0B2E5
:1008E000252898BFBDE8F081B1E0FFE704F170066C
:1008F000802200213046FDF7CAFDB571F5713573D0
:100900007573F57335747571B576F576212086F8B3
:100910004000492086F84100FE2086F874002688B1
:10092000702200212046FDF7B2FD2680012684F8C2
:10093000646084F86560282084F86600002104F172
:1009400030000DF066FE1B22A4F84E20A4F85020C3
:10095000A4F85220A4F854204FF4A470A4F8560030
:10096000A4F858006673A4F8F850202084F8FA0020
:1009700084F8F050C4F8F45084F8245184F82551D8
:1009800084F82E5184F82F5100E005E084F81451CA
:1009900084F82051BDE8F081618865480844B0FBC7
:1009A000F1F0A4F890004BF68030A4F89200E288B1
:1009B000A4F89850B4F89C70D2004F43B2FBF1F207
:1009C00097FBF1F7521CA4F89C7092B202FB01F75E
:1009D00004F17000A4F89A20B7F5C84FC4BF521EA6
:1009E0004285B6FBF1F2521C028601F5802202F527
:1009F000EE32561EB6FBF1F20284C68B06FB01F204
:100A0000B2FBF1F1C1830146207B00F01F0020738F
:100A10004D7600202218127A03EA5205521BD2B2F8
:100A200002F033050CEA92022A440D1802EB12126E
:100A300002F00F022A754D7E401C2A44C0B24A764D
:100A40000528E7D3D0B2252898BFBDE8F081FFDFA5
:100A5000BDE8F081D0F81811628804F1700348896C
:100A6000C989A4F89850B4F89CC0C9000CFB02FCDA
:100A7000B1FBF0F19CFBF0FC491CA4F89CC089B2CE
:100A800001FB00FCA4F89A10BCF5C84FC4BF491E76
:100A90005985B6FBF0F1491C1986598C00EBC10150
:100AA000491EB1FBF0F11984D98B5143B1FBF0F031
:100AB000D883BDE8F0812DE9F003447E0CB1252CEC
:100AC00003D9BDE8F00312207047002A02BF0020BE
:100AD000BDE8F003704791F80DC01F260123154DA6
:100AE0004FF00008BCF1000F7AD0BCF1010F1EBF1F
:100AF0001F20BDE8F0037047B0F800C00A7C8F7B70
:100B000091F80F907A404F7C87EA090742EA072262
:100B100082EA0C0C5FF000070CF0FF0999FAA9F9C2
:100B20004FEA1C2C4FEA19699CFAACFC04E0000067
:100B3000FFDB050053E4B36E4FEA1C6C49EA0C2C52
:100B40000CEB0C1C7F1C9444FFB21FFA8CFC032F8F
:100B5000E2D38CEA020CFB4F0022ECFB0572120977
:100B60006FF0240502FB05C2D2B201EBD2078276F8
:100B700002F007053F7A03FA05F52F4218BFC27647
:100B80007ED104FB0CF2120C521CD2B25FF00004B6
:100B900000EB040C9CF814C094453CBFA2EB0C0283
:100BA000D2B212D30D194FF0000C2D7A03FA0CF7C4
:100BB0003D421CBF521ED2B2002A69D00CF1010C7A
:100BC0000CF0FF0CBCF1080FF0D304F1010C0CF099
:100BD000FF04052CDCD33046BDE8F0037047FFE787
:100BE00090F81AC00C7E474604FB02C2D54C4FF069
:100BF000000CE2FB054C4FEA1C1C6FF024040CFBBC
:100C00000422D2B201EBD204827602F0070C247ADD
:100C100003FA0CFC14EA0C0F1FBFC2764046BDE875
:100C2000F003704790F819C0B2FBFCF40CFB1422DF
:100C3000521CD2B25FF0000400EB040C9CF814C00C
:100C400094453CBFA2EB0C02D2B212D30D194FF067
:100C5000000C2D7A03FA0CF815EA080F1CBF521E7F
:100C6000D2B272B10CF1010C0CF0FF0CBCF1080F08
:100C7000F0D304F1010C0CF0FF04052CDCD3AAE73F
:100C800009E00CEBC401C1763846BDE8F0037047BB
:100C90000CEBC401C1764046BDE8F0037047AA4A98
:100CA000016812681140A94A126811430160704737
:100CB00030B4A749A44B00244FF0010C0A78521C11
:100CC000D2B20A70202A08BF0C700D781A680CFA8C
:100CD00005F52A42F2D0097802680CFA01F1514078
:100CE000016030BC704770B46FF01F02010C02EA63
:100CF00090251F23A1F5AA4054381CBFA1F5AA4096
:100D0000B0F1550009D0A1F52850AA381EBFA1F5B1
:100D10002A40B0F1AA00012000D100204FF0000CC1
:100D2000624601248CEA0106F6431643B6F1FF3F02
:100D300011D005F001064FEA5C0C4CEAC63C03F00A
:100D4000010652086D085B08641C42EAC632162C84
:100D5000E8DD70BC704770BC0020704790F804C09C
:100D60003CF01F011CBF0020704730B401785522B1
:100D700002EA5103C91AC9B201F03304332303EA6A
:100D800091012144447801EB111102EA5405641BDE
:100D9000E4B204F0330503EA94042C4404EB141485
:100DA00001F00F0104F00F040C448178C07802EACE
:100DB0005105491BC9B201F0330503EA91012944E9
:100DC00001EB111101F00F01214402EA5004001B54
:100DD000C0B200F0330403EA9000204400EB10108E
:100DE00000F00F00014402EA5C00ACEB0000C0B26E
:100DF00000F0330203EA9000104400EB101000F002
:100E00000F00084401288CBF0120002030BC70472F
:100E10000A000ED00123012A0BDB491EC9B210F8CB
:100E200001C0BCF1000F01D0002070475B1C934251
:100E3000F3DD01207047002A08BF70471144401EAF
:100E400012F0010F03D011F8013D00F8013F5208E4
:100E500008BF704711F8013C437011F8023D00F8DB
:100E6000023F521EF6D1704770B58CB000F11004ED
:100E70001D4616460DF1FF3C5FF0080014F8012CEA
:100E80008CF8012014F8022D0CF8022F401EF5D129
:100E900001F1100C6C460DF10F0108201CF8012C1B
:100EA0004A701CF8022D01F8022F401EF6D1204690
:100EB00013F01CFB7EB16A1E04F130005FF00801E4
:100EC00010F8013C537010F8023D02F8023F491E31
:100ED000F6D10CB070BD08982860099868600A982F
:100EE000A8600B98E8600CB070BD38B505460C469C
:100EF000684607F03DFE002808BF38BD9DF9002078
:100F00002272E07E607294F90A100020511A48BFE4
:100F1000494295F82D308B42C8BF38BDFF2B08BF22
:100F200038BDE17A491CC9B2E17295F82E30994278
:100F300003D8A17A7F2918BF38BDA2720020E072C1
:100F4000012038BD53E4B36E04620200086202005F
:100F5000740000200C2818BF0B2810D00D2818BFD3
:100F60001F280CD0202818BF212808D0222818BFFD
:100F7000232804D024281EBF2628002070474FF0C5
:100F8000010070470C2963D2DFE801F006090E1357
:100F9000161B323C415C484E002A5BD058E0072AC1
:100FA00018BF082A56D053E00C2A18BF0B2A51D07C
:100FB0004EE00D2A4ED04BE0A2F10F000C2849D98B
:100FC00046E023B1A2F110000B2843D940E0122AD9
:100FD00018BF112A3ED090F8380020B1122A37D31A
:100FE0001A2A37D934E0162A32D31A2A32D92FE0F6
:100FF000A2F10F0103292DD990F8380008B31B2A5C
:1010000028D925E0002B08BF042A21D122E013B102
:10101000062A1FD01CE0012A1AD11BE01C2A1CBF83
:101020001D2A1E2A16D013E01F2A18BF202A11D00D
:10103000212A18BF222A0DD0232A1CBF242A262A9F
:1010400008D005E013B10E2A04D001E0052A01D032
:1010500000207047012070472DE9F0410D460446FD
:10106000866805F02FFA58B905F07EF840F236711F
:1010700004F061FDA060204605F024FA0028F3D0BA
:1010800095B13046A16805F067FD00280CDD2844C5
:10109000401EB0FBF5F707FB05F1304604F04BFDB1
:1010A000A0603846BDE8F0810020BDE8F08170B551
:1010B0000446904228BF70BD101B64280BD325182E
:1010C0008D4206D8042105F07AFD00281CBF284671
:1010D00070BD204670BD6420F1E711F00C0F13D0F5
:1010E00001F0040100290DBF4022102296214FF487
:1010F000167101F5BC71A0EB010388428CBF93FB14
:10110000F2F0002080B27047022919BF6FF00D0184
:1011100001EBD0006FF00E0101EB9000F2E7084404
:1011200018449830002A14BF042100210844704755
:1011300010B4002A14BF4FF429624FF4A472002B9C
:1011400019BF4FF429634FF0080C4FF4A4734FF00C
:10115000010C00280CBF0124002491F866001CF04B
:101160000C0F08BF0020D11808449830002C14BF81
:1011700004210021084410BC704700280CBF012343
:10118000002391F86600002BA0F6482000F50050DF
:1011900018BF04231844496A81422CBF0120002053
:1011A00012F00C0118BF012131EA000014BF002029
:1011B0000120704710B413680B66137813F00C030A
:1011C00018BF0123527812F00C0218BF012253EA13
:1011D000020C04BF10BC7047002B0CBF4FF4A4736B
:1011E0004FF42963002A19BF4FF429624FF0080C0D
:1011F0004FF4A4724FF0010C00280CBF012400240E
:1012000091F866001CF00C0F08BF00201A4410442F
:101210009830002C14BF0422002210444A6A8242F3
:1012200024BF10BC704791F860004FF0030230F00B
:101230000C0381F8603091F8610020F00C0081F817
:10124000610008BF81F86020002808BF81F8612094
:1012500010BC704710F0010F1CBF0120704710F048
:10126000020F1CBF0220704710F0040018BF0820B6
:1012700070472DE9F0470446174689464FF00108AC
:1012800008460DF0FAF8054648460DF0FAF810F059
:10129000010F18BF012624D015F0010F18BF01233C
:1012A0002AD000BF56EA030108BF4FF0000810F033
:1012B000070F08BF002615F0070F08BF002394F89A
:1012C0006400B0420CBF00203046387094F86510BE
:1012D000994208BF00237B70002808BF002B25D14E
:1012E00015E010F0020F18BF0226D5D110F0040F40
:1012F00014BF08260026CFE715F0020F18BF0223FF
:10130000D0D115F0040F14BF08230023CAE74846C4
:101310000DF0BDF8B4F87010401A00B247F6FE7137
:10132000884201DC002801DC4FF0000816B1082ECD
:101330000CD018E094F86400012818BF022812D0DD
:1013400004281EBF0828FFDF032D0CD194F8C0012C
:1013500048B1B4F8C401012894F8640006D0082804
:1013600001D0082038704046BDE8F087042818BF37
:101370000420F7D1F5E7012814BF0228704710F0C8
:101380000C0018BF0420704738B4CBB2C1F3072C4F
:10139000C1B2C0F30724012B07D0022B09D0042BC4
:1013A00008BFBCF1040F2DD006E0BCF1010F03D142
:1013B00028E0BCF1020F25D0012906D0022907D070
:1013C000042908BF042C1DD004E0012C02D119E02F
:1013D000022C17D001EA0C0161F3070204EA0301B1
:1013E00061F30F22D1B211F0020F18BF022310D007
:1013F000C2F307218DF8003011F0020F18BF02214F
:101400001BD111E0214003EA0C03194061F30702EC
:10141000E6E711F0010F18BF0123E9D111F0040F25
:1014200014BF08230023E3E711F0010F18BF0121C7
:1014300003D111F0040118BF08218DF80110082B09
:1014400001BF000C012804208DF80000BDF8000049
:1014500038BC70474FF0000C082902D0042909D08D
:1014600011E001280FD10420907082F803C013808E
:1014700001207047012806D00820907082F803C030
:1014800013800120704700207047162A10D12A22AD
:101490000C2818BF0D280FD04FF0230C1F280DD09B
:1014A00031B10878012818BF002805D0162805D0CA
:1014B00000207047012070471A70FBE783F800C0D6
:1014C000F8E7012908D002290BD0042912BF082906
:1014D00040F6A660704707E0002804BF40F2E240F3
:1014E000704740F6C410704700B5FFDF40F2E2409D
:1014F00000BD00000178406829B190F82C1190F8E7
:101500008C0038B901E001F0BDBD19B1042901D04A
:10151000012070470020704770B50C460546062133
:1015200002F0C4FC606008B1002006E007212846F4
:1015300002F0BCFC606018B101202070002070BD7A
:10154000022070BD2DE9FC470C4606466946FFF7B0
:10155000E3FF00287DD19DF8000050B1FDF7EEF8C3
:10156000B0427CD0214630460AF008FC002873D1F6
:101570002DE00DF097F9B04271D02146304612F0BF
:10158000B6FA002868D1019D95F8F00022E001200C
:1015900000E00020804695F839004FF0010A4FF036
:1015A0000009F0B195F83A0080071AD584F8019047
:1015B00084F800A084F80490E68095F83B1021722E
:1015C000A98F6181E98FA18185F8399044E0019D5F
:1015D00095F82C0170350028DBD1287F0028D8D061
:1015E000D5E7304602F0A5FD070000D1FFDF384601
:1015F00001F0B5FF40B184F801900F212170E68021
:10160000208184F804A027E0304602F080FD070026
:1016100000D1FFDFB8F1000F21D0384601F0F7FF0D
:10162000B8B19DF8000038B90198D0F81801418888
:10163000B14201D180F80090304607F00DFF84F8E8
:1016400001900C21217084F80490E680697F21725A
:1016500000E004E085F81C900120BDE8FC87002034
:10166000FBE71CB56946FFF757FF00B1FFDF68468F
:1016700001F014FDFE4900208968A1F8F2001CBDAC
:101680002DE9FC4104460E46062002F0B7FB054654
:10169000072002F0B3FB2844C7B20025A8463E4409
:1016A00017E02088401C80B22080B04202D3404620
:1016B000A4F8008080B2B84204D3B04202D2002025
:1016C000BDE8FC816946FFF727FF0028F8D06D1CB4
:1016D000EDB2AE42E5D84FF6FF7020801220EFE762
:1016E00038B54FF6FF70ADF800000DE00621BDF8EB
:1016F000000002F0EDFB04460721BDF8000002F0F7
:10170000E7FB0CB100B1FFDF00216846FFF7B8FF2F
:101710000028EBD038BD70B507F00CFF0BF034FF9C
:10172000D44C4FF6FF76002526836683D2A0257021
:1017300001680079A4F14002657042F8421FA11CC3
:101740001071601C12F0EFFA1B2020814FF4A4717D
:101750006181A081E18107212177617703212174D3
:10176000042262746082A082A4F13E00E1820570CE
:101770004680BF480C300570A4F11000057046800B
:1017800084F8205070BD70B5B94C16460D466060A7
:10179000217007F047FEFFF7A3FFFFF7BCFF20789B
:1017A0000FF0BDFFB6480DF0D0F92178606812F057
:1017B0005FFA20780BF0DCF8284608F0AFFEB0485E
:1017C000FCF7C7FF217860680AF0B2FB3146207849
:1017D00012F024FDBDE870400BF0D6BE10B5012418
:1017E0000AB1002010BD21B1012903D000242046F8
:1017F00010BD02210CF024FDF9E710B50378044672
:10180000002B406813460A46014609D05FF00100EC
:10181000FFF78EFC6168496A884203D9012010BD38
:101820000020F5E7002010BD2DE9F04117468A7829
:101830001E46804642B11546C87838B1044669074D
:1018400006D52AB1012104E00725F5E70724F6E7CC
:101850000021620702D508B1012000E0002001420A
:1018600006D0012211464046FFF7C7FF98B93DE078
:1018700051B1002201214046FFF7BFFF58B9600770
:1018800034D50122114620E060B1012200214046FA
:10189000FFF7B3FF10B10920BDE8F081680725D537
:1018A000012206E068074FEA44700AD5002814DBDD
:1018B000002201214046FFF7A0FFB8B125F0040542
:1018C00014E0002812DA012200214046FFF795FFBC
:1018D00060B100BF24F0040408E001221146404634
:1018E000FFF78BFF10B125F00405F3E73D7034706E
:1018F0000020D1E770B58AB0044600886946FFF73A
:101900000BFE002806D1A08830B1012804D002289F
:1019100002D012200AB070BD04AB03AA214668466B
:10192000FFF782FF0500F5D19DF800100120002689
:101930000029019906D081F8C101019991F80C1292
:10194000B1BB2DE081F82F01019991F8561139B9F9
:10195000019991F82E1119B9019991F8971009B1CF
:101960003A2519E00199059681F82E01019A9DF812
:101970000C0082F83001019B9DF8102083F8312182
:10198000A388019CA4F832318DF814008DF815203D
:1019900005AA0020FFF70EFC019880F82F6126E0D1
:1019A000019991F8C01119B9019991F8971009B1ED
:1019B0003A2519E00199059681F8C00101989DF832
:1019C0000C2080F8C221019B9DF8100083F8C30110
:1019D000A388019CA4F8C4318DF814208DF815005B
:1019E00005AA0120FFF7E6FB019880F8C1612846AF
:1019F00090E710B504460020A17801B90120E278F3
:101A00000AB940F0020001F058FB002803D120463B
:101A1000BDE810406EE710BD70B5044691F8650052
:101A200091F866300D4610F00C0F00D1002321898B
:101A3000A088FFF774FB696A814229D2401A401CD2
:101A4000A1884008091A8AB2A2802189081A208137
:101A5000668895F864101046FFF73FFB864200D277
:101A600030466080E68895F8651020890AE000001D
:101A70007800002018080020FFFFFFFF1F00000073
:101A8000D8060020FFF729FB864200D23046E080CE
:101A900070BDF0B585B00D46064603A9FFF73CFDC5
:101AA00000282DD19DF80C0060B300220499FB2082
:101AB000B1F84E30FB2B00D30346B1F85040FB2069
:101AC000FB2C00D30446DFF85CC59CE88110009035
:101AD0000197CDF808C0ADF80230ADF80640684671
:101AE000FFF79AFF6E80BDF80400E880BDF808009B
:101AF0006881BDF80200A880BDF80600288100209A
:101B000005B0F0BD0122D1E72DE9F04186B00446D1
:101B100000886946FFF700FD002876D12189E0881A
:101B200001F0E4FA002870D1A188608801F0DEFAA3
:101B300000286AD12189E08801F0CFFA002864D119
:101B4000A188608801F0C9FA07005ED1208802A947
:101B5000FFF79FFF00B1FFDFBDF81010628809207A
:101B6000914252D3BDF80C10E28891424DD3BDF89A
:101B70001210BDF80E2023891144A2881A44914204
:101B800043D39DF80010019D4FF00008012640F658
:101B9000480041B185F8B761019991F8F81105F550
:101BA000DB7541B91AE085F82561019991F84A1170
:101BB00005F5927509B13A2724E0E18869806188CA
:101BC000E9802189814200D30146A980A188814210
:101BD00000D208462881012201990FE0E18869803E
:101BE0006188E9802189814200D30146A980A188CA
:101BF000814200D208462881019900222846FFF739
:101C00000BFF2E7085F80180384606B044E67BE76E
:101C100070B504460CF0FCFDB0B12078182811D145
:101C2000207901280ED1E088062102F03FF9040056
:101C300008D0208807F010FC2088062102F048F91F
:101C400000B1FFDF012070BDF74D28780028FAD0E1
:101C5000002666701420207020223146201DFCF7DB
:101C600016FC022020712E70ECE710B50446FCF73C
:101C7000DBFC002813D0207817280FD1207968B119
:101C8000E088072102F012F940B1008807F0E4FB78
:101C9000E088072102F01CF900B1FFDF012010BD30
:101CA0002DE9F0475FEA000800D1FFDFDE4802219E
:101CB0001A308146FFF7E4FC00B1FFDFDA4C062062
:101CC000678B02F09BF80546072002F097F828443E
:101CD000C5B2681CC6B2608BB04203D14046FFF764
:101CE000C4FF58B9608BA84203D14046FFF790FF6C
:101CF00020B9608B4146FFF725FC38B1404601F022
:101D000003FA0028E7D10120BDE8F0870221484608
:101D1000FFF7B6FC10B9608BB842DCD14046BDE895
:101D2000F04712F0C1BA10B501F053F908B10C2018
:101D300010BD0BF07DFC002010BD10B504460078EE
:101D400018B1012801D0122010BD01F053F920B1C3
:101D50000BF0C0FD08B10C2010BD207801F013F984
:101D6000E21D04F11703611CBDE810400BF0DABC62
:101D700010B5044601F02DF908B10C2010BD2078F3
:101D800028B1012803D0FF280BD0122010BD01F08C
:101D9000FAF8611C0BF00CFC08B1002010BD072004
:101DA00010BD01200BF03EFCF7E710B50BF095FDE0
:101DB00008B1002010BD302010BD10B5044601F060
:101DC00019F908B10C2010BD20460BF080FD002051
:101DD00010BD10B501F00EF920B10BF07BFD08B17C
:101DE0000C2010BD0BF0F6FC002010BDFF2181700F
:101DF0004FF6FF7181808D4949680A7882718A881F
:101E000002814988418101214170002070477CB5E1
:101E10000025022A19D015DC12F10C0F15D009DCAF
:101E200012F1280F11D012F1140F0ED012F1100F71
:101E300011D10AE012F1080F07D012F1040F04D0FB
:101E40004AB902E0D31E052B05D8012806D0022886
:101E500008D003280AD0122528467CBD1046FDF77D
:101E600013F8F9E710460CF06BFEF5E70846144648
:101E70006946FFF751FB08B10225EDE79DF8000028
:101E80000198002580F86740E6E710B51346012267
:101E9000FEF7EAFF002010BD10B5044610F02FFA3F
:101EA000052804D020460FF029FC002010BD0C208E
:101EB00010BD10B5044601F09DF808B10C2010BD0E
:101EC0002146002007F037FB002010BD10B5044666
:101ED0000FF0A3FC50B108F0A6FD38B1207808F04F
:101EE00029FB20780DF04DF9002010BD0C2010BD0D
:101EF00010B5044601F07EF808B10C2010BD214653
:101F0000012007F018FB002010BD38B504464FF63D
:101F1000FF70ADF80000A079E179884216D02079F1
:101F2000FCF7E3FA90B16079FCF7DFFA70B10022B8
:101F3000A079114612F0A0FD40B90022E0791146C7
:101F400012F09AFD10B9207A072801D9122038BD65
:101F500008F076FD60B910F0D2F948B90021684662
:101F6000FFF78EFB20B1204606F044F9002038BD73
:101F70000C2038BD2DE9FC41817805461A2925D071
:101F80000EDC16292ED2DFE801F02D2D2D2D2D216E
:101F90002D2D2D2D2D2D2D2D2D2D2D2D2D21212195
:101FA0002A291FD00BDCA1F11E010C291AD2DFE86F
:101FB00001F019191919191919191919190D3A399D
:101FC00004290FD2DFE801F00E020E022888B0F5D6
:101FD000706F07D201276946FFF79EFA20B10220F1
:101FE000BDE8FC811220FBE79DF8000000F0D2FF65
:101FF000019C10B104F58A7401E004F5C6749DF8E3
:10200000000000F0C7FF019E10B106F2151601E0B6
:1020100006F28D166846FFF76DFA08B1207838B1E0
:102020000C20DDE70C620200180800207800002078
:102030002770A8783070684601F030F80020CFE7AC
:102040007CB50D466946FFF767FA002618B12E6089
:102050002E7102207CBD9DF8000000F09BFF019CCA
:102060009DF80000703400F095FF019884F84260FC
:1020700081682960017B297194F842100029F5D10B
:1020800000207CBD10B5044600F0B4FF20B10BF079
:1020900021FC08B10C2010BD207800F074FFE2791B
:1020A000611C0BF093FD08B1002010BD022010BD93
:1020B00010B5886E60B1002241F8682F0120CA7106
:1020C0008979884012F0CCFC002800D01F2010BD78
:1020D0000C2010BD1CB50C466946FFF71DFA002800
:1020E00009D19DF8000000280198B0F8700000D0D8
:1020F000401C208000201CBD1CB504460088694699
